:10A1CF0020466F726D6174696E67204C6F674361D3
:10A1DF0072642E2E2E2000506C6561736520646FA3
:10A1EF00204E4F542072656D6F7665204C6F6763FC
:10A1FF00617264202100005F00204D61696E206D47
:10A20F00656E75200020576F726B6F75742000207C
:10A21F005374616E6461726420776F726B6F7574C3
:10A22F002000204C4320637573746F6D20776F721D
:10A23F006B6F757473200020437573746F6D207787
:10A24F006F726B6F7574732000204C4320637573AE
:10A25F00746F6D20776F726B6F757420002043756C
:10A26F0073746F6D20776F726B6F75742000204E53
:10A27F006577204C4320637573746F6D20776F7211
:10A28F006B6F75742000204E657720637573746F44
:10A29F006D20776F726B6F75742000204E6577207D
:10A2AF004C4320776F726B6F75742000204E65776B
:10A2BF0020776F726B6F7574200020536574207454
:10A2CF00696D6520776F726B6F7574200020536511
:10A2DF00742064697374616E636520776F726B6F3E
:10A2EF0075742000204C6F67436172642072656340
:10A2FF00616C6C200020526563616C6C20002053F0
:10A30F00657475702000204D656D6F7279207365CF
:10A31F00747570200020485220736574757020008A
:10A32F0020414E542063686573742062656C7420FD
:10A33F00002050726F706572746965732000002081
:10A34F005369676E616C20636F65666669636965E3
:10A35F006E74732000002057656C636F6D6520006D
:10A36F0020476F6F646279652000204C6F674361EF
:10A37F0072642000204C6F67436172642073756DA7
:10A38F006D61727900204C6F674361726420757440
:10A39F00696C6974696573002045646974204C6F3A
:10A3AF006743617264206461746100205365742097
:10A3BF00726563616C6C2073706C69742000446506
:10A3CF006C657465206D656D6F7279203F00446513
:10A3DF006C657465206C6173742073657373696F3A
:10A3EF006E203F0053776974636820746F20776F16
:10A3FF00726B206D6F6465203F00537769746368DB
:10A40F0020746F2074657374206D6F6465203F0036
:10A41F00466F726D6174204C6F6743617264203FA9
:10A42F000044656C657465204C6F674361726420EE
:10A43F006D656D6F7279203F00536574207A657278
:10A44F006F207374617465203F00526573657420CB
:10A45F00616C6C20737461746573203F0052657377
:10A46F00657420776F726B696E672074696D6520F4
:10A47F003F00526561647920746F207365742063A7
:10A48F00616C69622E20636F6566732021005365CE
:10A49F00742063616C69622E20636F656673203F61
:10A4AF0000526561647920746F2073657420446570
:10A4BF0076696365494420210053657420446576AD
:10A4CF006963654944203F0020536574207A6572A3
:10A4DF006F20737461746520007E617474006176FF
:10A4EF0065007C004A00746F74616C006B4A007DDC
:10A4FF00002F316B6D006C656674006D0052616EDC
:10A50F006B007065616B00706163650072706D0048
:10A51F007E0020496E697469616C697A6520736584
:10A52F006E736F7273200020202000253464002585
:10A53F003364002E253164002532640025303464E5
:10A54F000020526573742000506F7765720053704E
:10A55F006C6974206D61782E5E5E3A202575207EC1
:10A56F0000456E657267790053706C6974206D6178
:10A57F00782E5E5E3A20252E3166206B4A0053708E
:10A58F006565640053706C6974206D61782E5E5E32
:10A59F003A202575206B6D2F680044697374616EC6
:06A5AF0063650053706CAF
:10A5B5006974206D61782E5E5E3A202575206D00E8
:10A5C500436164656E63650053706C6974206D61E9
:10A5D500782E5E5E3A2025752072706D00486561A3
:10A5E500727420726174650053706C6974206D61BA
:10A5F500782E5E5E3A2025752062706D0041766585
:10A60500726167655E5E3A202575207E00546F7421
:10A61500616C5E5E3A20252E3166206B4A004176DC
:10A6250065726167655E5E3A202575206B6D2F68E2
:10A6350000546F74616C5E5E3A202575206D004193
:10A645007665726167655E5E3A2025752072706D6C
:10A6550000417665726167655E5E3A202575206208
:10A66500706D002853706C6974202575206D696EB6
:10A675002900456E65726779205B4A5D00537065F8
:10A685006564205B6B6D2F685D00506F7765722088
:10A695005B7E5D0047726170680025752020002093
:10A6A5002025752020002020257500307300536972
:10A6B500676E616C0020302E3573200020203173C9
:10A6C5000020203173202000202032730050656166
:10A6D5006B20666F7263653A202575204E20202019
:10A6E500004C6566744C202020202020202020303E
:10A6F500232020313830232020202020526967680C
:10A70500744C0039302320202020202020202020B8
:10A715002020202020202020202020202020202034
:10A7250020202020202039302300313830232020DC
:10A735003023002575252520002025752525002594
:10A7450075270020257520002575206D2028256496
:10A75500206D2900252E3066206D20282564206D6A
:10A7650029002575206D00252E3066206D007000AE
:10A77500253032643A25303264004A75737420728C
:10A7850069646500576F726B6F757400526563611C
:10A795006C6C005365747570004C6F67436172642F
:10A7A500004C61737420776F726B6F75740053740E
:10A7B500616E646172640052655269646500437537
:10A7C50073746F6D20284C6F674361726429004371
:10A7D5007573746F6D004E657720776F726B6F754B
:10A7E500740031303030206D0033303030206D0052
:10A7F50034303030206D003130303030206D003352
:10A8050030206D696E75746573003630206D696E24
:10A8150075746573005E576F726B6F75745E5E520B
:10A825006573745E5E506163650025752E5E253027
:10A8350032643A253032643A253032645E5E253022
:10A8450032643A253032645E5E253032643A253012
:10A85500326420282F316B6D290025752E5E256CFD
:10A86500646D5E5E253032643A253032645E5E2565
:10A875003032643A2530326420282F316B6D29003F
:10A8850053657373696F6E003A2025750054696DC1
:10A8950065004E6F206D6F72652073657373696F08
:10A8A5006E730054696D652028683A6D3A73295EA8
:10A8B5005E5E3A0025303264203A2025303264202D
:10A8C5003A202530326420202000253032643A2594
:10A8D5003032643A253032642020202020202000A8
:10A8E50044697374616E636520286D295E5E5E3A06
:10A8F50000257520257520257520257520257520B1
:10A90500257500257525752575257525752575000C
:10A91500526573742074696D6520286D3A73295EDC
:10A925005E5E3A0025303264203A202530326420BC
:10A93500202000253032643A253032642020202042
:10A94500202020005061636520286D3A73295E5EE2
:10A955005E3A0025303264203A20253032642020CA
:10A9650020282F316B6D2900253032643A2530328D
:10A975006420282F316B6D292020202020200047BE
:10A98500726170686963616C005465787400536521
:06A99500742073706C6970
:10A99B0074004D656D6F72790048520050726F7084
:10A9AB006572746965730044656C65746520616CD0
:10A9BB006C0044656C657465206C61737420736501
:10A9CB007373696F6E0053616D706C652072617487
:10A9DB0065004F4646000025752073616D706C65F0
:10A9EB00730000414E542063686573742062656C7C
:10A9FB007400506F6C617200253575202825732902
:10AA0B0000414E542B53706F7274005375756E74F6
:10AA1B006F0053706C69745E5E3A202575206D690A
:10AA2B006E004669726D7761726520766572736927
:10AA3B006F6E5E5E5E3A20252E3166004465766948
:10AA4B0063652049445E5E5E3A20256C6400536565
:10AA5B006E736F722049445E5E5E3A20256C640013
:10AA6B0053656E736F722049445E5E5E3A204E6F83
:10AA7B007420636F6E6E65637465640042617474F9
:10AA8B006572795E5E5E3A20257300536573736958
:10AA9B006F6E735E5E5E3A20252D3264004D656DE0
:10AAAB006F72795E5E5E3A20252D642525206672D5
:10AABB0065650053706C69745E5E5E3A20252D648B
:10AACB00206D696E00466F7263655E5E5E3A204173
:10AADB00203D20252D382E3566003A2042203D2082
:10AAEB00252D362E3366003A2043203D20252D356B
:10AAFB002E3266004372616E6B20726164697573EE
:10AB0B005E5E5E3A202575206D6D00486F75727321
:10AB1B005E5E5E3A20256C64004C6F674361726425
:10AB2B00206D656E75004C6F6743617264206D65B7
:10AB3B006D6F72795E5E5E3A20252D342E3166255F
:10AB4B00252066726565004D61696E206D656E75B9
:10AB5B000053756D6D6172790055736572206E616E
:10AB6B006D655E5E5E3A202573005574696C697481
:10AB7B006965730055736572206E616D655E5E5E0F
:10AB8B005E3A202573004C6F6743617264206D65DC
:10AB9B006D6F72795E5E5E5E3A20252D342E3166C6
:10ABAB0025252066726565004E756D626572206F96
:10ABBB00662073657373696F6E735E5E5E5E3A20BB
:10ABCB002575004564697420757365722064617422
:10ABDB00610044656C657465204C6F6743617264FA
:10ABEB00206D656D6F727900466F726D61742061B7
:10ABFB006C6C0055736572206E616D655E3A002555
:10AC0B00630025730020496E666F20004553434156
:10AC1B00504500454E544552002043686F6F736595
:10AC2B0020726563616C6C2073657373696F6E2042
:10AC3B00002043686F6F73652072657269646520CD
:10AC4B0073657373696F6E200053657373696F6EF1
:10AC5B005E5E3A202575202F2025750044617465B2
:10AC6B005E5E3A20253032642E253032642E32302F
:10AC7B00253032640054696D655E5E3A20253032B2
:10AC8B00643A253032643A25303264004C656E6785
:10AC9B0074685E5E3A20253031643A253032643A6E
:10ACAB00253032643A2530326400496D706F72740E
:10ACBB00616E743A5E5E526563616C6C206D656D9E
:10ACCB006F72792066756C6C21005E5E4F6E6C79CD
:10ACDB002070617274206F662074686520736573D1
:10ACEB0073696F6E207761732073617665642E00D4
:10ACFB00526563616C6C206D656D6F727920667542
:10AD0B006C6C21004E6F2073756D6D6172792069CB
:10AD1B006E666F20666F722073657373696F6E005A
:10AD2B0028526563616C6C206D656D6F727920665E
:10AD3B00756C6C2900253031643A253032643A3019
:10AD4B00303A3030202D20253031643A25303264B2
:10AD5B003A253032643A2530326400506F77657291
:10AD6B002061762E5E5E3A202575207E00456E654D
:06AD7B007267795E5E3A8A
:10AD810020252E3166206B4A005370656564206171
:10AD9100762E5E5E3A20252E3166206B6D2F68007F
:10ADA10044697374616E63655E5E3A20252E306678
:10ADB100206D00436164656E63655E5E3A202575B2
:10ADC1002072706D0048522061762E5E5E3A202519
:10ADD100752062706D0053756D6D617279207365B8
:10ADE1007373696F6E202575004C656E6774685EBC
:10ADF1005E5E5E5E5E3A20253031643A2530326413
:10AE01003A253032643A2530326400506F776572EA
:10AE11002061762E5E5E5E5E5E5E3A202575207E46
:10AE210000506F77657220706B2E5E5E5E5E5E5EB7
:10AE31003A202575207E004C2525202F20522525DE
:10AE41005E5E5E5E5E5E3A202575202F20257500D0
:10AE5100436164656E63655E5E5E5E5E5E3A20259B
:10AE6100752072706D004361642E20706B2E5E5EE2
:10AE71005E5E5E5E3A2025752072706D00446973D6
:10AE810074616E63655E5E5E5E5E5E3A20252E30A5
:10AE910066206D00456E657267795E5E5E5E5E5E20
:10AEA1003A20252E3166206B4A0053706565642077
:10AEB10061762E5E5E5E5E5E5E3A20252E316620F4
:10AEC1006B6D2F680048522061762E5E5E5E5E5E7D
:10AED1005E3A2025752062706D002573253032643D
:10AEE1003A253032643A253032643B200000257324
:10AEF100256C646D3B200000456D70747900002560
:10AF01007520257300002E2E00002535640025755F
:10AF1100002530356C640025356C640025303164C2
:10AF21003A253032643A25303264004E6F20736521
:10AF31007373696F6E7320666F7220726563616CE3
:10AF41006C2021004572726F72202100456D707472
:10AF51007920637573746F6D20776F726B6F757481
:10AF61000057726F6E672073656E736F7220636F27
:10AF71006E6E65637465640053656E736F72206EE7
:10AF81006F7420636F6E6E656374656400536573DF
:10AF910073696F6E20656E642021004D656D6F725F
:10AFA1007920656D7074792021004C6F674361725F
:10AFB10064206D656D6F727920656D7074792021E3
:10AFC1000052656C617820210052657374207365AD
:10AFD1007373696F6E00526561647920746F2072BA
:10AFE1006572696465202100526561647920746F1E
:10AFF1002073746172742021002053657373696F2B
:10B001006E5E3A202575002054696D655E3A2025F3
:10B011003032643A253032643A25303264002044BB
:10B02100697374616E63655E3A20256C64206D00FE
:10B03100576F726B6F75742073657373696F6E20D0
:10B0410025752F257500456E64206F662072657227
:10B05100696465202100456E64206F6620776F72F8
:10B061006B6F757420210025752073657373696F8B
:10B071006E287329006576616C75617465640042A0
:10B0810061747465727920656D7074792021005442
:10B0910075726E696E67206F6666004E6F20616320
:10B0A100746976697479202100476F6F64627965EC
:10B0B10000536574207A65726F20647572696E67DA
:10B0C1000073657373696F6E206E6F7420616C6CB1
:10B0D1006F776564202100526563616C6C206D653A
:10B0E1006D6F72792066756C6C20210053657373E6
:10B0F100696F6E206E6F74207361766564004465BC
:10B101006C657465206C6173742073657373696F0A
:10B111006E20646F6E652021002575207365737341
:10B12100696F6E287329206C656674005472616EB4
:10B1310073666572206F662073657373696F6E0045
:10B14100257520696E2070726F67726573732100B7
:10B1510044617461207472616E736665722063610B
:06B161006E63656C65647D
:10B16700202100526573657420616C6C20737461D3
:10B1770074657320646F6E6520210043616E206ED5
:10B187006F742072656164204C6F6743617264203D
:10B1970021004D616B652073757265204C6F6743A5
:10B1A70061726420697300696E73657274656420E7
:10B1B700636F72726563746C7900526163652069AD
:10B1C7006E697469616C697A6174696F6E202100B8
:10B1D7005072657061726520666F72207261636577
:10B1E7002021003B3C00526163652066696E6973EC
:10B1F70068656420210046696E616C2072616E6B20
:10B207003A202575005261636520627265616B653E
:10B2170064202100536561726368696E6720666FF9
:10B227007220686561727420726174652062656C52
:10B2370074287329202100506C656173652077613C
:10B2470069742E2E2E004E6F2062656C7473206613
:10B257006F756E64210040205F202573004C6F7767
:10B267000048696768004D656469756D002530326F
:10B27700643A2530326420200003000000000000FB
:10B2870000000000028080808080008000000004B1
:10B29700A0A0000000000000000005609090600082
:10B2A7000000000000062070A8A07028A8702000E9
:10B2B7000748B05010283428000000073848487065
:10B2C70094887400000002808000000000000000E5
:10B2D700000420408080808080402000048040203F
:10B2E7002020202040800004A0A0000000000000D3
:10B2F70000000600002020F82020000000020000C7
:10B3070000000000808000000300000000C0000073
:10B317000000000200000000000080000000042080
:10B327002040404080800000000560909090909001
:10B33700600000000340C04040404040000000055E
:10B34700609010202040F000000005609010201051
:10B3570090600000000610305090F81010000000B8
:10B36700057040E09010906000000005609080E05C
:10B3770090906000000005F0102020404040000041
:10B3870000056090906090906000000005609090CC
:10B397007010906000000002000080000000800034
:10B3A70000000200008000000080800000040020F0
:10B3B7004080402000000000050000F000F0000081
:10B3C700000000040080402040800000000006705C
:10B3D700880830200020000000080000000000005E
:10B3E7000000000008102828447C44820000000662
:10B3F700F08888F08888F0000000067088808080D8
:10B40700887000000006F08888888888F0000000AF
:10B4170006F88080F88080F800000006F88080F049
:10B4270080808000000006708880988888700000FF
:10B437000006888888F88888880000000280808055
:10B4470080808080000000051010101010906000B0
:10B457000000068890A0C0A09088000000058080AA
:10B4670080808080F00000000882C6C6AAAAAA923F
:10B477000000000688C8C8A89898880000000670D1
:10B4870088888888887000000006F08888F08080A7
:10B497008000000006708888888890780000000681
:10B4A700F08888F09088880000000670888070080F
:10B4B700887000000006F8202020202020000000CF
:10B4C700068888888888887000000008828244443B
:10B4D7002828100000000882925454545428000071
:10B4E70000068850502050508800000006885050B1
:10B4F7002020202000000007FC0810204080FC00CE
:10B50700000003C080808080808080C0000480802D
:10B51700404040202000000003C0404040404040E1
:10B5270040C0000440A0A00000000000000006008A
:10B5370000000000000000F800028080000000000A
:06B54700000000000500F9
:10B54D00006010709070000000058080E090909079
:10B55D00E000000005000060908090600000000594
:10B56D00101070909090700000000500006090F039
:10B57D008060000000042040E0404040400000009A
:10B58D000500007090909070906000058080E090B4
:10B59D0090909000000002800080808080800000EC
:10B5AD0000034000404040404040800005808090B6
:10B5BD00A0C0A0900000000280808080808080006C
:10B5CD000000080000EC929292920000000500002D
:10B5DD00E0909090900000000500006090909060C9
:10B5ED00000000050000E0909090E08080000500D4
:10B5FD00007090909070101000050000B0C0808019
:10B60D008000000005000070806010E00000000464
:10B61D000040E04040402000000005000090909068
:10B62D00907000000006000088505050200000006F
:10B63D00060000A8A8A8A850000000050000906012
:10B64D00606090000000060000885050502020409F
:10B65D0000040000E0204080E00000000300000036
:10B66D0000000000000000028080808080808080CB
:10B67D0000001880404040204040408000098880F4
:10B68D009480550055005500550022000000000023
:10B69D0000000000000E001C002A0038004600616A
:10B6AD00007C008A009800A600B400C200D000DE25
:10B6BD0000EC00FA01080116012401320140014E8F
:10B6CD00015C016A01780186019401A201B001BEFD
:10B6DD0001CC01DA01F50210022B02460261026F64
:10B6ED00027D029802B302C102CF02EA02F80313EF
:10B6FD00032E03490364037F039A03B503C303DEDB
:10B70D0003F90414042F043D044B04590467047514
:10B71D0004830491049F04AD04BB04C904D704E55C
:10B72D0004F30501050F051D052B053905470562B8
:10B73D000570057E058C059A05A805B605C405D2CC
:10B74D0005ED060806160631063F064D06680690FD
:10B75D000400000000000000000000000000046074
:10B76D00606060606060006060000000076C6C6C81
:10B77D000000000000000000000007242424FC4805
:10B78D0048FC909090000000071038545070783CA1
:10B79D001C14543810000A720052005200540074E8
:10B7AD00000B800A800A80128013800000000000C8
:10B7BD0000091C00360036001E0018003D006D000B
:10B7CD00670067003D8000000000000004606060BD
:10B7DD000000000000000000000005103020606037
:10B7ED0060606060602030100480C0406060606008
:10B7FD0060606040C0800620F820D8000000000086
:10B80D00000000000800000018187E181800000045
:10B81D0000000400000000000000006060204000F7
:10B82D000500000000000000700000000000040092
:10B83D0000000000000000606000000005101020F6
:10B84D00202040404080800000000778CCCCCCCC3C
:10B85D00CCCCCCCC780000000718387858181818C4
:10B86D001818180000000778CC0C0C18383060C080
:10B87D00FC0000000778CC0C0C380C0C0CCC7800BC
:10B88D0000000718183838585898FC181800000090
:10B89D00077C60C0F8CC0C0C0CCC7800000007388D
:10B8AD004CC0C0F8CCCCCCCC7800000007FC0C18F8
:10B8BD00183030306060600000000778CCCCCC7858
:10B8CD00CCCCCCCC780000000778CCCCCCCC7C0C8C
:10B8DD000CC87000000004000000606000000060F3
:10B8ED006000000004000000606000000060602047
:10B8FD004000080000041C70C0701C040000000013
:10B90D000800000000FE00FE00000000000008001E
:10B91D000040701C061C704000000000087CC6062C
:06B92D00060C183000308A
:10B93300300000001088009001A682C544A54895F8
:10B94300508D680048008E01090209040908090B9B
:10B953000E000E001B001B001B00318031803F8056
:10B9630060C060C0000000000000097E0063006347
:10B973000063007E0063006300630063007E0000D9
:10B9830000000000000A1F003180600060006000BA
:10B9930060006000600031801F00000000000000B4
:10B9A300097C006600630063006300630063006357
:10B9B3000066007C00000000000000087E606060FC
:10B9C3007E606060607E000000087E606060607E74
:10B9D300606060600000000A1F003180600060004A
:10B9E300600067806180618031801F00000000007B
:10B9F30000000963006300630063007F006300636A
:10BA03000063006300630000000000000004606046
:10BA13006060606060606060000000080606060603
:10BA230006060666663C00000009630066006C00BB
:10BA33006C007C0076006600660063006300000013
:10BA430000000000086060606060606060607E000D
:10BA530000000B71C071C07BC07BC06AC06AC06A42
:10BA6300C06EC06EC064C000000000000009630027
:10BA7300730073007B006B006F0067006700630057
:10BA830063000000000000000A1E003300618061B3
:10BA930080618061806180618033001E000000004E
:10BAA300000000097E0063006300630063007E0002
:10BAB30060006000600060000000000000000A1EDB
:10BAC30000330061806180618061806180658033C3
:10BAD300001F00008000000000097E006300630077
:10BAE300630063007E006600630063006180000002
:10BAF30000000000093E006300600070003C001E6F
:10BB0300000700030063003E00000000000000087F
:10BB1300FF181818181818181818000000096300DF
:10BB230063006300630063006300630063006300FA
:10BB33003E000000000000000A60C060C031803198
:10BB43008031801B001B001B000E000E0000000054
:10BB53000000000F638C638C339836D836D836D800
:10BB630036D81C701C701C700000000000000963B4
:10BB730000630036001C001C001C001C0036006320
:10BB830000630000000000000008C3C3663C3C18CB
:10BB93001818181800000008FE060C18183030603A
:10BBA300C0FE0000000570606060606060606060FF
:10BBB300606070058080404040202020101000000D
:10BBC3000004E06060606060606060606060E00886
:10BBD3000030307848CC000000000000000700006F
:10BBE30000384446463E1C000000000460606000CC
:10BBF300000000000000000000080000003C461E9A
:10BC03003666663E000000086060606C76666666B5
:10BC1300766C000000080000003C66606060663CD3
:10BC230000000008060606366E6666666E3600007D
:10BC330000080000003C66667E60663C000000056C
:10BC4300306060F0606060606060000000080000C9
:10BC530000366E6666666E3606463C086060606C4B
:10BC63007666666666660000000460600060606079
:10BC7300606060600000000460600060606060609D
:10BC830060606060C008606060666C78786C6C6649
:10BC930000000004606060606060606060600000DD
:10BCA300000C0000000000006EC0776066606660F4
:10BCB3006660666066600000000000000800000027
:10BCC3006C766666666666000000080000003C66E7
:10BCD300666666663C000000080000006C766666D7
:10BCE30066766C60606008000000366E6666666E9D
:10BCF300360606060600000078606060606060003B
:10BD03000000080000003C66703C0E663C0000002A
:06BD13000600103078303C
:10BD190030303030180000000800000066666666A2
:10BD2900666E360000000900000000000063006331
:10BD3900003600360036001C001C00000000000020
:10BD4900000C000000000000623067303760356089
:10BD59003DE01DC018C00000000000000800000000
:10BD690066663C183C666600000009000000000099
:10BD790000630063003600360036001C001C001CFE
:10BD89000018007800070000007C0C183030607C37
:10BD99000000000600000000000000000000000094
:10BDA900000C31807BC0FFE0FFE0FFE07FC03F80F7
:10BDB9000E00040000000000000000001580018052
:10BDC9008002809762E0A49490C49490A49890947F
:10BDD9009890000000000000000000000000000032
:10BDE900000000000E00102C20304020802100228D
:10BDF9000004000BB01248224842480248000000E3
:10BE09000000000000000000000000000000000029
:10BE19000000000000000000000000004300700066
:10BE2900B300F60139017C01BF0202024502880212
:10BE3900CB030E03511100000000000000000000B8
:10BE490000000000000000000000000000000000E9
:10BE590000000000000000000000000000000000D9
:10BE690000000000000000000000000000000000C9
:10BE790000000000000000000B00000000000000AE
:10BE890000000000000000000000000000000000A9
:10BE990000000000000000000000000E001F001F4D
:10BEA900001F000E0011000000000000000000004B
:10BEB9000000000000000000000000000000000079
:10BEC9000000000000000000000000000000000069
:10BED9000000000000000000000000000000000059
:10BEE90000000000000000001107E0000FF0001F33
:10BEF900F8003FFC003C3C003C3C00781E00781EEA
:10BF090000781E00781E00781E00781E00781E003A
:10BF1900781E00781E00781E003C3C003C3C003F27
:10BF2900FC001FF8000FF00007E0001100F000000E
:10BF3900F00001F00003F00007F0001FF0003FF0EF
:10BF4900003EF00038F00020F00000F00000F000A2
:10BF590000F00000F00000F00000F00000F0000028
:10BF6900F00000F00000F00000F00000F000110700
:10BF7900E0001FF8003FFC003FFC007C3E00781EFB
:10BF890000781E00001E00001E00003C00007C001E
:10BF990000F80001F00003E00007C0000F80001F57
:10BFA90000001E00003FFE003FFE007FFE007FFEF6
:10BFB900001107C0001FF0003FF8003FF8007C7C2B
:10BFC90000783C00383C00003C0000780003F00099
:10BFD90003E00003F800003C00001E00001E00788A
:10BFE9001E00781E007C3E003FFC001FFC000FF085
:10BFF9000007E0001100780000780000F80001F85F
:10C009000003F80003F80007F8000F78000E780025
:10C019001E78003C7800387800707800F07800FFCE
:10C02900FE00FFFE00FFFE00FFFE00007800007822
:10C0390000007800007800113FFC003FFC003FFC45
:10C04900007FFC007800007800007800007FE000A5
:10C059007FF000FFF800FFFC00F87E00701E000072
:10C069001E00001E00F01E00F83E00FC7C007FFC54
:10C07900003FF8001FF0000FC0001103E0000FF8A7
:10C08900001FFC001FFC003E3E003C1E0078000023
:10C099007800007BE0007FF8007FFC007FFC007CDB
:10C0A9003E00781E00781E00781E00381E003C3EB7
:10C0B900003FFC001FFC000FF80003E000117FFEA9
:10C0C900007FFE007FFE007FFE00003C000078003C
:10C0D90000700000F00000E00001E00001C0000372
:10C0E900C00003C0000380000780000780000780AC
:06C0F900000F00000F0023
:10C0FF00000F00000F00000F00001107E0001FF8F5
:10C10F00003FFC007C3E00781E00781E00781E0069
:10C11F00781E003C3C001FF8000FF0001FF8003C99
:10C12F003C00781E00781E00781E00781E00781ED6
:10C13F00003C3C003FFC001FF80007E0001107C067
:10C14F00001FF0003FF8003FFC007C3C00781C0013
:10C15F00781E00781E00781E007C3E003FFE003FD8
:10C16F00FE001FFE0007DE00001E00001E00783ECE
:10C17F00007C7C003FFC003FF8001FF0000FC00068
:10C18F00090000000018003C003C001800000000EF
:10C19F000000000000000000000000000000001878
:10C1AF00003C003C001800000000000000000000F0
:10C1BF000000000000000000000000000000000070
:10C1CF00000000000000000000008D00D400D50129
:10C1DF006201EF027C03090396042304B0053D05B9
:10C1EF00CA0657069E074E07FE1B00000000000000
:10C1FF000000000000000000000000000000000030
:10C20F00000000000000000000000000000000001F
:10C21F00000000000000000000000000000000000F
:10C22F0000000000000000000000000000000000FF
:10C23F0000000000000000000000000000000000EF
:10C24F0000000000000000000000000000000000DF
:10C25F0000000000000000000000000000000000CF
:10C26F0000000000000000000000000000000000BF
:10C27F000000000000000F000000000000000000A0
:10C28F00000000000000000000000000000000009F
:10C29F00000000000000000000000000000000008F
:10C2AF00000000000000000000000000000000037C
:10C2BF008007C00FE00FE00FE007C00380001B00F6
:10C2CF003F800000FFE00003FFF80007FFFC0007BE
:10C2DF00FFFC000FFFFE000FF1FE001FE0FF001F2D
:10C2EF00C07F001FC07F001F803F003F803F803F07
:10C2FF00803F803F803F803F803F803F803F803F37
:10C30F00803F803F803F803F803F803F803F803F26
:10C31F00803F803F803F803F803F803F803F801F36
:10C32F00803F001FC07F001FC07F001FE0FF000F76
:10C33F00F1FE000FFFFE0007FFFC0007FFFC0003EC
:10C34F00FFF80000FFE000003F80001B0003F0003B
:10C35F000003F0000007F000000FF000001FF000D6
:10C36F00003FF000007FF00001FFF00007FFF0003A
:10C37F000FFFF0000FF7F0000FE7F0000FC7F0000E
:10C38F000F07F0000C07F0000007F0000007F000A7
:10C39F000007F0000007F0000007F0000007F000B2
:10C3AF000007F0000007F0000007F0000007F000A2
:10C3BF000007F0000007F0000007F0000007F00092
:10C3CF000007F0000007F0000007F0000007F00082
:10C3DF000007F0000007F0001B003FC00000FFF84F
:10C3EF000001FFFC0003FFFE0007FFFF000FFFFF30
:10C3FF00000FF0FF800FE07F801FC03F801FC03F06
:10C40F00800FC03F8000003F8000003F8000007F12
:10C41F000000007F000000FE000001FE000003FC92
:10C42F00000007F800000FF000001FE000003FC001
:10C43F0000007F800000FF000001FE000003FC00F1
:10C44F000003F8000007F000000FFFFF800FFFFF51
:10C45F00801FFFFF801FFFFF803FFFFF803FFFFF19
:10C46F00803FFFFF801B003F800000FFE00003FFC5
:10C47F00F00007FFF80007FFFC000FFFFC000FF1B3
:10C48F00FE001FE0FE001FC0FE0003C0FE00000004
:10C49F00FE000001FC000003FC00000FF800001F6D
:10C4AF00E000001FC000001FF800001FFC0000008C
:10C4BF00FE0000007F0000007F0000003F800000B2
:10C4CF003F8000003F800F803F803F803F803FC014
:06C4DF007F801FC07F00FA
:10C4E5001FF1FF001FFFFE000FFFFE0007FFFC000E
:10C4F50003FFF80001FFE000003F80001B0000FC87
:10C50500000001FC000003FC000003FC000007FC28
:10C5150000000FFC00000FFC00001FFC00003FFCAA
:10C5250000007FFC00007FFC0000FDFC0001F9FC21
:10C535000001F9FC0003F1FC0007E1FC0007E1FC48
:10C54500000FC1FC001F81FC001F81FC003F01FCA6
:10C55500007E01FC007FFFFF807FFFFF807FFFFFE4
:10C56500807FFFFF807FFFFF807FFFFF800001FC52
:10C57500000001FC000001FC000001FC000001FCC2
:10C58500000001FC000001FC001B01FFFF0001FF92
:10C59500FF0001FFFF0003FFFF0003FFFF0003FF94
:10C5A500FF0003FFFF0003F8000007F0000007F09D
:10C5B500000007F0000007F0000007E7C0000FFFCC
:10C5C500F0000FFFFC000FFFFE000FFFFE000FFF46
:10C5D500FF001FF0FF001FC07F8003803F80000029
:10C5E5003F8000003F8000003F800F803F803F80FC
:10C5F5003F803FC07F801FC07F001FF0FF001FFFEF
:10C60500FE000FFFFE0007FFFC0003FFF80001FF1F
:10C61500E000003F80001B001FC000007FF000010C
:10C62500FFF80003FFFC0007FFFC0007FFFE000FFB
:10C63500F1FE000FE0FF001FC07F001F807C001F80
:10C645008000003F8000003F8000003F8FC0003F1A
:10C65500BFF0003F7FF8003FFFFC003FFFFE003FBB
:10C66500FFFF003FE0FF003FC07F803F803F803FEE
:10C67500803F803F803F801F803F801F803F801F1D
:10C68500C03F801FC07F800FF0FF000FFFFF000736
:10C69500FFFE0003FFFC0001FFF80000FFF00000B3
:10C6A5003FC0001B3FFFFF803FFFFF803FFFFF8034
:10C6B5003FFFFF803FFFFF803FFFFF803FFFFF0001
:10C6C50000007E000000FC000001F8000003F800F7
:10C6D5000003F0000007E0000007E000000FC000C5
:10C6E500001FC000001F8000003F8000003F0000C9
:10C6F500003F0000007F0000007E000000FE0000FB
:10C7050000FE000000FE000001FC000001FC00002E
:10C7150001FC000001FC000001F8000003F8000026
:10C7250003F8000003F8000003F8000003F8000018
:10C735001B003F800001FFF00003FFF80007FFFC2E
:10C74500000FFFFE000FF1FE001FE0FF001FC07F7E
:10C75500001FC07F001FC07F001FC07F001FC07F5C
:10C76500000FE0FE000FF1FE0007FFFC0001FFF0E7
:10C775000000FFE00003FFF80007FFFC000FE0FEEC
:10C78500001FC07F001FC07F003F803F803F803F6C
:10C79500803F803F803F803F803F803F803FC07F1C
:10C7A500801FC07F001FF0FF000FFFFE0007FFFE88
:10C7B5000003FFF80001FFF000003FC0001B007FF1
:10C7C500800001FFE00003FFF00007FFF8000FFF06
:10C7D500FC001FFFFE001FE1FE003FC07F003F8001
:10C7E5007F003F803F003F803F003F803F803F808C
:10C7F5003F803F803F803FC07F801FE0FF801FFF5D
:10C80500FF800FFFFF8007FFFF8003FFDF8001FF31
:10C81500BF80007E3F8000003F8000003F80000019
:10C825003F0007C03F001FC07F001FE07E000FF1E3
:10C83500FE000FFFFE000FFFFC0007FFF80003FFDF
:10C84500F00001FFC000007F00000F0000000000A5
:10C855000000000000038007C00FE00FE00FE007B5
:10C86500C003800000000000000000000000000080
:10C87500000000000000000000038007C00FE00F6B
:10C88500E00FE007C003800000000000000000008A
:10C89500002700003F00000007FFF800001FFFFE13
:10C8A50000007FFFFF8000FFFFFFC001FFFFFFE0EB
:10C8B50003FFFFFFE007FFFFFFF007FF007FF00F1B
:06C8C500FC001FE00FF86B
:10C8CB000010001FF80000001FF00000001FF00018
:10C8DB0000001FF00000003FF00FFFF83FF00FFFCC
:10C8EB00F83FF00FFFF83FF00FFFF81FF00FFFF8C6
:10C8FB001FF00FFFF81FF00FFFF81FF0001FF81FBE
:10C90B00F8001FF80FF8001FF80FFC001FF807FFC7
:10C91B00007FF807FFFFFFF803FFFFFFF801FFFFA2
:10C92B00FFF000FFFFFFC0007FFFFF00003FFFFC99
:10C93B00000007FFF00000003E00002700007C0015
:10C94B00000007FFC000003FFFF800007FFFFC0066
:10C95B0000FFFFFF0001FFFFFF0003FFFFFF80074A
:10C96B00FFFFFFC007FE00FFE00FFC007FE00FF8AA
:10C97B00003FE01FF8003FF01FF0001FF01FF0001A
:10C98B001FF01FF0001FF01FF0001FF83FF0001FFB
:10C99B00F83FF0001FF83FF0001FF81FF0001FF0EA
:10C9AB001FF0001FF01FF0001FF01FF0001FF01F03
:10C9BB00F8003FF00FF8003FE00FFC007FE007FEB0
:10C9CB0000FFE007FFFFFFC003FFFFFF8001FFFF3A
:10C9DB00FF8000FFFFFF00007FFFFC00003FFFF820
:10C9EB00000007FFE00000007C00000102040810BB
:10C9FB0020408080402010080402017FBFDFEFF74A
:10CA0B00FBFDFE1E466982ADB75C707A02BC02BCB0
:10CA1B0002D402E302ED02F402F802FB02FE03026F
:10CA2B0003090400000004002B00020304050607A1
:10CA3B0007040102030405050001020304010204BB
:0DCA4B0008102006000000190032006404ED
:10CA5800411DF700012880012900012A00417BEBD4
:10CA680000411A420041699300411A6B104169C1A3
:10CA780000416C6B004169AF004213A90000426895
:10CA8800190000441A3D000000004269AA000A4249
:10CA98006601006542660F00C8411A670062041506
:10CAA800D80100007A440000000000000001008066
:10CAB8003B45000000000000000100007A4500002E
:10CAC80000000000000100401C46000000000000BB
:10CAD800000200000000001E00000000000200002C
:10CAE800000001000000000000010000000000003C
:10CAF800000000000000000000000000000000002E
:10CB0800000000000000000000000000000000001D
:10CB1800000000000000000000000000000000000D
:10CB280000000000000000000000000000000000FD
:10CB380000000000000000000000000000000000ED
:10CB480000000000000000000000000000000000DD
:10CB580000000000000000000000000000000000CD
:10CB680000000000000000000000000000000000BD
:10CB780000000000000000000000000000000000AD
:10CB8800000000000000000000000000000000009D
:10CB9800000000000000000000000000000000008D
:10CBA800000000000000000000000000000000007D
:10CBB800000000000000000000000000000000006D
:10CBC800000000000000000000000000000000005D
:10CBD800000000000000000000000000000000004D
:10CBE800000000000000000000000000000000003D
:10CBF800000000000000000000000000000000002D
:10CC0800000000000000000000000000000000001C
:10CC1800000000000000000000000000000000000C
:10CC280000000000000000000000000000000000FC
:10CC380000000000000000000000000000000000EC
:10CC480000000000000000000000000000000000DC
:10CC580000000000000000000000000000000000CC
:10CC680000000000000000000000000000000000BC
:10CC780000000000000000000000000000000000AC
:10CC8800000000000000000000000000000000009C
:10CC9800000000000000000000000000000000008C
:05CCA800000000000087
:10004600759850438780758DFEE589540F4420F5D9
:1000560089D28EC2ABD2ACC20CC20FE4901A41F068
:090066009017E2F0C298C2992241
:10006F00D20F9002D57406F09002D4E0FF24809056
:10007F006994F0901A417401F0C2998F99C20D22C0
:10008F00D20F9002D57406F09002D4E0FF24809036
:10009F006994F0901A417401F0C2998F99C20D22A0
:030023000200AF29
:1000AF00C0E0C0F0C083C082C0D075D00830993294
:1000BF00C299300F2D901A41E0C394C85003E00449
:1000CF00F0906994E0FF901A41E0FED39F4006E460
:1000DF00F0C20F800D74D32EF582E43402F583E065
:1000EF00F599309847C298900000E599F09017E283
:1000FF00E0C394C85003E004F0900000E0FF9017B5
:10010F00E2E0FE240FF582E43415F583EFF0EFF40F
:10011F00701AEEFF7E0078087C027D027B027A1552
:10012F00790F12E94FD20CE49017E2F0D0D0D082C1
:07013F00D083D0F0D0E032C4
:06000600200FFDD20D22C7
:1001460090BFFFE05403B403F790BFFF7481F090B3
:10015600BFFFE05403B403F790BFFF7498F090BF5D
:10016600FFE05403B403F790BFFEE4F090BFFFE056
:100176005403B403F790BFFEE4F090BFFFE05403CE
:10018600B403F790BFFF7442F090BFFFE05403B48E
:1001960003F790BFFE741EF090BFFFE05403B40354
:1001A600F790BFFEE4F090BFFFE05403B403F7906E
:1001B600BFFF7443F090BFFFE05403B403F790BF52
:1001C600FEE4F090BFFFE05403B403F790BFFE7463
:1001D6000FF090BFFFE05403B403F790BFFF7440E5
:1001E600F090BFFFE05403B403F790BFFE7428F00D
:1001F60090BFFFE05403B403F790BFFEE4F090BF56
:10020600FFE05403B403F790BFFF7441F090BFFFC3
:10021600E05403B403F790BFFEE4F090BFFFE05450
:1002260003B403F790BFFEE4F090BFFFE05403B4BD
:0902360003F790BFFF7424F022CD
:10023F00EF1460201460541470030202D124036081
:10024F000302033E7E0F7F007D007B027A6C79E311
:10025F0012ED47227564047565CE756329E563C396
:10026F009470400302033E7E007F107D0074E325EF
:10027F0065F9746C3564FA7B0212ED47741E2565BF
:10028F00F565E43564F564056380D27564037565BF
:10029F004975631CE563C39480400302033E7E00EF
:1002AF007F0E7D0074E32565F9746C3564FA7B026B
:1002BF0012ED47741E2565F565E43564F564056335
:1002CF0080D275640B7565D6756365E563C39472EB
:1002DF0050247E007F1A7D0074E32565F9746C3518
:1002EF0064FA7B0212ED47741E2565F565E43564EB
:1002FF00F564056380D5741E2565F565E43564F5F1
:10030F0064756373E563C3948050247E007F1A7D08
:10031F000074E32565F9746C3564FA7B0212ED47BE
:10032F00741E2565F565E43564F564056380D52293
:10033F0075600275616C7562E375A61E75A6E1E4C2
:10034F00FFEFC3940F4003020478E4FE90BFFFE079
:10035F005403B403F790BFFEEEF090BFFFE05403D9
:10036F00B403F790BFFEEFF090BFFFE05403B40368
:10037F00F790BFFF7424F0902D82E0605590BFFF7F
:10038F00E05403B403F790BFFEEEF090BFFFE054CC
:10039F0003B403F790BFFEEFF090BFFFE05403B438
:1003AF0003F790BFFF7424F090BFFFE05403B40332
:1003BF00F7AB60AA61A96212E98190BFFEF090BF0E
:1003CF00FFE05403B403F790BFFF74C4F0E4902D23
:1003DF0082F090BFFFE05403B403F7AB60AA61A9AA
:1003EF006212E98190BFFEF090BFFFE05403B403A7
:1003FF00F790BFFF74C4F0902D82E0605590BFFF5F
:10040F00E05403B403F790BFFEEEF090BFFFE0544B
:10041F0003B403F790BFFEEFF090BFFFE05403B4B7
:10042F0003F790BFFF7424F090BFFFE05403B403B1
:10043F00F7AB60AA61A96212E98190BFFEF090BF8D
:10044F00FFE05403B403F790BFFF74C4F0E4902DA2
:10045F0082F074012562F562E43561F561EEF460B6
:0A046F00040E02035B0F020350228B
:10047900EFC394F0503BEDC394805035EF13131341
:10048900541FFE75F01EEDA42EF582E435F0F583B8
:10049900E58224E3F582E583346CF583C083C08269
:1004A900E0FEEF540790C9FE93FFEE4FD082D08350
:0204B900F0222F
:10000C00AC07ECD39B5008AF041204790C80F3229C
:10002E00AC07EDD39B5008AF041204790D80F32278
:0A04BB007B027A0179C81204C52201
:1004C5008F638D648B658A668967E4900001F0AB64
:1004D50065AA66A96712E981FF606FB45E12900094
:1004E50001E090CA0E93F563900001E004F0804DA1
:1004F500EF24E0FFE434FFFE7C007D0B12E9DF8E84
:10050500688F6974812FF974B23EFA7B05AD6385F6
:10051500646F74802FF582EE34B2F583E493F57041
:1005250075710A1207E574802569F582E56834B2AC
:10053500F583E4932563F563C394F0500D740125A9
:0B05450067F567E43566F566808522E7
:10055000E4FE8B688A69896AAB68AA69A96A12E9AC
:1005600081FD601F75F00BA42420F582E5F034B105
:10057000F583E4932EFE7401256AF56AE43569F586
:100580006980D5EF24FE6009047010C3E5679EFF03
:0E05900022EEC313FFC3E5679FFF227F002208
:0A059E007B027A0179C81205A82239
:1005A8008F638D648B658A668967E4900002F0AB7F
:1005B80065AA66A96712E981FF7003020690644084
:1005C8007049E56475F01EA4AEF024C5F56AEE34F2
:1005D800FFF569E4F568E568C3940F4003020682F5
:1005E8007E007F1C901DF7E075F0FFA4FD74E325E5
:1005F8006AF9746C3569FA7B0212ED47741E256A34
:10060800F56AE43569F569056880CBAB65AA66A922
:100618006712E981FFB45E12900002E090CA149359
:10062800F563900002E004F08050EF25E0245FF5C8
:1006380082E434B6F583E493FE7401938E69F56A17
:10064800245EF974B73EFA7B05AD6385646F745D0B
:10065800256AF582EE34B7F583E493F57075710D6C
:100668001207E5745D256AF582E56934B7F583E418
:10067800932563F563C394F0500E74012567F567FD
:09068800E43566F5660205B722AF
:10069100E4FE8B658A668967AB65AA66A96712E97C
:1006A10081FD602B25E0245FF582E434B6F583E417
:1006B10093FC740193245DF582EC34B7F583E493E4
:1006C1002EFE74012567F567E43566F56680C9EF8E
:1006D10024FE6009047010C3E5649EFF22EEC3137B
:0A06E100FFC3E5649FFF227F0022A3
:0A06EB007B027A0179C81206F5229D
:1006F5008F578D588B598A5A895BAB59AA5AA95B72
:1007050012E981FF605C25E024C8F582E434BDF57B
:1007150083E493FE7401938E5CF55D243FF974BE0A
:100725003EFA7B05AD5785586F743E255DF582EE23
:1007350034BEF583E493F5707571161207E5743EC2
:10074500255DF582E55C34BEF583E4932557F557C1
:10075500C394F0500D7401255BF55BE4355AF55AE9
:0307650080982257
:0A0768007B027A0179C812077222A1
:100772008F608D618B628A638964AB62AA63A964AC
:1007820012E981FF605C25E0247CF582E434C1F546
:1007920083E493FE7401938E65F56624F9F974C1BE
:1007A2003EFA7B05AD6085616F74F82566F582EED1
:1007B20034C1F583E493F5707571231207E574F87B
:1007C2002566F582E56534C1F583E4932560F5601D
:1007D200C394F0500D74012564F564E43563F56348
:0307E200809822DA
:1007E5008B6B8A6C896D8D6EED2570F577E433F52D
:1007F50076D3E57794F0E576940040067576007536
:1008050077F0E5702407FF131313541FF570129347
:1008150066856F74E4F572E572C39571400302094C
:100825002A856E75E4F573E573C395704003020977
:1008350023AB6BAA6CA96D12E981FDE574C39480A5
:10084500400302090DE57554077039E575C394E851
:100855005032E575131313541FFB7A00E57475F0D8
:100865001EA42BFFEA35F0FE901DF7E06005EDF4C0
:10087500FC8002AC0574E32FF582EE346CF583EC55
:10088500F002090D7980AC75E5752408FFECC39F6E
:10089500400302090DECC395775066EC131313540E
:1008A5001FFB7A00E57475F01EA42BFFEA35F0FEF8
:1008B500901DF7E06005EDF4FB8002AB05EB596098
:1008C5002174E32FF582EE346CF583C083C082E09A
:1008D500FBEC540790C9FE93FAEB4AD082D083F023
:1008E500801F74E32FF582EE346CF583C083C082DC
:1008F500E0FFEC540790CA0693FEEF5ED082D083EA
:10090500F0E9C313F90C808074082575F575740139
:10091500256DF56DE4356CF56C057302082C0574D1
:06092500057202081C220D
:10092B008F63AA05A903E56304FFE914FB12000C0E
:10093B00E56304FFAD66AB0112000CAF63EA04FD87
:10094B00E56614FB12002EAF01EA04FDE56614FB0D
:10095B0012002EE914FFE56614FD120479E904FF79
:10096B00EA2402FDAB6612002EE5632402FFE56666
:08097B0004FDAB0112000C2287
:100983007F4A7D6C7B6D75667912092B7F5C7D7563
:100993001204797F5B1D7B5D12000C7F5A1D0B12C5
:1009A300000C7F591D0B12000C7F581D0B12000CFD
:1009B3007F571D0B12000C7F8B7D6C7BAE756679A8
:1009C30012092B7F9D7D701204797F9C0D7B9E12F3
:1009D300000C7F9B0D0B12000C7F9A0D0B12000C69
:0F09E3007F990D0B12000C7F980D0B12000C2248
:1009F200D297D296C297E4FFEFC394105004000F2F
:050A020080F6C29622FF
:100A0700C297D296E4FFEFC394105004000F80F60C
:030A1700D2972251
:100A1A003097047F0180027F00D296E4FEEEC394F1
:0A0A2A00105004000E80F6C2962260
:06001C00D297120A1A221D
:100A3400AD07E4FBEBC39408500EED339297120A12
:090A44001AED25E0FD0B80EC2207
:100A4D00E4FDFCECC39408500EED25E0FD120A1AEE
:0A0A5D00EF60010D0C80ECAF0522E4
:100A67008E5B8F5C8B5D8A5E895FE4F563F564C39B
:100A7700E5649561E56395605067908002E0F52A2B
:100A870020E3037F0122120C10EF7002FF221209EC
:100A9700F27FA0120A3412001CE55BFF120A34121F
:100AA700001CAF5CE55C120A3412001C1209F27FCD
:100AB700A1120A3412001C120A4DAB5DAA5EA95F8F
:100AC700EF12E9CB7401255FF55FE4355EF55E054E
:100AD7005CE55C7002055B0564E564700205638094
:100AE7008EAB5DAA5EA95FE412E9CBD297120A1A10
:060AF700120A077F012234
:100AFD008E4A8F4B8B4C8A4D894EE4900003F090BB
:100B0D008002E0F52A20E3037F0122120C10EF7022
:100B1D0002FF221209F27FA0120A3412001CE54ACC
:100B2D00FF120A3412001CAF4BE54B120A341200AF
:100B3D001CAB4CAA4DA94E12E981FE700990000321
:100B4D00E0C3954F5030908002E0F52A20E3037FFB
:100B5D000022EE6011FF120A347401254EF54EE4A9
:100B6D00354DF54D8005E4FF120A3412001C90003E
:0C0B7D0003E004F080BB120A077F012295
:100B89008E578F588B598A5A895BE4900004F090EC
:100B99008002E0F52A20E3037F0122900004E0C3EC
:100BA900955C5060120C10EF7002FF22908002E0F9
:100BB900F52A20E3037F00221209F27FA0120A34EA
:100BC90012001CE557FF120A3412001CAF58E558F1
:100BD900120A3412001CAB59AA5AA95B12E981FF07
:100BE900120A347401255BF55BE4355AF55A120093
:100BF9001C900004E004F00558E5587002055712EE
:070C09000A0780977F01221A
:100C1000E4F5661209F27FA0120A3412001C8F65F7
:100C2000129366E566B4FA037F00220566E56570F7
:070C3000E2120A077F012216
:100C3700438E02123966129366906C6BE0D394323E
:100C4700400A7F1B123FEFE4906C6BF0D390681A59
:100C5700E0942C906819E094014019902D8BE07076
:100C67000C12033F7F02E4FD7B01128EEAE49068D9
:100C770019F0A3F09069C2E06003020D177B027AB6
:100C870000790612DCE8EF644270677F417EF0FD71
:100C9700FC12ECCF900006E0FCE412E4ED12E494C1
:100CA700406E7F437E707D007C0012ECCF90000683
:100CB700E0FCE412E4ED12E4946002505390000665
:100CC700E0FB901DFAF07F457EBB7D807C0012EC37
:100CD700CFAC03E412E4ED12E3E512E5219069D20B
:100CE700EEF0A3EFF0E49069A8F0A3F0D208D20BDE
:100CF700801EC39069A9E094BC9069A8E094024063
:100D07000FE4901DFAF09069A8F0A3F0D208D20B77
:090D17007F71123FEF020C3D2236
:0300430002002692
:0100260032A7
:03000300020D20CB
:100D2000C0E0C0F0C083C082C0D075D018129366F6
:100D3000E490681EF0200803020E12C208D3906CE3
:100D4000E0E09401906CDFE094005003020E127F0B
:100D5000417EF07D007C0012ECCF901DFAE0FCE4B7
:100D600012E4ED12E4945003020E127F437E707D74
:100D7000007C0012ECCF901DFAE0FCE412E4ED12CE
:100D8000E49460054003020E129069D2E0FAA3E0F9
:100D9000FB901DF3E02BF0901DF2E03AF0901DDE89
:100DA00012EC6612ECCFAF1BAE1AE4FCFD12EAACFB
:100DB000901DDE12EC82901DF1E004F0901DDA121D
:100DC000EC6612ECCF7F017E007D007C0012EAAC65
:100DD000901DDA12EC82901DDA12EC66E412E4E562
:100DE00012ECCF7F427EC87D007C0012E36D12ECD6
:100DF000CF901DDE12EC66E412E4E512ECCF7F42E8
:100E00007E707D007C0012E3E512E3E5901DA212E6
:100E1000EC82200E03021228C20EE4906C75F0A33F
:100E2000F0906CDFE0FEA3E0FFD39401EE9400505D
:100E3000030210B8EF64024E700C90681D04F0E4D9
:100E40009013A9F0A3F012568B901DC212EC6612FB
:100E5000E5217C007D0A12E9F3901DF6E0FD75F0B6
:100E600002A424B3F582E5F03413F583EEF0A3EF8A
:100E7000F075F002EDA424B3F582E5F03413F583A8
:100E8000E0FEA3E0FFC390668DE09F90668CE09E3D
:100E90005005EEF0A3EFF075F002EDA424B3F58257
:100EA000E5F03413F583C083C082E0FEA3E0FF7C4D
:100EB000007D4412E9DFD082D083EEF0A3EFF09002
:100EC0001DBE12EC6612E5217C007D0A12E9F3904A
:100ED0001DF6E0FD75F002A42427F582E5F0341438
:100EE000F583EEF0A3EFF075F002EDA42427F58270
:100EF000E5F03414F583E0FEA3E0FFC390668FE0D5
:100F00009F90668EE09E5005EEF0A3EFF075F00224
:100F1000EDA42427F582E5F03414F583C083C08264
:100F2000E0FEA3E0FF7C007D4412E9DFD082D083A5
:100F3000EEF0A3EFF0901DC612EC6612E5217C00E6
:100F40007D0A12E9DF901DF6E0FD75F002A4249BF6
:100F5000F582E5F03414F583EEF0A3EFF075F002BE
:100F6000EDA4249BF582E5F03414F583E0FEA3E0C4
:100F7000FFC3906691E09F906690E09E5005EEF072
:100F8000A3EFF075F002EDA4249BF582E5F0341494
:100F9000F583C083C082E0FEA3E0FF7C007D4412A5
:100FA000E9DFD082D083EEF0A3EFF0901DF6E004ED
:100FB000F0E0FFC3943A400E9065E7E004F070065D
:100FC0009065E6E004F0EF75F03A84901DF6E5F0E8
:100FD000F0901DFBE070030212281200069002D46C
:100FE00074BAF09002D6744CF0754004E4F53FE515
:100FF0003FC3940B40030210B2E53F75F003A424F5
:1010000045F582E4341AF583E0FBA3E0FAA3E0F9A6
:1010100012EC288F278E268D258C24E524547FFF03
:10102000AE40054074D32EF582E43402F583EFF030
:10103000E525547FFFAE40054074D32EF582E4349D
:1010400002F583EFF0E526547FFFAE40054074D3F0
:101050002EF582E43402F583EFF0E527547FFFAEEE
:1010600040054074D32EF582E43402F583EFF0E5B9
:1010700025A2E713A2E7135420FFE524A2E71354A7
:05108000404FFFE526D2
:101085007803A2E713D8FB54104FFFE5277804A295
:10109500E713D8FB54084FFFAE40054074D32EF537
:1010A50082E43402F583EFF0053F020FEF12006F83
:1010B500021228906CDFE07004A3E0640160030273
:1010C5001228901A43E02486601024FE601A240436
:1010D5007022901A437479F0801A901A43747BF049
:1010E5009013A67401F0800C901A43747DF0901350
:1010F500A67401F07E007F667D007B027A1D798EE5
:1011050012ED477E007F637D007B027A6C79771252
:10111500ED479003A1E0C3942840297427F0E0FF30
:101125007E007C007D6312E9DF741B2FF9741E3E7F
:10113500FA7B02C01B78C67C69AD1BD01B7E007F85
:101145000612E94F78907C6C7D027B027A6979C63C
:101155007E007F0612E94F78967C6C7D027B027AD1
:101165006979C67E007F0612E94F906C7C12EC8E81
:1011750000000000906C9E12EC8E00000000906C48
:10118500867403F09069C6E0D394034003021216F7
:101195009069B9E07003FF80079069B9E02402FF08
:1011A500906CA2EFF09069B9E025E0244FF582E458
:1011B50034CAF583E493740193906CB1F09013AE47
:1011C500E0906CA3F090660312EC66906CA412ECB0
:1011D5008290660712EC66906CA812EC8290660B02
:1011E50012EC66906CAC12EC829002D1E0906CB07F
:1011F500F09013AF12EC66906C8712EC82906695B6
:1012050012EC66906C8B12EC829013A7E0906C8FB9
:10121500F0902D8B7401F090681DF0901DF4F09006
:10122500667CF0432980908001E529F090681E7462
:0D12350001F0D0D0D082D083D0F0D0E032D4
:03002B000212427C
:10124200C0E0C0F0C083C082C0D075D010C2CF90C1
:101252006C76E004F07006906C75E004F090667CA9
:10126200E0601DC3906CE0E09401906CDFE09400BC
:10127200400E901DE8E004F07006901DE7E004F0D7
:10128200901A6BE0700312962D9065E8E0D39400FB
:101292004005E014F08003432880908000E528F0A8
:1012A2009069A9E004F070069069A8E004F09068E3
:1012B2001AE004F07006906819E004F0906C6BE09C
:1012C20004F09013AAE004F070069013A9E004F071
:1012D200C39013AAE0942C9013A9E09401401990B2
:1012E200681D7401F0E49013A9F0A3F0FF1293A813
:1012F2009066A7EEF0A3EFF090667CE06003129395
:10130200D5907BE8E070030218D3906820E0600378
:101312000218D390667CE0601A901DB612EC661239
:10132200ECCF7F3F7E807D007C0012E262901DB692
:1013320012EC829069B9E0D3940050030213CA9070
:10134200669BE0FF9069C1E0C39F50030213CAE4A9
:10135200F090669AE0FF9069BFE02FFF9069BEE0CF
:101362003400FE90669BE0FD7C0012EA489017E094
:10137200EEF0A3EFF0E49069BEF0A3F09065EAE02E
:10138200902D83F0E49065EAF09069B0E090699066
:10139200F0E49069B0F0906C67E09001C7F0E490DF
:1013A2006C67F09069C0E09065FCF0E49069C0F071
:1013B20090667CE06012C3906CE0E09401906CDF78
:1013C200E0940040031243759069C1E004F0906814
:1013D20021E0700302152B906601E0FEA3E0FF24DA
:1013E20064901E01F0E43E901E00F0901A67E0FD4A
:1013F200B402047C0180027C00907BEAECF0EDB444
:1014020002047C0180027C00906C74ECF0EDB4016B
:10141200047D0180027D00906CDAEDF0E4901A67A1
:10142200F09069AAE0FCA3E02FFFEE3CFE90660F6D
:10143200E0FCA3E0FDC3EF9DEC6480F8EE648098CD
:10144200400A9069AA74FFF0A374F6F09069AAE0CA
:10145200FEA3E0FF906602E02FFF906601E03EFEF1
:101462009013ADE0FCA3E0FDD3EF9DEC6480F8EEB9
:101472006480984003021515901A3D12EC6612EC36
:10148200CF7F017E007D007C0012EAAC901A3D12F3
:10149200EC82901A3D12EC6612ECCF7F027E007D48
:1014A200007C0012F51C12ECF6EC4D4E4F60047FEE
:1014B2000180027F02901A67EFF09069AAE4F0A31C
:1014C200740AF0EF6402704B906610E02405F0900D
:1014D200660FE03400F0E0FEA3E0FF7C027D5812CC
:1014E200EA4890660FECF0A3EDF09013ADE0FEA396
:1014F200E0FFD3ED9FEE6480F8EC64809850149086
:1015020013AEE024C8906610F09013ADE034009062
:10151200660FF09069AAE0FEA3E0FF906602E02F5A
:10152200F0906601E03EF080447F011293A8901E85
:1015320000EEF0A3EFF07F011293A8901E00EEF0F0
:10154200A3EFF030C0047F0180027F00907BEAEFBE
:10155200F03092047F0180027F00906C74EFF030D3
:1015620094047F0180027F00906CDAEFF09069C2F0
:10157200E06402600302162D901DF5E004F090690C
:10158200C0E004F0901DF5E0FF700D907BE904F0DF
:10159200E4901DFAF0021625907BEAE07003021631
:1015A20025906C6CE06003021625907BE9EFF0FB5E
:1015B200E4901DF5F0906C6704F0E49069C0F07F50
:1015C200417EF0FDFC12ECCFAC13E412E4ED12E428
:1015D2009440197F437E707D007C0012ECCF907B9B
:1015E200E9E0FCE412E4ED12E4944007E4901DFA11
:1015F200F08030907BE9E0FB7A007EEA7F60FDAC10
:041602001212E9F3E4
:10160600EF2405FFE43EFE7C007D0A12E9F3901DFF
:10161600FAEFF09069D2EAF0A3EBF0D208D20B9081
:101626007BEAE0906C6CF0901DFBE07006200D03E9
:101636001218FD901E00E0FEA3E0FF9069BFE02FA8
:10164600F09069BEE03EF09013ADE0FCA3E0FDD360
:10165600EF9DEC6480F8EE648098500F9013ADE037
:10166600FFA3E0901E00CFF0A3EFF0906CDAE0FF4E
:101676006019906C68E07013901A687402F09069B3
:10168600B014F0901A6CE09013ACF0906C68EFF028
:10169600906C74E0FB7003021794906C65E0600335
:1016A600021794901A68E06402600302179404F02B
:1016B6009065EAF0902F2DE0FFA3E090681BCFF035
:1016C600A3EFF0E4902F2DF0A3F09069BA12EC6628
:1016D600902D8612EC829069BA12EC8E0000000002
:1016E600906CE0E004F07006906CDFE004F0902F60
:1016F60032E0902F31F0B401047F0080027F019028
:101706002F32EFF0901A6CE09013A5F09013ACE036
:10171600907BE7F09066A0E0902D81F090698C12A6
:10172600EC669065ED12EC8290039CE0FFA3E090DE
:101736006692CFF0A3EFF0907BE7E025E0FFE4337D
:10174600FE748A2FF582EE342DF583E0FFA3E09038
:101756006822CFF0A3EFF0E4901A6CF09013ACF08F
:1017660090698C12EC8E00000000E49066A0F09068
:10177600039CF0A3F09065E9E0600BE4906992F0B9
:101786009065E9F080069069927401F0D20E906C33
:1017960065EBF09013ADE0FEA3E07802C333CE33E1
:1017A600CED8F924A2F582EE3403F58312EC661244
:1017B600ECCF901E00E0FEA3E07802C333CE33CE1A
:1017C600D8F924A2F582EE3403F58312EC6612EA08
:1017D600BF90000912EC829069BA12EC6612ECCF47
:1017E60090000912EC6612EAAC9069BA12EC82908B
:1017F600000912EC66780C12EC01900008EFF090EC
:101806001A6CE0C394C740030218A2900008E0F9DE
:10181600FF7E009017E3E0FCA3E0FD12E9DFAC16C3
:10182600AD17901A6CE025E0FFE433FE902F32E00E
:10183600FB75F090A4246EF582E5F0341AF583EB7F
:101846002583F583E5822FF582EE3583F583ECF06B
:10185600A3EDF09066A0E0C399500EE9F090000960
:1018660012EC6690698C12EC82E9FF90039DE02FE2
:10187600F090039CE03400F0E0FCA3E0FD901A6CCD
:10188600E025E0FFE433FE748C2FF582EE342DF56F
:1018960083ECF0A3EDF0901A6CE004F0C3902F2EC9
:1018A600E094B8902F2DE0940B40069013A6E060CC
:1018B60010902F2EE004F07006902F2DE004F0809B
:1018C6000C902D8BE06006902D8A7401F090681EB6
:1018D600E06009200E0330080353297F908001E55C
:1018E60029F0902D827401F0902D84F0D0D0D08212
:0718F600D083D0F0D0E032F6
:1018FD001200069002D47488F09002D67435F090E0
:10190D001E00E0FCA3E0FDAE147803CEA2E713CEDB
:10191D0013D8F8547F9002D7F0901DFAE0FFC3134F
:10192D00547F9002D8F0E4A3F0ED30E004E04401E0
:10193D00F0906C74E0600D906C65E070079002D9CA
:10194D00E04402F0E49002DAF0901E00E0FEA3E025
:10195D00FF30E1079002DAE04401F0906CDAE060CC
:10196D000D906C68E070079002DAE04402F0E490AC
:10197D0002DBF0EF30E204E04401F0901DFAE030BC
:0D198D00E0079002DBE04402F012008F2220
:10199A008D5AAB07AA06E4900010F0A3F0A3F0A3B7
:1019AA00F0A312EC8E0000000090001812EC8E00DA
:1019BA0000000090001C12EC8E0000000090002035
:1019CA0012EC8E0000000090002412EC8E00000041
:1019DA0000906CE2E06026AE02AF037C007D0A1242
:1019EA00E9DF906C78E02428FD906C77E03400CD34
:1019FA002F90000FF0ED3E90000EF08012906C9543
:101A0A00E02B90000FF0906C94E03A90000EF012E8
:101A1A00936690668812EC8E00007042E490000D86
:101A2A00F090000DE0FF9065FFE0FCA3E0FDC3EF3E
:101A3A009DE49C4003021CAB906CE2E07003021A26
:101A4A00FC906C79E0FEA3E0FF24F6FDEE34FFFC87
:101A5A0090000EE0FAA3E0FB6D7002EC6A706190F0
:101A6A006C7BE0705B906C78E02428FD906C77E0EA
:101A7A003400FCC3EF9DFFEE9CFE7C007D0A12E958
:101A8A00F3EF24FFFFEE34FFFEE4FCFD12ECCF7F00
:101A9A00707E177D007C0012EAD312ECCF906C7C2A
:101AAA0012EC6612EABFE412E4E512ECCF7F427E42
:101ABA00C87D007C0012E3E590668812EC828018EB
:101ACA00906C79E0FEA3E0FFC390000FE09F9000C6
:101ADA000EE09E4003021CAB90000EE0FEA3E0FF66
:101AEA007B027A66797E75600075610A120A67025E
:101AFA001BAE906C9AE0FEA3E0FF24FFFDEE34FFDC
:101B0A00FC90000EE0FAA3E0FB6D7002EC6A7052E2
:101B1A00906C9CE0704C906C94E0FCA3E0FDC3EFE9
:101B2A009DFFEE9CCF24FFCF34FFFEE4FCFD12ECB8
:101B3A00CF7F707E177D007C0012EAD312ECCF9023
:101B4A006C7C12EC6612EABFE412E4E512ECCF7F79
:101B5A00427EC87D007C0012E3E590668812EC8222
:101B6A008018906C9AE0FEA3E0FFC390000FE09FFC
:101B7A0090000EE09E4003021CAB90000EE0FEA314
:101B8A00E0FF7C007D0A12E9DF74332FF9742F3EDF
:101B9A00FA7B02C003787E7C66AD03D0037E007FA9
:101BAA000A12E94F90001412EC6612ECCF90667E8E
:101BBA00E0FCA3E0FDE412E4E912ECCF7F447E7A74
:101BCA007D007C0012E3E512E26290001412EC82BE
:101BDA0090001812EC6612ECCF906685E0FCA3E048
:101BEA00FDE412E4E912E26290001812EC82E55A6E
:101BFA0020E00920E10620E20330E34A90002012A7
:101C0A00EC6612ECCF906680E0FCA3E0FDE412E4FF
:101C1A00E912E26290002012EC8290002412EC6633
:101C2A0012ECCF906682E0FCA3E0FDE412E4E91234
:101C3A00ECCF7F417E207D007C0012E3E512E26258
:101C4A0090002412EC82E55A30E412906684E0FF98
:101C5A00900011E02FF0900010E03400F0E55A30C7
:101C6A00E512906687E0FF900013E02FF0900012D3
:101C7A00E03400F0906CE2E0601090000FE0240A7B
:101C8A00F090000EE03400F0800E90000FE004F0B7
:101C9A00700690000EE004F090000DE004F0021AC5
:101CAA002B7E007F187D007B027A6979D412ED477A
:0C1CBA0090668812EC6612ECCF90000DD2
:101CC600E014FCE412E4ED12ECCF7F427E707D005E
:101CD6007C0012E36D12E26290668812EC8290003C
:101CE6000DE07003021E297F007E007D007C00123D
:101CF600ECCF90001412EC6612E494601C401A902B
:101D0600002012EC6612ECCF90001412EC6612E37F
:101D1600E59069D412EC82800A9069D412EC8E00A8
:101D26000000007F007E007D007C0012ECCF9069F1
:101D3600D412EC6612E494602A402890002412EC37
:101D46006612ECCF90001412EC6612E3E512ECCFAB
:101D56007F407E667D667C6612E36D9069DC12ECE0
:101D660082800A9069DC12EC8E0000000090002050
:101D760012EC669069D812EC8290002412EC669000
:101D860069E012EC82900010E0FCA3E0FDE412E4AE
:101D9600E912ECCF90001412EC6612ECCF7F427E73
:101DA600707D007C0012E3E512E3E59069E412EC35
:101DB60082900012E0FCA3E0FDE412E4E912ECCF0D
:101DC6007F427EC87D007C0012E36D12ECCF90004E
:101DD6001812EC6612ECCF7F427E707D007C0012FA
:101DE600E3E512E3E59069E812EC827F417EF07D3F
:101DF600007C0012ECCF9069E812EC6612E4944085
:101E0600187F437E707D007C0012ECCF9069E8124B
:101E1600EC6612E494600C400A9069E812EC8E00BD
:091E260000000090000DE0FF2215
:101E2F00E4906C75F0A3F0906991E070087F65FD08
:101E3F00FB1296152290020BE075F00AA4FF900298
:101E4F000AE075F064A42FFF90020CE02F90002899
:101E5F00F012ED211ED3101EC2171F2F181F3E198F
:101E6F001EC81A1EC81B1EE51C1F0D1D1EF11F1FAD
:101E7F0005201ED9211F21221EBC301F52311F7178
:101E8F00371EA6491F7C4D1F8E4E206F5020AD511F
:101E9F0020AD52000020D67F01124B00901A4374E0
:101EAF0002F0E4FF124A08129DF10220D612443BC1
:101EBF000220D61220E30220D6900028E0FF1295D0
:101ECF006B0220D61295EC0220D67F217D03E4FB16
:101EDF001296150220D67F1C7D17E4FB1296150271
:101EEF0020D6901A43E064B660030220D674B9F08E
:101EFF001235050220D67F01129CB00220D6901A0F
:101F0F0043E064B560030220D674B8F012350502C1
:101F1F0020D67F067B027A6579F812A0CE0220D6F2
:101F2F00124361EF60030220E2124DE60220D61247
:101F3F004361EF60030220E290020DE0FF124FB702
:101F4F000220D6124361EF60030220E27F011249A3
:101F5F0042E4FF12023F901A437402F01235050259
:101F6F0020D67F37E4FDFB1296150220D6901A4338
:101F7F0074BEF07F187DFFE4FB1296CB0220D67F54
:101F8F004EE4FDFB12961590020DE0FF7E007C00E3
:101F9F007D6412E9DF12936D7F077B027A667911F8
:101FAF0012A0CE90661112EC669069B312EC82907B
:101FBF0013AB7406F0901A4374BFF0E490669CF074
:101FCF00A3F0A37406F0E4A3F0902D8004F09066C4
:101FDF007CF09065ECF0E4902F20F0902D7A12ECCD
:101FEF008E000000009069CE12EC8E000000009071
:101FFF0013ABE0D39400403C1293669065ECE06025
:10200F00149013ABE014F07F18E0FDE4FB1296CBB5
:10201F00E49065ECF07F52129DC9EF60D2C20C9034
:10202F001A437402F0901A6B7410F07F1AE4FDFBE0
:10203F001296CB22E4906C71F07F067D0112842DF5
:10204F00906CDFE4F0A304F0D20E53297F9080014F
:10205F00E529F0907BE87401F090669404F08067B6
:10206F00901DFBE0606190020DE0902F20F07F0645
:10207F007B027A66791112A0CE90661112EC6690EF
:10208F002D7A12EC827F0B7B027A66791112A0CE29
:10209F0090661112EC669069CE12EC828029901D29
:0720AF00FBE06023901A43DF
:1020B60074C0F0901A6B7410F0900028E0B45104CC
:1020C6007F1980027F1A90020DE0FDE4FB1296CB89
:0D20D6007F7E900028E0FDE4FB12961522AD
:1020E3001200069002D474A4F09002D6744BF07FD1
:1020F300049013ADE0FCA3E0FD129FDF7F08900284
:10210300D1E0FD7C00129FDF90660312EC668F4FD7
:102113008E4E8D4D8C4C7F0A12A00D90660712ECEB
:10212300668F4F8E4E8D4D8C4C7F0F12A00D906697
:102133000B12EC668F4F8E4E8D4D8C4C7F1412A07C
:102143000D9013AF12EC668F4F8E4E8D4D8C4C7FDE
:102153001912A00D90669512EC668F4F8E4E8D4D21
:102163008C4C7F1E12A00D7F239013A7E0FD7C00F3
:07217300129FDF12006F2232
:10217A00E4F548EF24E070030224E124E07003024E
:10218A00290324C07003022D0A249070030234A389
:10219A0024E06003023502901A43E012ED2123176E
:1021AA0002231703231704231705231706232007DF
:1021BA0023200823200923200A23200B23290C2368
:1021CA00290D23290E23290F23291023291123320C
:1021DA0012233213233214233215233216233217D1
:1021EA00233B1823461923461A23461B23461C233E
:1021FA00461D23461E234F1F234F20234F21236CA6
:10220A0022236C23236C2423CA2623CA2723CA2801
:10221A0023D32D23D32E23D32F246932247233249C
:10222A00B13424A83523DC3923DC3A23E53C23E501
:10223A003D23E53E23E53F23E54023E54123EE50D8
:10224A0023EE5124005524005624005724125A2400
:10225A00125B24125C24095F24BA60241B6124C324
:10226A006223F77023F77123F77222ED7822ED7952
:10227A0023017A23017B23017C23017D23807E2392
:10228A00897F239280239B81239B82231783235A4E
:10229A008C235A8D235A8E235A8F235A90235A916C
:1022AA00235A922363A02363A12363A22363A32354
:1022BA0063A42363A52363A62363A72363A82363D5
:1022CA00A92484B4248DB52496B6249FB724CCB807
:1022DA0024D8B9247BBB22EDBE22EDBF22EDC0007B
:1022EA000035027F01124B00EF6003023502901A9B
:1022FA00437402F00235027F01124B00EF600302C1
:10230A003502906694E0901A43F0023502901A431F
:10231A007402F0023502901A437403F002350290F7
:10232A001A437408F0023502901A43740AF002350F
:10233A0002906694E0901A43F0023502901A4374B0
:10234A000BF0023502906694E0901A43F0023502CF
:09235A00901A43741FF0023502D1
:10236300901A437420F0023502906CE2E060047F1F
:102373005680027F04901A43EFF0023502901A430D
:102383007409F0023502901A437422F00235029068
:102393001A437423F00235029003A0E06013E4F0C3
:1023A300906820F090667CF0901A437402F0023536
:1023B30002901A43E0B48106747FF0023502901A4A
:1023C300437480F0023502901A437405F00235021B
:1023D300901A437426F0023502901A437427F002D0
:1023E3003502901A437439F0023502901A43742867
:1023F300F0023502901A437402F0023502901A4338
:102403007406F0023502901A437455F002350290B7
:102413001A437457F0023502906999E0FF647B60B8
:1024230003EF700F7E007F0A7D007B027A69799942
:1024330012ED47901A69E0FFC3940A501074992F64
:10244300F582E43469F583E0B47B02E4F0E4FF7ED3
:10245300017B027A697999755C0B120B89901A4397
:10246300745AF0023502901A43742DF0023502902B
:102473001A43742EF0023502901A437426F0023583
:1024830002901A437450F0023502901A437451F0CB
:10249300023502901A437405F0023502901A437410
:1024A30028F0023502901A43742FF0023502901A75
:1024B300437424F0023502901A43745CF00235022F
:1024C300901A43745BF0023502901A437451F01270
:1024D300931F023502901A437405F0023502901AD5
:1024E30043E012ED21262802262803262804262865
:1024F3000526280626430726430826430926430ABA
:1025030026430B26520C26520D26520E26520F2618
:102513005210265211266112266113266114266178
:102523001526611626611726701926701A26701B48
:1025330026701C26701D26701E267F1F267F2026D0
:102543007F21274322274323274324275226275229
:102553002727522827612D27612E27612F285234E0
:1025630027703927703A277F3C277F3D277F3E27F7
:102573007F3F277F40277F4127935027935127B6DB
:102583005527B65627B65727C55A27C55B27C55CB7
:1025930027D46127A77027A77125F47825F4792616
:0125A3000E29
:1025A4007A260E7B260E7C260E7D28187E28187F20
:1025B40028188028A08128AD8226A48C26B58D26D3
:1025C400C68E26D78F26E89026F991270A92271BD4
:1025D400A0271BA1271BA2271BA3271BA4271BA5DE
:1025E40026D7A626E8A726F9A8270AA900003502B7
:1025F400E4FFFDFBF54D123DF7E490681DF07F0705
:102604007D017B01128EEA023502E4FFFDFBF54DEC
:10261400123DF7E490681DF07F077D017B01128E67
:10262400EA0235027F047D017B02906C4BE0B40822
:10263400047E0680027E058E4D123DF70235027F30
:10264400047D017B07754D0B123DF70235027F04B3
:102654007D017B0C754D11123DF70235027F047D1F
:10266400017B12754D17123DF70235027F047D017F
:102674007B19754D1E123DF70235027F047D017BE7
:102684001F901A6AE024F975F00684E5F0D39400EB
:1026940040047E2180027E208E4D123DF7023502D9
:1026A400906C5AE004F0E075F00A84E5F0F002352D
:1026B40002906C5BE004F0E075F03C84E5F0F0021D
:1026C4003502906C5CE004F0E075F03C84E5F0F0D9
:1026D400023502906C5DE004F0E075F03C84E5F0B6
:1026E400F0023502906C5EE004F0E075F03C84E5A5
:1026F400F0F0023502906C5FE004F0E075F03C8489
:10270400E5F0F0023502906C60E004F0E075F03C16
:1027140084E5F0F0023502901A43E024B4F582E433
:10272400346BF583E004F0901A43E024B4F582E4BA
:10273400346BF583E075F00A84E5F0F00235027F2E
:10274400047D017B22754D24123DF70235027F047E
:102754007D017B26754D28123DF70235027F047DED
:10276400017B2D754D2F123DF70235027F047D014B
:102774007B39754D3A123DF70235027F047D017BAA
:102784003C902F30E0243BF54D123DF70235027F9B
:10279400047D017B50754D51123DF7E49069C5F0FD
:1027A4000235027F047D017B70754D71123DF70285
:1027B40035027F047D017B55754D57123DF7023577
:1027C400027F047D017B5A754D5C123DF702350290
:1027D400901A69E0FFC3940A400302350274992FEA
:1027E400F582E43469F583E0FE70057441F0800CF1
:1027F400EE24C075F03B84E5F02441F074992FF584
:1028040082E43469F583E0645B6003023502746139
:10281400F0023502902F2FE004F0906CE2E0601794
:10282400902F2FE0FF906C45E0FEEF8EF084902F08
:102834002FE5F0F0023502902F2FE0FF9003A1E086
:10284400FEEF8EF084902F2FE5F0F00235029066B3
:1028540000E004F070069065FFE004F09065FFE08E
:102864007004A3E0643D70079065FFF0A304F0904A
:1028740065FFE0FFA3E0906611CFF0A3EFF07F04C3
:102884007E00906611E0FD12DF5A7F057E0090669F
:1028940012E0FD12DF5A12DF6C0235027F03E4FD01
:1028A400FBF54D123DF70235029065FFE0FEA3E013
:1028B400FF9066AEE0FCA3E0FDD39FEC9E403D900C
:1028C40065FFE0FEA3E0FFC3ED9FFFEC9EFEC39017
:0228D4006CDEB8
:1028D600E09F906CDDE09E50179065FFE0FEA3E060
:1028E600FF906CDEE02FF0906CDDE03EF0023502EA
:1028F600E4906CDDF0A3F00235027F0022901A43CB
:10290600E012ED212A4C022A4C032A4C042A4C05DB
:102916002A4C062A67072A67082A67092A670A2AA5
:10292600670B2A760C2A760D2A760E2A760F2A76D9
:10293600102A76112A85122A85132A85142A8515C6
:102946002A85162A85172A94192A941A2A941B2A44
:10295600941C2A941D2A941E2AA31F2AA3202AA364
:10296600212B6F222B6F232B6F242B7E262B7E276A
:102976002B7E282B8D2D2B8D2E2B8D2F2C81342BC2
:102986009C392B9C3A2BAB3C2BAB3D2BAB3E2BAB5C
:102996003F2BAB402BAB412BBF502BBF512BE255EE
:1029A6002BE2562BE2572BF15A2BF15B2BF15C2CC9
:1029B60000612BD3702BD3712A16782A16792A3107
:1029C6007A2A317B2A317C2A317D2C447E2C447F25
:1029D6002C44802CCB812CD9822AC88C2ADA8D2AC9
:1029E600EC8E2AFE8F2B10902B22912B34922B46A5
:1029F600A02B46A12B46A22B46A32B46A42B46A5CD
:102A06002AFEA62B10A72B22A82B34A900003502DC
:102A1600E4FF7D01FBF54D123DF7E490681DF07F64
:102A2600077D017B01128EEA023502E4FF7D01FB80
:102A3600F54D123DF7E490681DF07F077D017B019F
:102A4600128EEA0235027F04E4FD7B02906C4BE0B5
:102A5600B408047E0680027E058E4D123DF70235CF
:102A6600027F04E4FD7B07754D0B123DF70235022C
:102A76007F04E4FD7B0C754D11123DF70235027F94
:102A860004E4FD7B12754D17123DF70235027F04F3
:102A9600E4FD7B19754D1E123DF70235027F04E4F5
:102AA600FD7B1F901A6AE024F975F00684E5F0D3E1
:102AB600940040047E2180027E208E4D123DF70256
:102AC6003502906C5AE02409F0E075F00A84E5F0CE
:102AD600F0023502906C5BE0243BF0E075F03C843C
:102AE600E5F0F0023502906C5CE0243BF0E075F016
:102AF6003C84E5F0F0023502906C5DE0243BF0E0AA
:102B060075F03C84E5F0F0023502906C5EE0243B03
:102B1600F0E075F03C84E5F0F0023502906C5FE081
:102B2600243BF0E075F03C84E5F0F0023502906C51
:102B360060E0243BF0E075F03C84E5F0F0023502FD
:032B4600901A439F
:102B4900E024B4F582E4346BF583E02409F0901AAB
:102B590043E024B4F582E4346BF583E075F00A842C
:102B6900E5F0F00235027F04E4FD7B22754D241265
:102B79003DF70235027F04E4FD7B26754D28123DA1
:102B8900F70235027F04E4FD7B2D754D2F123DF7C9
:102B99000235027F04E4FD7B39754D3A123DF70297
:102BA90035027F04E4FD7B3C902F30E0243BF54D5A
:102BB900123DF70235027F04E4FD7B50754D511239
:102BC9003DF7E49069C5F00235027F04E4FD7B70AE
:102BD900754D71123DF70235027F04E4FD7B557591
:102BE9004D57123DF70235027F04E4FD7B5A754DBE
:102BF9005C123DF7023502901A69E0FFC3940A405E
:102C09000302350274992FF582E43469F583E0FEF5
:102C19007005747AF0800CEE24F975F03B84E5F0C8
:102C29002441F074992FF582E43469F583E06460F6
:102C39006003023502745AF0023502906CE2E060DA
:102C490017906C45E0FF14FE902F2FE02EF0E08FD7
:102C5900F084E5F0F00235029003A1E014FF902F13
:102C69002FE02FF0E0FF9003A1E0FEEF8EF08490BB
:102C79002F2FE5F0F0023502906600E024FFF09076
:102C890065FFE034FFF0E07002A3E070089065FF93
:102C9900F0A3743CF09065FFE0FFA3E0906611CFCC
:102CA900F0A3EFF07F047E00906611E0FD12DF5A79
:102CB9007F057E00906612E0FD12DF5A12DF6C027A
:102CC90035027F037D01E4FBF54D123DF702350224
:102CD9009065FFE0FEA3E0FF906CDDE0FCA3E0FD62
:102CE900C39FEC9E40189065FFE0FEA3E0FFC3ED93
:102CF9009F906CDEF0EC9E906CDDF00235027F0057
:102D090022901A43E012ED212EEC022F23032F2CDF
:102D1900042F350531AE062E93072F3E083073096F
:102D29002F470A2F500B2F590C2F590D2F590E2FA2
:102D3900590F2F59102F59112F70122F70132F70EF
:102D4900142F70152F70162F70172F8F182F9C198D
:102D59002F9C1A2F9C1B2F9C1C2F9C1D2F9C1E2FB8
:102D6900C11F2FCA202FD32130732230732330D8AB
:102D79002430E12630EA27319C28337C2D33932EE9
:102D890033C42F33853233B633347534334D35314B
:102D9900003930F33A31193C31193D31193E3119B5
:102DA9003F31194031194131B75531C05631C957F1
:102DB90031D25A31E05B31E95C31F26032A86133DA
:102DC9001E6231A57031AE7131A5722E3B782E3B52
:062DD900792E3B7A2E3B2F
:102DDF007B2E3B7C2E3B7D340F7E341F7F34338024
:102DEF003447813447822FF08C2FF08D2FF08E2FA8
:102DFF00F08F2FF0902FF091301C92302BA0302BB2
:102E0F00A1302BA2302BA3302BA4302BA5302BA617
:102E1F00302BA7302BA83064A93345B43369B734AE
:102E2F007EB8348AB93498BB000035029066ABE0A7
:102E3F0090CA3493640560179066ABE090CA3493E0
:102E4F006406600B9066ABE090CA3493B4070D7FB5
:102E5F0001E4FDFBF54D123DF7023502901DFBE03D
:102E6F0060030235027F05FDFBF54D123DF77F0133
:102E7F00124568E490681DF07F077D017B01128E7B
:102E8F00EA023502901A43E0906694F0906C4BE0A2
:102E9F00B408167430FF7E017B047A00794975609F
:102EAF0000756101120A678006906C69E0F5499020
:102EBF00CA33E493FFE5498FF08485F049E549C3B0
:102ECF009406500AAF49E4FD12842D023502901A80
:102EDF006AE549F0901A437418F0023502906821A0
:102EEF00E07006901A44E0601B7FFFE4FD1284AA95
:102EFF00901A437478F07F01124568907BE8740153
:102F0F00F00235027F04E4FDFB1296CBE4907BE8E0
:102F1F00F0023502901A437407F0023502901A43FB
:102F2F007422F0023502901A437426F00235029093
:102F3F001A43740CF0023502901A437412F00235E2
:102F4F0002901A437419F0023502901A43E090660A
:102F5F0094F0901A43E024F4FFE4FD12842D02351F
:102F6F0002901A43E0906694F0901A43E075F006D1
:102F7F00A4249B901A6AF0901A437418F002350239
:102F8F00901A6AE0FFE4FD12842D023502901A4375
:102F9F00E0906694F0901A43E075F006A4247190C7
:102FAF001A6AF0F0E4FFFD1280C4901A43EFF002AA
:102FBF003502901A43748CF0023502901A4374A0B4
:102FCF00F0023502901A6AE075F00CA424D8F5824D
:102FDF00E5F03415F583E4F0901A43740BF00235E5
:102FEF0002901A43E0B48E11906C5AE0700BA3E07C
:102FFF007007A3E070030235027F04E4FD7B8C753C
:10300F004D92123DF7E49069C5F00235027F027DC3
:10301F00011280C4901A43EFF0023502901A43E078
:10302F0064A5701D906C54E07017A3E07013A3E0BB
:10303F00700FA3E0700BA3E07007A3E070030235DD
:10304F00027F04E4FD7BA0754DA9123DF7E4906962
:10305F00C5F00235027F017D011280C4901A43EF43
:10306F00F0023502906CE2E060147480FF7E017B09
:05307F00027A6C7945A6
:10308400756000756101120A67906CE2E0FF6006EA
:10309400906C45E06009EF70119003A1E0700B7F24
:1030A40001E4FDFB1296CB023502901A43E0B422F0
:1030B40005747FF08016901A43E0B423057480F001
:1030C400800A901A43E0B40903747EF0E4902F2F31
:1030D400F0023502901A437434F0023502901A4318
:1030E400742DF0023502901A437439F002350290BF
:1030F40069C27402F0901A43F002350212A154EF2F
:10310400B40109901A43743CF0023502901A4374D6
:1031140039F0023502901A43E025E024DFF582E419
:10312400347BF583E0FFA3E09065E3CFF0A3EFF0F9
:10313400901A43E0244FF582E4347CF583E0701E5A
:10314400907CB37478F0907CB27401F0907CB47489
:1031540039F0907C7F741FF0A37486F0801C907CFF
:10316400B37404F0907CB27402F0907CB47441F0B7
:10317400907C7F7419F0A3749AF012D21CE4FF902F
:1031840065E3E0FCA3E0FD12DD12E49069C2F09077
:103194001A437402F0023502901A437450F0023557
:1031A40002901A437402F0023502901A437455F0E7
:1031B400023502901A43745FF0023502901A437488
:1031C40022F0023502901A43745AF0023502E49058
:1031D4001A69F0901A437461F0023502901A43742C
:1031E40062F0023502901A437460F00235027E00E8
:1031F4007F0B7D007B027A69799912ED477B057A12
:10320400A179CF129D5E7F417D327BAF75664612F8
:10321400092B7F557D6C7B057AA179E61204C512D2
:10322400033FE4F546E546C394045066E4F547E5F8
:1032340047C394805058129366908002E0F52A5454
:10324400087002FF22E54775F080A4FDE546C4330B
:103254003354C0FEE42DFFEE35F0FE7B057AA279EF
:1032640005754F80120AFDE547543F701D129366A1
:10327400AF480548EF75F00CA4244BFF7D377B0560
:103284007AA279061205A812033F054780A10546D4
:103294008093E4906C45F0901A69F0901A4374613D
:1032A400F0023502901A69E0FFC3940A50437499FE
:1032B4002FF582E43469F583E0FF647B6003EF70EB
:1032C40030901A69E0FFFDC3740A9DFDE49400FC8C
:1032D400C004C0057E0074992FF9E43469FA7B02B6
:1032E400AD06D007D00612ED47901A69740AF08033
:1032F40006901A69E004F0901A69E0640A60030217
:103304003502FF7E017B027A697999755C0B120B99
:1033140089901A43745AF0023502E4906C45F074B3
:1033240080FF7E017B027A6C7945755C01120B8902
:103334007F07E4FDFB1296CB901A43745BF00235D1
:10334400027F01124A08023502906821E06004E419
:10335400F080069068217401F0901A43742FF012E3
:10336400443B023502901A437428F09065F412EC41
:103374008E00000000023502901A437432F00235C8
:013384000246
:103385007F01124942901A43742DF00235029003D1
:10339500A1E0D394004009901A437433F00235023A
:1033A5007F06E4FDFB1296CB901A43742EF002358E
:1033B500027F01124989901A43742EF00235027F6B
:1033C50002E4FDFBF54D123DF79069B9E0D3940099
:1033D5004029E025E0244FF582E434CAF583E493DF
:1033E500FC740193FD7E007F6412EA4890669BEFB2
:1033F500F0E0FFC31390669AF08009E490669BF0B5
:1034050090669AF012033F0235029066947409F0B3
:103415007F067D0212842D023502901A437481F0D5
:10342500E4906CDDF0A3F0906CDBF0023502901AAD
:10343500437482F0E4906CDDF0A3F0906CDBF00255
:103445003502906CDBE064017012901A43E0B4829F
:10345500057481F08006901A437482F0906CDBE06D
:1034650060047F0080027F01906CDBEFF002350283
:10347500901A437424F0023502901A437451F012E5
:1034850053FE023502901A437405F0E4FF129CB016
:10349500023502901A437426F012443B805F901A5D
:1034A50043E024FB605124DD604524F9602924DFD5
:1034B500602D146032242B7044906821E0700690D2
:1034C5001A44E06008901A4374BBF080307F04E42E
:1034D500FDFB1296CB8026901A437435F0801E9022
:1034E5001A4374B4F08016901A4374B5F0800E90A8
:1034F5001A4374B7F08006901A4374B6F07F012220
:10350500901A43E012ED2136330236330336330485
:103515003633053633063648073648083648093601
:10352500480A36480B365E0C365E0D365E0E365E44
:103535000F365E10365E11367412367413367414F7
:1035450036741536741636741736991836B9193611
:10355500B91A36B91B36B91C36B91D36B91E36DE51
:103565001F36DE2036DE21372F22372F23372F2433
:1035750037532637532737532837692D37692E3761
:10358500692F38B83238C63338623438D435377F86
:1035950039377F3A37953C37953D37953E37953FD7
:1035A50037954037954137AB5037BF5137FF5537C2
:1035B500FF5637FF5738265A38265B38265C3815AC
:1035C5005F38EF60383C6138FC6237D37037D371B0
:1035D50037E972384D7E385A7F385A8038738138CA
:1035E500918237038C37038D37038E37038F37036B
:1035F500903703913703923719A03719A13719A2CC
:103605003719A33719A43719A53719A63719A737B5
:1036150019A83719A93916B43930B5394AB6392335
:10362500B7393DB83957B93909BB00003962E4FFEC
:103635007B057AA27908901A43E014F551126E0AB7
:103645000239627F017B057AA27914901A43E0243E
:10365500FAF551126E0A0239627F027B057AA27968
:103665001E901A43E024F5F551126E0A0239627F65
:1036750003906C4BE0B408087B057AA2793180068B
:103685007B057AA27946901A43E024EFF551126E34
:103695000A0239627F04906C4BE0B408087B057A16
:1036A500A2795880067B057AA2796C7551FF126E56
:1036B5000A0239627F05906C4BE0B408087B057AF5
:1036C500A2797D80067B057AA27995901A43E0243C
:0636D500E8F551126E0A37
:1036DB000239627F0A906C4BE0B408087B057AA232
:1036EB0079AA80067B057AA279BB901A43E024E283
:1036FB00F551126E0A0239627F107B057AA279C9E5
:10370B00901A43E02475F551126E0A0239627F114B
:10371B007B057AA279DC901A43E02461F551126E95
:10372B000A0239627F3C906CE2E060087B057AA26A
:10373B0079F380067B057AA37904901A43E024DFA2
:10374B00F551126E0A0239627F067B057AA3790D59
:10375B00901A43E024DBF551126E0A0239627F0B9B
:10376B007B057AA37915901A43E024D4F551126E98
:10377B000A0239627F0C7B057AA37924901A43E005
:10378B0024C8F551126E0A0239627F0D7B057AA3AC
:10379B00792F901A43E024C5F551126E0A02396253
:1037AB007F147B057AA37940E4F551126E0A120956
:1037BB00830239627F157B057AA3794EE4F55112AA
:1037CB006E0A1209830239627F287B057AA3796519
:1037DB00901A43E02491F551126E0A0239627F2947
:1037EB007B057AA3796F901A43E0248FF551126E03
:1037FB000A0239627F2A7B057AA37979901A43E012
:10380B0024ACF551126E0A0239627F2D7B057AA327
:10381B007983E4F551126E0A0239627F2B7B057AAC
:10382B00A37994901A43E024A7F551126E0A02393A
:10383B00627F2C7B057AA379A7E4F551126E0A02FD
:10384B003962E4906C47F07F04127A930239627FFD
:10385B0002127A930239627F3D7B057AA379BAE42F
:10386B00F551126E0A0239627F08E4FD7B01125B8F
:10387B0089906820E070030239627F04E4FD7B01CC
:10388B00128EEA023962906CDDE0FEA3E0FF7DFF51
:10389B0012199A7F18127A93906820E070030239FC
:1038AB00627F04E4FD7B01128EEA0239627B057AAA
:1038BB00A379CD7D011278A60239627B057AA379B3
:1038CB00DD7D011278A6023962906821E060087BE9
:1038DB00057AA379F380067B057AA479097D011219
:1038EB0078A680737B057AA4791F7D011278A68058
:0C38FB00667B057AA479307D011278A666
:1039070080597B057AA479487D011278A6804C7B83
:10391700057AA479597D011278A6803F7B057AA4A0
:10392700796C7D011278A680327B057AA47981E4CF
:10393700FD1278A680257B057AA4799D7D011278F2
:10394700A680187B057AA479B0E4FD1278A6800BCF
:0F3957007B057AA479C87D011278A612033F225E
:10396600D2C1C2AFC2A875F60375B71075B8307567
:10397600F702E4F5F843A70712936690800374896B
:10398600F0908000E528F0A3E529F0A3E52AF0539E
:1039960029DF908001E529F07F0A7E0012936D43AE
:1039A6002920908001E529F0120146E4FF12023F2A
:1039B60012033F75F63FE4F5F275F320D2E9C2CD66
:1039C600C2CCC2C9C2C8C2CBF5C975CB70F5CA751F
:1039D600CD70F5CCD2CAD2ADC2B3C2C2901A42F0F3
:1039E60012CCD012004612D21C432980908001E5E9
:1039F60029F0D288123B66E4901A44F012931FEF26
:103A060060067E007F0080047E007F0012936DD2E8
:103A1600AFD2A89069C2E070179065E3E07002A388
:103A2600E0600DE4FF9065E3E0FCA3E0FD12DD122B
:103A36001295EC901A43E0906694F07F04123FEFE3
:103A4600906991E06401703D906694E0901A43F0AD
:103A5600E02487600824FB50112406701A901A434C
:103A66007402F0901A6B7480F022901A437403F07B
:103A7600901A6B7480F022901A437402F0E4901A44
:063A86006BF01235052271
:103A8C007E007F667D007B027A1D798E12ED4712D7
:103A9C004A87E4907BE8F0901A68F0906C75F0A37C
:103AAC00F09065EBF09065EAF09069B0F0902D8B9A
:103ABC00F090667CF0906C6CF09003A0F030920467
:103ACC007F0180027F00906C74EFF0906C65F03099
:103ADC0094047F0180027F00906CDAEFF0906C68A8
:103AEC00F0C208D20BC20EE4906992F09065E9F036
:103AFC009069C0F09065ED12EC8E000000009069AA
:103B0C008C12EC8E00000000E4902D81F09066A0E9
:103B1C00F0902F32F0902F3104F0E4901DFAF090D9
:103B2C007BE9F0901DF5F0902D7EF0906CDFF0A30A
:103B3C00F0902F2DF0A3F09069BEF0A3F090669258
:103B4C00F0A3F0906822F0A3F090039CF0A3F09007
:0A3B5C0069BA12EC8E00000000228E
:103B6600E49066B0F0906C72F090681E04F07E00EF
:103B76007F407D007B027A0179C812ED47E49065AB
:103B8600E8F0906C4BF090699104F0E49017E3F044
:103B9600A3F09069C5F09066ACF0902D8004F0E437
:103BA6009065ECF0901DF4F0902D8AF0901DFBF0DE
:103BB600906C47F090039EF0C20D9013A6F09068AB
:103BC60020F0901A44F0902F2FF0906CDDF0A3F0C7
:103BD6009069B2741EF0E4906993F0901A6B74FFCA
:103BE600F0E4906819F0A3F0123A8C7E107F007D05
:103BF600007B027A0379A212ED4790669512EC8E4D
:103C0600000000007E007F0C7D007B027A6679034F
:103C160012ED47E49002D1F0906C6D12EC8E00002C
:103C260000009069A412EC8E000000009003A1E051
:103C3600D39400405DE0FF7E007C007D6312E9DFE7
:103C460074BE2FF9741D3EFA7B02C00378C67C69E8
:103C5600AD03D0037E007F0612E94F9069C9E004E8
:103C6600F070069069C8E004F0D39069C9E094FF4B
:103C76009069C8E0943F4029E4F0A3F09069C7E05A
:103C860004F0E0D3941F4019E4F09069C6E004F014
:103C9600800F7E007F067D007B027A6979C612ED71
:103CA600479069C6E0D3940340047F0180027F00F9
:103CB600906615EFF0C39069CBE094789069CAE0FE
:103CC600940540047F0180027F00906C73EFF090B2
:103CD600CA57E493FF9069B9E0C39F4003EF14F01D
:103CE6009069B9E0D394004029E025E0244FF5829D
:103CF600E434CAF583E493FC740193FD7E007F648B
:103D060012EA4890669BEFF0E0FFC31390669AF0C4
:103D16008009E490669BF090669AF090CA3BE49323
:103D2600FF9066ABE0C39F4002E4F090CA42E49382
:103D3600FF906C71E0C39F40037402F090CA47E4A1
:103D460093FF901A6DE0C39F4002E4F090CA4EE4E0
:103D560093FF9065FEE0C39F4002E4F09069C2E0E5
:103D6600D394024002E4F0901A457402F0A3741D45
:103D7600F0A374B6F0A37402F0A3741DF0A3749AB2
:103D8600F0A37402F0A3741DF0A374C2F0A374022E
:103D9600F0A3741DF0A3748EF0A37402F0A3741D37
:103DA600F0A374C6F0A37402F0A3741DF0A3749676
:103DB600F0A37402F0A3741DF0A374BAF0A3740206
:103DC600F0A3741DF0A3749EF0A37402F0A3741DF7
:103DD600F0A374BEF0A37402F0A3741DF0A3749252
:103DE600F0A37402F0A3741DF0A374FAF0129DF10F
:013DF60022AA
:103DF7008D4B8B4CEF147003023F03147003023F8B
:103E070046147003023F89147003023FBD14700308
:103E1700023E8724056003023FEB901DFBE0600C28
:103E270090CA3CE49314900029F0800A90CA3BE4BE
:103E37009314900029F0E54B14601C04702F900038
:103E470029E0FF9066ABE0C39F5005E004F0801DBA
:103E5700E49066ABF080169066ABE0D39400400523
:103E6700E014F08008900029E09066ABF09065E9D7
:103E77007401F0E4906992F07F01124568023FEB0C
:103E8700E54B14601E04703390CA42E49314FF900C
:103E97006C71E0C39F5005E004F0801FE4906C71E3
:103EA700F08018906C71E0D394004005E014F08026
:103EB7000A90CA42E49314906C71F0906C47E060EA
:103EC70003023FEB901A43E0647B600EE0647D6081
:103ED70009E0647A6004E0B47C129013A3E0C39411
:103EE7000640099069AEE06003023FEB906C71E019
:103EF700608EE064016003023FEB8084E54B146051
:103F07001E04703390CA47E49314FF901A6DE0C300
:103F17009F5005E004F0801FE4901A6DF080189020
:103F27001A6DE0D394004005E014F0800A90CA4768
:103F3700E49314901A6DF07F01124568023FEBE598
:103F47004B146023046003023FEB90CA57E49314B9
:103F5700FF9069B9E0C39F5006E004F0023FEBE42D
:103F67009069B9F0023FEB9069B9E0D3940040063D
:103F7700E014F0023FEB90CA57E493149069B9F04C
:103F87008062E54B14600B0470159065FEE004F049
:103F9700800D90CA4EE49314FF9065FEE02FF090D9
:103FA70065FEE0FF90CA4EE493FEEF8EF0849065C5
:103FB700FEE5F0F0802EE54B146014047020901A93
:103FC70043E004F0E0D3954D4014E54CF0800F90AA
:103FD7001A43E014F0E0C3954C5003E54DF09069A7
:083FE700C57401F0129366227B
:103FEF008F45E490002CF090002EF0E54520E30380
:103FFF000240CF9066B0E0600890002C7417F080FC
:10400F0047D3906C76E094C0906C75E0945D400857
:10401F0090002C740EF0803090CA17E493FE740158
:10402F0093FFC39066A8E09F9066A7E09E50149000
:10403F006993E004F0E0C39432400D90002C740DAE
:10404F00F08005E4906993F090002CE060727F019E
:10405F00124B0090002CE0FFE4FDFB1296CBE4FF27
:10406F0012023F12033F9065F412EC669066111234
:10407F00EC827F087E00906611E0FD12DF5A7F0907
:10408F007E00906612E0FD12DF5A7F0A7E00906676
:10409F0013E0FD12DF5A7F0B7E00906614E0FD12D5
:1040AF00DF5A12DF6C7FD07E0712936DC2C17F641F
:1040BF007E0012936DD2C17F647E0012936D80ECEF
:1040CF00E54530E457906991E064016007E4901A88
:1040DF006BF08048901A6BE0FF6041E4906C75F0D4
:1040EF00A3F090002DEFF0E4901A6BF09065E87458
:1040FF0002F053287F908000E528F012217AEF64B8
:10410F00017019901A43E0FF90002EE06F600D9040
:10411F001A43E090002EF012350580E7E54530E0B8
:10412F0058901A43E0B4BF037F01229065ECE06022
:10413F00489065F412EC6612ECCF7F017E007D0093
:10414F007C0012EAAC9065F412EC8278957C697D64
:10415F00027B027A66799C7E007F0312E94F7F040F
:10416F00E4FD7B01128EEA906820E06007E4906C1A
:10417F0075F0A3F0E49065ECF0E54520E10620E250
:10418F00030242C5908002E0F52A540890002BF0FC
:10419F007019906991E0701304F0E4906C4BF090FB
:1041AF001A437402F01235050242C590002BE0FF4E
:1041BF00906C4BE0FE6F70030242C5EE600302424B
:1041CF00A97F01124B00E4FF7E017B027A69799986
:1041DF00F56075610B120A67EF7015906991F09099
:1041EF001A437402F07F16E4FDFB1296CB7F002278
:1041FF00E49069A3F090002AF090002AE0FFC394A6
:10420F000B502174992FF582E43469F583E0FFC3D5
:10421F0094414006EFC3947B4002E4F090002AE003
:10422F0004F080D57480FF7E017B027A6C7945752E
:10423F006000756101120A67906C45E0FFD394002E
:10424F004039EF1475F040A42400FFE5F03414FE5C
:10425F007B027A6C7977756000756127120A67D3D4
:10426F00906C7AE094F5906C79E094FF40047F01B4
:10427F0080027F009013A2EFF08005E49013A2F06C
:10428F00906999E0700C901A69F0901A437461F07C
:10429F00800E901A437470F08006901A437472F077
:1042AF0090002BE0906C4BF09069917401F0E54514
:1042BF0030E103123505E54530E608300C05121ED6
:1042CF002FC20CE54520E50302435E901DF4E0602C
:1042DF0007E4FF124B008027902D8AE060217F05B5
:1042EF00E4FDFB1296CB7F01124B00EF700E901A7C
:1042FF00437402F0901A6B7480F0800312350590AE
:10430F0065EBE06011E4F090667CE060047F018073
:09431F00027F00125A2D9066ACD9
:10432800E064017031F0906820E0600F9013A3E022
:1043380004F0E0FFE4FD1284AA801B7F01124B0009
:10434800906C47E0600690039E7401F09013A3E020
:09435800FF7D011284AA7F0122FD
:10436100902D8BE0600B7F64E4FDFB1296157F01BD
:04437100227F002285
:10437500E490002FF0906615E06003024425901745
:10438500E0E0FEA3E07802CEA2E713CE13D8F8FF53
:104395001294F69017E0E0FEA3E07806C333CE331F
:1043A500CED8F954C0FF90002FE02FF0902D83E078
:1043B500600790002FE04420F0906990E06007903E
:1043C500002FE04410F0901DFAE0900030F0300B23
:1043D50047902D7EE0FF700F90002FE0240FF090A6
:1043E5002D7E7401F08031EFB40119900030E0FFAB
:1043F500C4540F540FFF90002FE02FF0902D7E74C2
:1044050002F08014900030E0540FFF90002FE02F51
:10441500F0E4902D7EF0C20B90002FE0FF1294F691
:10442500906615E0600F901DB612EC6612E52190BE
:064435006C9E12EC8222D5
:10443B00E4900031F090003512EC8E0000000090FB
:10444B002D8BE060167F23E4FDFB1296157F0FE4A6
:10445B00FDFB1296CB7F0112456822901A43E0FFB9
:10446B00900033E4F0A3EFF0E4901A43F07B057A6D
:10447B00A479D7129D5E7F417D327BAF7566461264
:10448B00092B12033FC2ADE4900032F0900032E0F2
:10449B00C394C8505812936690003512EC6612EC18
:1044AB00CF7F011293A8E4FCFD12EAAC9000351209
:1044BB00EC827F057E0012936D900032E075F0194F
:1044CB0084E5F07020129366900031E0FF04F0EF6A
:1044DB0075F00CA4244BFF7D377B057AA27906126D
:1044EB0005A812033F900032E004F0809F90003546
:1044FB0012EC6612ECCF7FC87E007D007C0012F5BB
:10450B001C12ECEE9013ADEEF0A3EFF0906821E0EF
:10451B0060099013ADE4F0A37464F01220E37F0103
:10452B007D0212906F900034E0901A43F0E4FF127A
:10453B00023F901A43E064786018E064796013E0FE
:10454B00647A600EE0647C6009E0647B6004E0B434
:0D455B007D057F01124568123505D2AD22A5
:104568008F4EE4FF12023F90681D7401F09066AB15
:10457800E090CA349324FA600E1470149017E3E4A0
:10458800F0A3742DF080099017E3E4F0A37442F0CF
:104598009066ABE090CA349324FE604E1470030218
:1045A800462914607C24FC400302468624086003E4
:1045B80002474B7FDB7D3C7B057AA479E81204C572
:1045C8007F697D507B057AA479ED1204C57F697DEA
:1045D8005A7B057AA479E81204C57FDB7D587B05F0
:1045E8007AA479F11205A802474B7FDB7D3C7B0555
:1045F8007AA479F31204C57F697D507B057AA47982
:10460800F51204C57F697D5A7B057AA479FB1204EB
:10461800C57FDB7D587B057AA479F11205A802478E
:104628004B9066ABE090CA3493B4030F7FDB7D3CBC
:104638007B057AA479FE1205A8800D7FDB7D3C7B83
:10464800057AA579001204C5901A43E0647D6004D8
:10465800E0B47C0D7F697D507B057AA5790512044D
:10466800C57F697D5A7B057AA5790A1204C57FDB67
:104678007D587B057AA479F11205A802474B901A58
:104688006DE090CA439314603714605D14605A2437
:1046980003600302473E7FDB7D3C7B057AA479E813
:1046A8001204C57FDB7D507B057AA479ED1204C521
:1046B8007FDB7D5A7B057AA479E81204C502473E60
:1046C8007FDB7D3C7B057AA479F31204C57FDB7D13
:1046D800507B057AA479F51204C57FDB7D5A7B05EA
:1046E8007AA479FB1204C5804D901A6DE090CA43F4
:1046F80093B4020F7FDB7D3C7B057AA479FE12051B
:10470800A8800D7FDB7D3C7B057AA579001204C566
:10471800901A43E0647D6004E0B47C0D7FDB7D503B
:104728007B057AA579051204C57FDB7D5A7B057A5E
:10473800A5790A1204C57FDB7D767B057AA479F119
:104748001205A89066ABE090CA3493D39404400352
:104758000248B1906C71E090CA3D9324FE70030248
:1047680047F014700302482714700302485D147060
:104778000302485D240460030248B19000397404C0
:10478800F0900039E0C394CB5013E0FF7D72240809
:10479800FB12000C900039E02410F080E4906C6665
:1047A80074BEF07FD07D647B7F12002E901DFBE0ED
:1047B800600F7FD67D687B057AA5790C1204C580C9
:1047C800097FD07D727BEF12000C906C66E0FCE4F0
:1047D80012E4ED12ECCF906C4C12EC6612E3E5900B
:1047E8007BE312EC820248B17F697D6E7B057AA576
:1047F80079111204C57F697D787B057AA479E8125E
:1048080004C57FDB7D6E7B057AA579161204C57F0A
:10481800DB7D787B057AA579001204C50248B17F53
:0C482800697D6E7B057AA579111204C52C
:104834007F697D787B057AA479E81204C57FDB7DE6
:104844006E7B057AA579111204C57FDB7D787B0523
:104854007AA5791B1204C580547F697D6E7B057A25
:10486400A479ED1204C57F697D787B057AA479FE6D
:104874001205A8906C71E090CA3D93640570187F8E
:10488400DB7D747BE512000C7FDB7D767B057AA4EF
:1048940079F11205A880167FDB7D717BE712000C8D
:1048A4007FDB7D737B057AA5791F1205A87FDB7DED
:1048B4000A7B057AA5791F1205A8E4FF7D1A7BEF10
:1048C40012000CE4FF0D12000C9066ABE090CA34A9
:1048D400931460540424FB500624FD502C80497F1B
:1048E4007FE4FD7B1A12002E7F7F7D497B641200DA
:1048F4002EE4FF7D477BEF12000CE4FF0D12000C49
:10490400E4FF7D6412000C801F7F7FE4FD7B7F1237
:10491400002E7F7F7D477BEF12000C7F7F0D1200FE
:104924000C7F7F7D6412000CE490681DF07F077D8E
:0E493400017B01128EEAE54E600312033F2262
:104942008F4AC2AFE49003A1F0FE7F06FD7B027A9C
:104952006979C612ED47E4906615F0906C73F07EAB
:104962000F7F78FD7B027A1E790212ED47D2AFE506
:104972004A60087F06E4FDFB1296CB124DE67F31BA
:07498200E4FDFB1296152273
:104989008F4A9003A1E0D394004057E014F0E0FF70
:104999007E007C007D6312E9DF741B2FF9741E3ED3
:1049A900FA7B02C00378C67C69AD03D0037E007F21
:1049B9000612E94F9069C6E0D3940340047F018051
:1049C900027F00906615EFF0C39069CBE094789070
:1049D90069CAE0940540047F0180027F00906C73EE
:1049E900EFF0E54AB4010C7F129003A1E0FDE4FB6E
:0F49F9001296CB124DE67F3FE4FDFB129615227E
:104A08008F4AE4906821F090CA5793149069B9F0DE
:104A1800E025E0244FF582E434CAF583E493FC747E
:104A28000193FD7E007F6412EA4890669BEFF0E0F8
:104A3800FFC31390669AF0E49066ABF0906C7174C3
:104A480002F0E49069AEF0901A6DF0906C6904F091
:104A58009065F3F0FE7FB07D007B027A16792C1208
:104A6800ED477F01E4FD12549FE54A60117F15E48C
:0F4A7800FDFB1296CB901A437450F012350522B5
:104A8700C2AF1293667E037F207D007B027A1A797C
:104A97006E12ED47E4901A6CF09013A5F09013ACEA
:104AA700F0907BE7F090698C12EC8E00000000908C
:104AB70065ED12EC8E00000000E49066A0F0902DEA
:104AC70081F090039CF0A3F0906692F0A3F0901D04
:104AD700F6F07E017F5CFD7B027A1379B312ED4716
:104AE7007E007F067D007B027A66798C12ED47E4B3
:094AF7009065E6F0A3F0D2AF22B5
:104B00009002D27401F0EF147003024B980460031A
:104B1000024DE0E4FF12E08C78807C6C7D027B0229
:104B20007A6679A17E007F0612E94F906C4BE064B3
:104B3000087056906C45E0FFD39400403BEF14752D
:104B4000F040A42400FFE5F03414FE7B027A0079E3
:104B50003C756000756104120A6790003EE0FEA398
:104B6000E0FF906C77EEF0A3EFF02428906C7AF0E1
:104B7000E43E906C79F08011906C777440F0A3E47F
:104B8000F0A37440F0A37428F0E4901DF4F07F3992
:104B9000FDFB129615024DE0E4907BE8F0902D8B22
:104BA000E07003024DDBE4901DFBF0906C47F09049
:104BB0002D8AF090667CF09065ECF0902D8BF09053
:104BC00013A6F0901DB612EC6612E521906C7C12D3
:104BD000EC827F007E007D007C0012ECCF906C9E0A
:104BE00012EC6612EBDC700F901DB612EC6612E54B
:104BF00021906C9E12EC82D3906CE0E09401906C5A
:104C0000DFE094005003024D05D3901DE8E09400CE
:104C1000901DE7E0940050069065EBE06009E49099
:104C200065EBF0FF125A2D906C9AE0FEA3E0FF9026
:104C30006C94E06E7003A3E06F7003024CF6906C0E
:104C400090E0FFD39403503C9069C6E0FED39403F8
:104C50004014906C967403F0A3741FF0A3743FF09B
:104C6000A374FFF0803A906C96EEF09069C7E090E4
:104C70006C97F09069C8E0FDA3E0906C98CDF0A32C
:104C8000EDF0801C906C96EFF0906C91E0906C973A
:104C9000F0906C92E0FFA3E0906C98CFF0A3EFF05F
:104CA0009003A1E0FF7E007C007D6312E9DF7402C7
:104CB0002FF9741E3EA801FC7D027B027A6C797785
:104CC0007E007F6312E94F9003A1E0FF7E007C002D
:104CD0007D6312E9DF743D2FF9741E3EA801FC7D4F
:104CE000027B027A1D798E7E007F2812E94F9003A5
:104CF000A1E004F080557F10E4FDFB1296CBE49018
:104D000002D2F0804678C67C697D027B027A6C799B
:104D1000967E007F0612E94F9069C6E0D394034067
:104D2000047F0180027F00906615EFF0C39069CB8D
:104D3000E094789069CAE0940540047F0180027F86
:104D400000906C73EFF0E49002D2F0906C4BE06452
:104D500008705A906C77E0FEA3E0FF2428FDE43E43
:104D6000FCA3E0FAA3E0FB6D7002EC6A603F7B02FB
:104D70007A1D798E755C28120B89906C45E075F070
:104D800040A42400FFE5F03414FE7B027A6C7977AE
:104D9000755C27120B89906C45E004F07480FF7EEF
:104DA000017B027A6C7945755C01120B899002D205
:104DB000E0602D7F3AE4FDFB1296159003A074018C
:104DC000F0A3E014902F2FF0901A437482F0E49037
:104DD0006CDDF0A3F0906CDBF08005E49002D2F083
:064DE0009002D2E0FF2268
:104DE600E49000A0F09003A1E0D394005003024F9A
:104DF600A2E490009FF09003A1E0FF90009FE0C323
:104E06009F4003024FA274F4FF7E0112936D90003F
:104E16009FE0FF7E007C007D6312E9DF74022FF9BC
:104E2600741E3EFA7B02C00378777C6CAD03D00318
:104E36007E007F6312E94F1200067F007E007D0030
:104E46007C0012ECCF906C9E12EC6612EBDC6002DA
:104E56005003024F99906C91E0FFE4FCFDFE12ECCA
:104E6600CF7F007E407D007C0012EAD312ECCF900B
:104E76006C90E0FFE4FCFDFE12ECCF7F007E007D2F
:104E8600087C0012EAD312EAAC12ECCF906C92E0E6
:104E9600FEA3E0FFE4FCFD12EAAC12ECCF906C97A7
:104EA600E0FFE4FCFDFE12ECCF7F007E407D007C3F
:104EB6000012EAD312ECCF906C96E0FFE4FCFDFE04
:104EC60012ECCF7F007E007D087C0012EAD312EA46
:104ED600AC12ECCF906C98E0FEA3E0FFE4FCFD1270
:104EE600EAAC12EABF9000A112EC8212936690021D
:104EF600D474A5F09002D67418F090009FE0045484
:104F06007F9002D7F0E4A3F078D97C027D027B0281
:104F16007A6C7980FE7F0612E94F906CB1E09002C0
:104F2600DFF0906C86E09002E0F0906CA2E09002D8
:104F3600E1F09000A112EC668F4F8E4E8D4D8C4C99
:104F46007F0F12A00D906C9E12EC668F4F8E4E8DC9
:104F56004D8C4C7F1412A00D906C8712EC668F4F0F
:104F66008E4E8D4D8C4C7F1912A00D906C8B12ECD1
:104F7600668F4F8E4E8D4D8C4C7F1E12A00D7F235B
:104F8600906C8FE0FD7C00129FDF12006F9000A0F6
:104F9600E004F090009FE004F0024DFC9000A0E0D9
:104FA60070077F18FDFB1296157F967E0012936D93
:014FB60022D8
:104FB7008F46901A43E0906694F07F13E54604FD10
:104FC700E4FB1296CBAF467E007C007D6312E9DFDF
:104FD70074022FF9741E3EFA7B02C00378777C6C4B
:104FE700AD03D0037E007F6312E94F1200069002E3
:104FF700D474A4F09002D6744BF07F04906CA3E0B5
:10500700FD7C00129FDF7F08906CB0E0FD7C0012F2
:105017009FDFE49000A5F09000A5E0C39403503112
:10502700E0FE75F005A4240AFFC007EE25E025E0A1
:1050370024A4F582E4346CF58312EC668F4F8E4E10
:105047008D4D8C4CD00712A00D9000A5E004F08088
:10505700C6906C8712EC668F4F8E4E8D4D8C4C7FB1
:105067001912A00D906C8B12EC668F4F8E4E8D4DE2
:105077008C4C7F1E12A00D7F23906C8FE0FD7C006F
:10508700129FDF12006F7F32AD46E4FB129615AF19
:10509700467E007C007D6312E9DF74022FF9741EDF
:1050A7003EFA7B02C00378777C6CAD03D0037E00A9
:1050B7007F6312E94F906C91E0FBFFE4FCFDFE1269
:1050C700ECCF7F007E407D007C0012EAD312ECCF4C
:1050D700906C90E0FFE4FCFDFE12ECCF7F007E00B9
:1050E7007D087C0012EAD312EAAC12ECCF906C92E6
:1050F700E0FEA3E0FFE4FCFD12EAAC901DFC12EC1D
:1051070082906C97E0FFE4FCFDFE12ECCF7F007EFF
:10511700407D007C0012EAD312ECCF906C96E0FF42
:10512700E4FCFDFE12ECCF7F007E007D087C0012C0
:10513700EAD312EAAC12ECCF906C98E0FEA3E0FF42
:10514700E4FCFD12EAAC902F1C12EC829000AC122A
:10515700EC82906C90E090039FF09013A4EBF0909A
:105167006C92E0FFA3E09069CCCFF0A3EFF0902D15
:10517700857452F09002D474E1F09002D67433F043
:10518700901DFC12EC6612ECCF902F1C12EC6612ED
:10519700EABF12ECCF7F52E4FCFDFE12EB3512ECB6
:1051A700F69000ABEFF02401FFE433FE3395E0FD0A
:1051B700FC12ECCF902F1C12EC6612EABF902F1C4A
:1051C70012EC82125237EF60667F017E007D007C11
:1051D7000012ECCF902F1C12EC6612EAAC901DFC6B
:1051E70012EC829000AC12EC66902F1C12EC8290AD
:1051F70000ABE0902D85F0E0FF75F0078475F008AF
:10520700A4FEEF75F00784EE25F024849002D4F015
:10521700125237EF60197F34AD46E4FB12961590B2
:105227006694E0901A43F0E4FF12023F123505221C
:10523700120006901DFC12EC669000B812EC8290EA
:105247002F1C12EC6612ECCF9000B812EC6612EB32
:10525700DC40030253FB129366120006E49000B091
:10526700F09000B2F09000B57403F0A37407F090CB
:105277002D85E0FF9000B0E0FEC39F400302539CE2
:10528700C3EF9E9000B4F0C39407500FE09000B6B0
:10529700F004FF9000B5E02FF080079000B5E02400
:1052A70008F09000B5E024D3F582E43402F583E4F6
:1052B700F09000B704F0E49000B1F09000B6E0FF82
:1052C7009000B1E0C39F400302539390039FE0FF18
:1052D7001392C3EFD394014003D38001C392C45305
:1052E70029E09013A4E04229908001E529F0906914
:1052F700CCE044C0FEA3E0F5828E83E09000B4F0DA
:105307009069CDE004F070069069CCE004F0D3908A
:1053170069CDE094FF9069CCE0943F4018E4F0A396
:10532700F09013A4E004F0E0D3941F4008E4F09059
:10533700039FE004F09000B4E0FF547FFE9000B2BA
:10534700E024D7F582E43402F583EEF0EF30E71F6F
:105357009000B5E024D3F582E43402F583C083C01E
:1053670082E0FF9000B7E0FEEF4ED082D083F0904E
:1053770000B7E0FF25E0F09000B0E004F09000B245
:10538700E004F09000B1E004F00252C29000B2E0F5
:1053970004F002527612006FE4906C75F0A3F07F70
:1053A70037129DC9EF7006901A6BE06029C20CE4B2
:1053B700901A6BF07F37FDFB1296157F14E4FDFB07
:1053C7001296CB906694E0901A43F0E4FF12023FE6
:1053D7001235057F00229000B812EC6612ECCF90D0
:1053E7002D85E0FFE4FCFDFE12EAAC9000B812EC5C
:0753F700820252467F0122F1
:1053FE009065F812EC6690669512EC827F077B0240
:10540E007A66790312A0CE7F0C7B027A6679071238
:10541E00A0CE7F117B027A66790B12A0CE7F187B0D
:10542E00027A0079BC12A0CE9000BC12EC6612E596
:10543E00219002D1EFF0E0FCE412E4ED12ECCF7F0C
:10544E00407EC97D0F7CDB12E36D12ECCF7F447E74
:10545E007A7D007C0012E3E5906C6D12EC82906C0C
:10546E006D12EC6612ECCF90CA2F12EC72EC12E4B5
:10547E00E512E3E59069A412EC827F017D011290A2
:10548E006FE4FF7D0112549F7F1DE4FDFB12961504
:01549E0022EB
:10549F008D4B9000C1744BF0907BE8E09000C0F012
:1054AF00E4907BE8F0EF1470030255D5046003021B
:1054BF005682E54B602A901A43E0FF9000C4E4F057
:1054CF00A3EFF0E4901A43F07B057AA57921129DA2
:1054DF005E7F417D327BAF75664612092B12033F0B
:1054EF00E49000C2F0A3F09000C2E0FCA3E0FDC383
:1054FF0094FFEC940340030255BBE412E4E912EC71
:10550F00CF90660B12EC6612E36D12ECCF9066072C
:10551F0012EC6612E26212ECCF9000C2E0FCA3E044
:10552F00FDE412E4E912E36D12ECCF90660312EC86
:10553F006612E26212ECCF90CA2F12EC72EC12E4F8
:10554F00E512E36D12E52112ECCF9000C2E0FEA34D
:10555F00E07802C333CE33CED8F924A2F582EE34ED
:10556F0003F58312ECEE12EC82129366E54B602B7F
:10557F009000C2E0FEA3E0FF547F701FEF7807CECC
:10558F00C313CE13D8F975F00CA4244BFF7D377BD2
:10559F00057AA279061205A812033F9000C3E00412
:1055AF00F070069000C2E004F00254F6E54B700371
:1055BF000256829000C5E0901A43F0E4FF12023FBA
:1055CF001235050256821293669000C612EC8EDBDE
:1055DF000FC93FE49000C2F0A3F0C39000C3E09462
:1055EF00689000C2E0940140030256829000C612F8
:1055FF00EC6612F3F412ECCF7F427EC87D007C0084
:10560F0012E36D12E5219000C2E0FCA3E024B1F596
:10561F0082EC3466F583EFF01293669000C2E0FEE1
:10562F00A3E0FF24B1F582EE3466F583E0FBEF24AF
:10563F005AFFE43EFE7C017D6812E9F374242DF5D8
:10564F0082EC3468F583EBF09000C612EC6612EC36
:10565F00CF7F3C7E8E7DFA7C3512E2629000C612BF
:10566F00EC829000C3E004F070069000C2E004F0FA
:0C567F000255E99000C0E0907BE8F022AA
:10568B001293667F457EBB7D807C0012ECCF9068C9
:10569B001BE0FCA3E0FDE412E4E912E3E5901DBA84
:1056AB0012EC8290681BE0FCA3E0FDE412E4E9122B
:1056BB00ECCF7F427EC87D007C0012E3E5901DD6C7
:1056CB0012EC82901DE312EC6612ECCF901DD612F9
:1056DB00EC6612E262901DE312EC82901DD212EC8A
:1056EB006612ECCF901DD612EC6612E262901DD2C0
:1056FB0012EC821293667F417EA07D007C0012EC3F
:10570B00CF901DBA12EC6612E4945003025A297F13
:10571B00437EC87D007C0012ECCF901DBA12EC6664
:10572B0012E49460054003025A29901DE2E004F054
:10573B00901DB212EC6612ECCF7F017E007D007CD7
:10574B000012EAAC901DB212EC82902D82E060FA4E
:10575B00E4902D82F0901DBA12EC6612ECCF901DE6
:10576B00AA12EC6612E494500C901DBA12EC6690DF
:10577B001DAA12EC82901DB212EC66E412E4E51243
:10578B00ECCF901DD212EC6612ECCF7F427E707D77
:10579B00007C0012E3E512E3E5901D9E12EC82D330
:1057AB00906693E09400906692E09400403C906881
:1057BB0022E0FCA3E0FDE412E4E912ECCF90669248
:1057CB00E0FCA3E0FDE412E4E912E3E5901DCE1248
:1057DB00EC82901DAE12EC6612ECCF901DCE12EC4B
:1057EB006612E262901DAE12EC82902D82E060FA9E
:1057FB00E4902D82F0902D8612EC66EC12E4E5120B
:10580B00ECCF90681BE0FCA3E0FDE412E4E912E3AB
:10581B00E512ECCF9069A412EC6612E36D901DBEFD
:10582B0012EC827F007E007D007C0012ECCF901D7D
:10583B00BE12EC6612E494500A901DBE12EC8E0060
:10584B00000000901DE912EC6612ECCF901DBE1209
:10585B00EC6612E262901DE912EC82901D9212EC42
:10586B006612ECCF901DBE12EC6612E262901D9296
:10587B0012EC82129366901DBE12EC6612ECCF9066
:10588B001DD612EC6612E3E5901DC212EC82901D40
:10589B009212EC6612ECCF901DD212EC6612E3E57D
:0958AB00901D8E12EC82901DC2CA
:1058B40012EC6612ECCF901DA612EC6612E4945022
:1058C4000C901DC212EC66901DA612EC82902D82E3
:1058D400E060FAE4902D82F0FFFEFDFC12ECCF9024
:1058E4001DC212EC6612E49460324030901DC21264
:1058F400EC6612F2B112ECCF7F3E7EBD7D2F7C1B95
:1059040012E36D12F21512ECCF7F407EA77D347C3A
:10591400D712E36D901DC612EC82800A901DC61248
:10592400EC8E00000000901DD612EC6612ECCF90B5
:105934001DC612EC6612E36D12ECCF7F407E667DCD
:10594400667C6612E3E5901DCA12EC82902D82E01B
:1059540060FAE4902D82F0901A43E0647D706590C3
:105964006C4C12EC6612ECCF901DCA12EC6612EC71
:10597400CF901D9A12EC6612E26212E494404590B4
:105984001DED12EC6612ECCF901D9A12EC6612EC2F
:10599400CF906C4C12EC6612E25E12E262901DED46
:1059A40012EC82906C4C12EC66901D9A12EC829070
:1059B4001DFBE06007E4907BE8F080389066AC74EF
:1059C40001F08030901DED12EC6612ECCF901DCAF0
:1059D40012EC6612E262901DED12EC82901D9A1296
:1059E400EC6612ECCF901DCA12EC6612E262901DB6
:1059F4009A12EC82902D82E060FAE4902D82F0906D
:105A04001D9A12EC6612ECCF901DD212EC6612E3D2
:105A1400E512ECCF7F407E667D667C6612E36D9076
:095A24001D9612EC821293662219
:105A2D008F4A901DE2E07003025B88786A7C667D88
:105A3D00027B027A1D79E27E007F1212E94F7E0011
:105A4D007F0A7D007B027A66797E12ED477F447E68
:105A5D007A7D007C0012ECCF90666B12EC6612E33F
:105A6D006D12E52190667EEEF0A3EFF090667AE080
:105A7D00FFA3E0906685CFF0A3EFF07F3F7E007D22
:105A8D00007C0012ECCF90667112EC6612E262128D
:105A9D00E521906680EEF0A3EFF07F417E207D0042
:105AAD007C0012ECCF90667512EC6612E36D12E578
:105ABD0021906682EEF0A3EFF090666AE090668426
:105ACD00F0906679E0906687F09013A2E0703E90BA
:105ADD006C4BE064087036906C79E0FEA3E0FFD368
:105AED0094F5EE94FF501C7B027A66797E755C0A04
:105AFD00120B89906C7AE0240AF0906C79E03400F6
:105B0D00F0800A9013A27401F0906C7BF0906C738E
:105B1D00E070599069CAE0FEA3E0FFC39478EE945B
:105B2D0005503F7C007D0A12E9DF74332FF9742F85
:105B3D003EA801FC7D027B027A66797E7E007F0A9B
:105B4D0012E94F9069CBE004F070069069CAE00449
:105B5D00F09069CAE0FFA3E0906C9ACFF0A3EFF04C
:105B6D00800A906C737401F0906C9CF07E007F1233
:0C5B7D007D007B027A1D79E212ED4722C8
:105B89008F548D558B56129366E55424FB24FD5092
:105B9900087003025DD7026126901A6DE090CA432E
:105BA90093147003025C42147003025CE5147003E1
:105BB900025CE5240360030261267F3F7E007D00CD
:105BC9007C0012ECCF90664A12EC6612E26212E592
:105BD900219000DAEEF0A3EFF0C394E8EE940340CD
:105BE900277F837D207B057AA579361207727B058D
:105BF9007AA5793A9000DAE0FCA3E0FD129ECF7F06
:105C0900907D2D1206EB80187B057AA5793E9000D0
:105C1900DAE0FCA3E0FD129ECF7F837D20120768A6
:105C29007B057AA5793A90661612EC66129F077F72
:105C3900907D4B1206EB0261267F3F7E007D007C42
:105C49000012ECCF90664612EC6612E26212E52170
:105C59009000DAEEF0A3EFF0C394E8EE9403402746
:105C69007F837D207B057AA579361207727B057AB9
:105C7900A5793A9000DAE0FCA3E0FD129ECF7F906F
:105C89007D2D1206EB80187B057AA5793E9000DA06
:105C9900E0FCA3E0FD129ECF7F837D201207689070
:105CA900661A12EC6612ECCF7F447E7A7D007C0086
:105CB90012E3E59000E312EC82902D84E06004E4A5
:105CC900F080DC7B057AA5793A9000E312EC661244
:105CD9009F077F907D4B1206EB026126901A6DE0BB
:105CE90090CA43936402704B7F417E20FDFC12EC05
:105CF900CF90664E12EC6612E36D12E5217C007DB1
:105D09000A12E9F37B057AA57942129ECF7FB87D05
:105D19002D1206EB90664E12EC6612E521AC06AD2B
:105D2900077B057AA57947129ECF7F837D201207CD
:105D390068800CE4FF129F4F7F877D2D1206EB7F51
:105D4900107E277D007C0012ECCF906C6112EC660E
:105D590012EBDC4051906C6112EC6612ECCF7F10B3
:105D69007E277D007C0012EB3512ECEEAD07AC0608
:105D79007B057AA57947129ECF7F817D4B12059EBF
:105D8900906C6112EC6612ECCF7F107E277D007C4F
:105D99000012EB3512ECF6AD07AC067B057AA57956
:105DA9004B129ECF801E7F817D4B7B057AA579366C
:105DB9001205A87B057AA5793A906C63E0FCA3E00B
:105DC900FD129ECF7F907D4B1206EB026126E4FF08
:105DD90012023F906820E060087B057AA57950801F
:105DE900067B057AA37904129D5E9000D37411F0A5
:105DF900E49000DAF0A3F09000F712EC8E000000B6
:105E090000E49000CFF0906CE2E06019906C77E0CC
:105E1900FEA3E0FF7B027A1D798E7560007561280B
:075E2900120A678013788E56
:105E30007C1D7D027B027A6C79B27E007F2812E99C
:105E40004F9066AEE0FCA3E0FD9000DAE0FEA3E038
:105E5000FFC39DEE9C4003025F679065FEE090CA21
:105E60004893FD12199A9065FEE090CA489324FE6B
:105E7000602224FE602C24FC603624F8604024F06C
:105E8000604A241F70529069D412EC669000F3129D
:105E9000EC8280449069D812EC669000F312EC8298
:105EA00080369069DC12EC669000F312EC82802858
:105EB0009069E012EC669000F312EC82801A90690F
:105EC000E412EC669000F312EC82800C9069E81208
:105ED000EC669000F312EC82906CDDE0FEA3E0FF34
:105EE000C39000DBE09F9000DAE09E40439000CF3B
:105EF000E0C39464503A7F3F7E007D007C0012EC4A
:105F0000CF9000F312EC6612E26212E521AC06AD0E
:105F1000079000CFE025E0FFE433FE748C2FF5827C
:105F2000EE342DF583ECF0A3EDF09000CFE004F01B
:105F30009000F312EC6612ECCF9000F712EC6612B0
:105F4000E494500C9000F312EC669000F712EC828F
:105F50009065FFE0FEA3E0FF9000DBE02FF09000F3
:105F6000DAE03EF0025E417F10127A939065FEE027
:105F700090CA489324FE603F24FE606724FC7003AF
:105F800002600124F8700302601F24F070030260B5
:105F90003D241F60030260597F0C7D157B057AA5A7
:105FA00079571204C57B057AA5795D9000F712EC4C
:105FB00066129F070260597F0C7D157B057AA579D3
:105FC000701204C59000F712EC6612ECCF7F447E8D
:105FD0007A7D007C0012E3E57B057AA57977129E35
:105FE000B180767F0C7D157B057AA5798D1204C56D
:105FF0007B057AA579939000F712EC66129F0780D3
:10600000587F0C7D157B057AA579A91204C57B05FF
:106010007AA579B29000F712EC66129F07803A7F5A
:106020000C7D157B057AA579C51204C57B057AA57B
:1060300079CD9000F712EC66129F07801C7F0C7DD3
:10604000157B057AA579E21204C57B057AA579ED61
:106050009000F712EC66129F077F0C7D221204BBA2
:106060009065FEE090CA489324FE602524FE6040BF
:1060700024FC604D24F8605A24F06067241F70727D
:106080007B057AA679029069D412EC66129F07808C
:10609000619069D812EC6612ECCF7F447E7A7D0065
:1060A0007C0012E3E57B057AA67912129EB180424C
:1060B0007B057AA679239069DC12EC66129F078033
:0760C000317B057AA6793659
:1060C7009069E012EC66129F0780207B057AA6791B
:1060D700449069E412EC66129F07800F7B057AA64D
:1060E70079569069E812EC66129F077F0C7D2F1294
:1060F70004BB7B057AA679689065FFE0FCA3E0FD09
:10610700129ECF7F017B027A0179C87567821205DB
:10611700507D151204BB7F0C7D1E7B8012000C1274
:106127009366E55424FA70030263711470030265E1
:10613700131470030268051470030268DE240460F8
:1061470003026E027F0112023F7F7FE4FD7B7F1215
:10615700002E7F057D2A7B7212002EE55660677F31
:10616700057D707B7912000C7F3F7B7212002E7FBA
:10617700797D7012002E901A6DE090CA439324FE29
:1061870060161460132402701E7F057D207B057A3C
:10619700A679771204C580217F057D207B057AA625
:1061A70079821204C58012E4901A6DF07F057D2074
:1061B7007B057AA6798F1204C57F617D207B057ADE
:1061C700A679991204C59065E6E0FEA3E0FFD39493
:1061D70000EE9400401AEF24FFFFEE34FFFE7C0030
:1061E7007D3A12E9DF901DF6E02FFFEC3EFE8004BA
:1061F7007E007F009000DAEEF0A3EFF0AC06FD7BA7
:10620700057AA6799F129ECF7F057D751204BB7B09
:10621700057AA679A49000DBE0241DFD9000DAE062
:106227003400FC129ECF7F027B027A0179C8756722
:106237003F1205507D751204BB7B057AA679AB909A
:1062470000DBE0243AFD9000DAE03400FC129ECF38
:106257007F017B027A0179C875677B1205507D75CE
:106267001204BB901A6DE09000D5F0D3940240035E
:106277007402F09000D5E0FF7E007C007D7412E987
:10628700DF74B32FF974133EFA9000DE7402F0A3A3
:10629700EAF0A3E9F09000D5E025E0248CF582E44C
:1062A7003466F583E0FFA3E09000E1CFF0A3EFF0C1
:1062B700D3906CE0E09401906CDFE094005003020F
:1062C7006E02D39000E2E094009000E1E094005069
:1062D7000302636B9000D37406F0D39065E7E094F4
:1062E700009065E6E094004007901DF6E0FF80020D
:1062F7007F009000D0EFF0E49000CEF09000CEE069
:10630700FFC3943A505E9000D0E0FEEF2E75F03A4E
:1063170084E5F025E0FFE433FE9000DEE0FBA3E038
:10632700FAA3E0F98F828E8312EA72FFAEF0900033
:10633700E1E0FCA3E0FD12E9F3C374709FFF900056
:10634700D2F0FDA3E0FF04F07B6F12002E9000D384
:10635700E0FF04F09000D2E0FD12002E9000CEE0A6
:1063670004F08098129366026E027F0112023F7F4B
:106377007FE4FD7B7F12002E7F057D2A7B72120052
:106387002EE55660317F057D707B7712000C7F3ECE
:106397007B7212002E7F777D7012002E7F057D7530
:1063A7007B057AA679B01204C57F627D207B057ACA
:1063B700A679B31204C59013A5E0C3946C50047F6B
:1063C7000180027F029000D4EFF06401701C7F33DC
:1063D7007D757B057AA679BA1204C57F6B7D757BBF
:1063E700057AA679C11204C5801A7F347D757B05AD
:0F63F7007AA679C61204C57F697D757B057AA6E3
:1064060079CD1204C5129366906992E07003026E0C
:10641600099013A5E0D394005003026E02902D81DB
:10642600E0D394005003026E029000D37406F0E4A9
:106436009000CEF09013A5E0FF9000CEE0FEC39F43
:1064460040030264D0EE25E0FFE433FE902F31E0F6
:10645600FD75F090A4246EF582E5F0341AF583ED0F
:106466002583F583E5822FF582EE3583F583E0FEFD
:10647600A3E0FF902D81E0FD7C0012E9F3C3746E6A
:106486009FFF9000D2F0FDA3E0FF1204799000D3A5
:10649600E004FF9000D2E0FD1204799000D3E0FF03
:1064A6009000D2E004FD1204799000D3E004FF903E
:1064B60000D2E004FD1204799000D3E004F0A3E0DA
:1064C600FF9000CEE02FF002643A1293669065EDDD
:1064D60012EC66EC12E4E512ECCF7F447E807D0080
:1064E6007C0012E3E512ECCF7F3F7E007D007C004E
:1064F60012E26212E521AC06AD077B057AA679D2D7
:10650600129ECF7F057D201204BB026E027F02120F
:10651600023FE4FF7D1E7B057AA679E61204C5E4F8
:10652600FF7D4B7B057AA779081204C57F2A7D7803
:106536007B057AA7792F1204C57F117D4D7B6B12DF
:10654600000C7F3E7D207B7A12002E906992E070CF
:1065560003026E099013A5E0C3941E50030267FF61
:10656600E0C394C740030267FF7F437E347D007C0F
:106576000012ECCF907BE7E0FCE412E4ED12E3E5D9
:106586009000EF12EC82902D84E06010E4F0900011
:10659600E712EC669000E312EC8280CDE49000CE28
:1065A600F09013A5E014FF9000CEE0C39F400302D5
:1065B600677A9000CEE0FF70169000E312EC8E0032
:1065C6000000009000E712EC8E000000008075903D
:1065D6007BE7E06F704A7F437E34FDFC12ECCF9080
:1065E6007BE7E0FF9013A5E0C39FFCE412E4ED1205
:1065F600E3E59000EF12EC829000E312EC66900067
:10660600E712EC827F437E347D007C0012ECCF9053
:1066160000EF12EC6612E2629000E312EC82802434
:106626009000E312EC669000E712EC829000E31211
:10663600EC6612ECCF9000EF12EC6612E26290006C
:10664600E312EC82902D84E06011E4F09000E712F2
:10665600EC669000E312EC820265B89000CEE0256D
:10666600E0FFE433FE902F31E0FD75F090A4247036
:10667600F582E5F0341AF583ED2583F583E5822F5F
:10668600F582EE3583F583E0FCA3E0FDE412E4E950
:1066960012ECCF902D81E0FCE412E4ED12E3E5125A
:1066A600E5219000D6EEF0A3EFF0902D84E0600493
:1066B600E4F080A79000E312EC6612E5219000DA80
:1066C600EEF0A3EFF0D39467EE94014007E4900058
:1066D600DAF0A3F09000DAE0FAA3E0FB24B1F58249
:1066E600EA3466F583E0FF3395E0FE9000D6E0FCE1
:0D66F600A3E0FD12E9DF7C007D6412EA489C
:10670300EF243D9000D0F074242BF582EA3468F531
:1067130083E0FF3395E0FE9000D6E0FCA3E0FD129A
:10672300E9DF7C007D6412EA48C3744D9F9000D179
:10673300F0902D84E06005E4F00266BA9000D0E0AA
:10674300FFA3E0FD1204799000D0E004FFA3E01260
:1067530004799000D0E0FFA3E004FD1204799000D7
:10676300D0E004FFA3E004FD1204791293669000C5
:10677300CEE004F00265A77F427EC87D007C001254
:10678300ECCF901DCE12EC6612E36D12ECCF7F3F7F
:106793007E007D007C0012E26212E5219000DCEEB7
:1067A300F0A3EFF0D39464EE940050507B057AA7E6
:1067B30079389000DCE0FCA3E0FD129ECF7F087DDA
:1067C300767B027A0179C81205A87B057AA7793E00
:1067D3009000DCE0FEA3E0FFC374649FFDE49EFC35
:1067E300129ECF7F017B027A0179C8756478120605
:1067F300917D767B027A0179C81205A8129366020D
:106803006E027F107D6E7B7412000C7F107D3C7BCB
:106813007012002E7F427D6E12002E7F747D6E12E9
:10682300002EE49000CEF09000CEE0FFC39403501E
:106833003E7B057AA77944EF75F032A4FFAEF09062
:1068430065FFE0FCA3E0FD12E9DFAC06AD07129E95
:10685300CF9000CEE075F030A4240DFF7D737B0252
:106863007A0179C81204C59000CEE004F080B8E440
:106873009000CEF09000CFE0FF9000CEE0FEC39FEB
:106883004003026E02EE25E0FFE433FE748C2FF525
:1068930082EE342DF583E0FEA3E0FFE4FCFD12EC71
:1068A300CF7F307E007D007C0012EAD3EC12E4E55A
:1068B30012ECCF9000F712EC6612E3E512E521C368
:1068C300746E9FFF9000D2F0FDA3E0FF04F07B6D98
:1068D30012002E9000CEE004F080997F0312023F55
:1068E300901DFBE0601A902F20E0FF60137B057A78
:1068F300A77948FD7C00129ECF7FD87D7212059E3A
:10690300129366901A43E0647D6008E0647C600340
:10691300026B01901DFBE0FF7009906C47E0700370
:10692300026A3BEF60437F007E007D007C0012EC37
:10693300CF9069CE12EC6612E4947007FFFC12EC60
:10694300CF8015902D7A12EC6612ECCF906622124E
:10695300EC6612E25E12ECCF9069CE12EC6612E2A4
:10696300629000FF12EC82807090666FE0FCA3E0FF
:10697300FDE412E4E912ECCF7F427EC87D007C0087
:1069830012E3E512ECCF7F427E707D007C0012E3C0
:10699300E512ECCF9069C4E025E0FF9069C3E033D2
:1069A300FE74E52FF582EE3417F583E0FCA3E0FDDA
:1069B300E412E4E912E36D9000EB12EC829017DC31
:1069C30012EC66E412E4E512ECCF9000EB12EC66F5
:1069D30012E2629000FF12EC82906C4C12EC661291
:1069E300ECCF9000FF12EC6612E494400E906C4CD6
:0369F30012EC663D
:1069F6009000FF12EC8280207F007E007D007C00EC
:106A060012ECCF9000FF12EC6612E494500A90004C
:106A1600FF12EC8E00000000907BE312EC6612EC95
:106A2600CF9000FF12EC6612E36D12E5219000D3C1
:106A3600EFF0026AB89065F1E0FCA3E0FDE412E431
:106A4600E912ECCF906C52E0FCA3E0FDE412E4E91D
:106A560012E3E59000FF12EC82906C52E0FEA3E098
:106A6600FFD39065F2E09F9065F1E09E400FEEF057
:106A7600A3EFF0906C66E09000D3F0801D906C66FA
:106A8600E0FCE412E4ED12ECCF9000FF12EC66128B
:106A9600E36D12E5219000D3EFF09000FF12EC6653
:106AA60012ECCF906C4C12EC6612E36D9000FF1264
:106AB600EC8290662212EC669000FB12EC82906CDF
:106AC6004C12EC6612ECCF9000FB12EC6612E494CA
:106AD600400C906C4C12EC669000FB12EC82907BA2
:106AE600E312EC6612ECCF9000FB12EC6612E36D3B
:106AF60012E5219000D2EFF0026BFD901A43E0649C
:106B06007B6008E0647A6003026BFD90662212ECFB
:106B16006612ECCF906C4C12EC6612E494504A90DC
:106B26002F2BE0FF7E007C007D3C12E9DFA3E02FE7
:106B3600FDEC3EFCE412E4E912ECCF90662212EC86
:106B46006612ECCF7F447E7A7D007C0012E3E5126C
:106B5600E36D12E521906C52EEF0A3EFF090662201
:106B660012EC66906C4C12EC8290662212EC6690E7
:106B760000FB12EC8290662212EC6612ECCF906C4F
:106B86004C12EC6612E3E512ECCF906C66E0FCE486
:106B960012E4ED12E36D12E5219000D2EFF090655C
:106BA600F1E0FCA3E0FDE412E4E912ECCF906C52B4
:106BB600E0FCA3E0FDE412E4E912E3E59000FF1235
:106BC600EC82906C66E0FCE412E4ED12ECCF9000EF
:106BD600FF12EC6612E36D12E5219000D3EFF09000
:106BE60000FF12EC6612ECCF906C4C12EC6612E3CE
:106BF6006D9000FF12EC82902D84E06005E4F002B7
:106C060069061293667F3F7E007D007C0012ECCF02
:106C16009000FF12EC6612E26212E521C006C00780
:106C26007F3F7E007D007C0012ECCF9000FB12ECD3
:016C360066F7
:106C370012E26212E521AC06AD07D007D006C3ED1C
:106C47009F9000D9F0EC9E9000D8F0902D84E060E2
:106C570004E4F080AF7F477E7F7DDC7C0012ECCFC1
:106C67009000FB12EC6612E494503A75660575675E
:106C7700A775684D7F3F7E007D007C0012ECCF90AA
:106C870000FB12EC6612E26212E5218E698F6A90B0
:106C970000D8E0FEA3E08E6BF56C7B027A0179C821
:106CA70012EE05802B7566057567A7756859900004
:106CB700FB12EC668F6C8E6B8D6A8C699000D8E046
:106CC700FEA3E08E6DF56E7B027A0179C812EE05A0
:106CD7009000D2E0FED3946E40047F028004EE243D
:106CE70012FF7D687B027A0179C81204C59000D231
:106CF700E0FF7D66240EFB75666E12092B7F477ECB
:106D07007F7DDC7C0012ECCF9000FF12EC6612E472
:106D17009450117B057AA779679000FF12EC6612F1
:106D27009F07800F7B057AA7796C9000FF12EC66AE
:106D3700129EB19000D3E0FED3946E40047F028090
:106D470004EE2412FF7D777B027A0179C81204C50D
:106D57009000D3E02406FF7D757B057AA77973122F
:106D670004C59000D3E0FF7D75240EFB75667D1288
:106D7700092B901DFBE06003026E027F01129F4FFB
:106D87007FD67D687B027A0179C81204C5906C476B
:106D9700E060399069C4E025E0FF9069C3E033FE05
:106DA70074EC2FF582EE3469F583E0FAA3E0FB7CFF
:106DB700007D3CFFAE0212E9F3902F2BEFF07C0031
:106DC7007D3CAF03AE0212E9F3A3EDF075660575DE
:106DD70067A7756875902F2BE0756900F56AA3E0C2
:106DE700756B00F56C7B027A0179C812EE057FD6C8
:106DF7007D767B027A0179C81204C5E555600312D6
:036E0700033F2224
:106E0A008F4DE54DC394285007E4906CE2F080144E
:106E1A00E54DC39428400DE54DC3943C5006906C53
:106E2A00E27401F0129D5E90681FE551F0E54D1283
:106E3A00ED216E85006ECA016F13026F58036F97BA
:106E4A00046F580573750670C60A73990B741D0C86
:106E5A0074360D71371071371174D014759F157609
:106E6A00332876332977042A77D32B77F72C772898
:106E7A002D73513C74B53D000078A07F017B057AE3
:106E8A00A7797F129AF87F027B057AA77989129AE5
:106E9A00F87F037B057AA77991129AF87F047B051C
:106EAA007AA77998129AF8906C4BE064086003020A
:106EBA0078A07F057B057AA7799E129AF80278A0B6
:106ECA007F017B057AA779A6129AF87F027B057A59
:106EDA00A779B3129AF87F037B057AA779BC129A2D
:106EEA00F87F04906C4BE0B408087B057AA779C355
:106EFA0080067B057AA779D4129AF87F057B057AF2
:106F0A00A779DB129AF80278A07F017B057AA77924
:106F1A00E7129AF87F027B057AA779EE129AF87F30
:106F2A00037B057AA779F5129AF87F047B057AA77D
:106F3A0079FC129AF87F057B057AA87904129AF8E7
:106F4A007F067B057AA8790F129AF80278A07F0744
:106F5A001282F17F01129AF87F0D1282F17F0212DA
:106F6A009AF87F131282F17F03129AF87F1912821C
:106F7A00F17F04129AF87F1F1282F17F05129AF8A4
:106F8A007F251282F17F06129AF80278A07F0C7D83
:106F9A00197B057AA8791A1204C57F147D237BE32D
:106FAA0012000CE4900117F0900117E0C394064018
:106FBA00030278A0129366900117E0FE75F00EA402
:106FCA002428A3F0E4FF901A6AE02EFD12801290A2
:106FDA002F21E01460671460030270A475660575BA
:106FEA0067A875682F900117E004756900F56A9023
:106FFA002F26E0756B00F56CA3E0756D00F56EA3A6
:10700A00E0756F00F570A3E0757100F572A3E07585
:10701A007300F574A3E0757500F576A3E075770043
:0B702A00F5787B027A0179C812EE05B0
:107035007F0C900118E0FD7B027A0179C81204C526
:1070450080767566057567A875685F900117E00419
:10705500756900F56A902F2212EC6612E5218F6E94
:107065008E6D8D6C8C6B902F29E0756F00F570A37C
:10707500E0757100F572A3E0757300F574A3E07512
:107085007500F5767B027A0179C812EE057F0C90C2
:107095000118E0FD7B027A0179C81204C5801990B8
:1070A5000117E060030278A57F02FDFB1296CB90E5
:1070B5006694E0901A43F022900117E004F0026F05
:1070C500B27F077D647BE775667812092B7F0F7D9C
:1070D500697B057AA879851205A87B057AA8798D3B
:1070E500901A6AE024F975F00684E5F004FD7C0049
:1070F500129ECF7F6C7D6912059E7F017B057AA864
:107105007992129AF87F027B057AA579A9129AF8E5
:10711500901A6AE024F975F00684E5F0D3940050DE
:10712500030278A07F037B057AA87997129AF80263
:1071350078A0E54D641060030271BC7F0C7D197B5E
:10714500057AA879A81205A87401D39551500FE5C1
:1071550051D3940350087B057AA879B980067B053D
:107165007AA879CF8B668A678968906C5AE07569C9
:1071750000F56AA3E0756B00F56CA3E0756D00F58D
:107185006E7B027A0179C812EE057F8A7D19120598
:107195009EE551D394035016E55175F01AA4FE24CB
:1071A5006BFF7D14EE2481FB75662812092B900177
:1071B500197404F00272437F0C7D197B057AA87956
:1071C500E51205A8E551D3940650087B057AA87900
:1071D500F680067B057AA979088B668A67896890A7
:1071E5006C54E0756900F56AA3E0756B00F56CA356
:1071F500E0756D00F56EA3E0756F00F570A3E075A1
:107205007100F572A3E0757300F5747B027A01795C
:10721500C812EE057F8A7D1912059EE551D39406A5
:107225005016E55175F00BA4FE247BFF7D14EE246A
:1072350088FB75662812092B9001197407F07F0CDD
:107245007D377B057AA979151205A8900119E0FF0C
:10725500D395515011EF04FFE551D39F50087B059D
:107265007AA9792980067B057AA979388B668A6798
:087275008968906C5DE0756909
:10727D0000F56AA3E0756B00F56C7B027A0179C8A5
:10728D0012EE057F8A7D3712059E900119E0FFD31E
:10729D0095515021EF04FEE551D39E5018C3E55191
:1072AD009F75F01AA4FE2485FF7D32EE249BFB759D
:1072BD00664612092B7F0C7D557B057AA9794912FB
:1072CD0005A8900119E0FF2402D395515012EF2427
:1072DD0004FFE551D39F50087B057AA979588006A4
:1072ED007B057AA9796D8B668A678968906C5FE0FA
:1072FD00756900F56AA3E0756B00F56C7B027A0188
:10730D0079C812EE057F8A7D5512059E900119E010
:10731D00FF2402FED3955140030278A0EF2403FF12
:10732D00E551D39F40030278A0C3E5519E75F01A35
:10733D00A4FE2485FF7D50EE249BFB756664120927
:10734D002B0278A07F017B057AA97984129AF87FA8
:10735D00027B057AA9798E129AF87F037B057AA9AB
:10736D007993129AF80278A07F017B057AA9799D0D
:10737D00129AF87F027B057AA979A4129AF87F03F5
:10738D007B057AA979A7129AF80278A07F017B056F
:10739D007AA979B2129AF87F027B057AA979BD1282
:1073AD009AF87F037B057AA979D1129AF89069B979
:1073BD00E025E0244FF582E434CAF583740193701F
:1073CD000193700D7B057AA979DDFDFC129ECF80AE
:1073DD001F7B057AA979E29069B9E025E0244FF584
:1073ED0082E434CAF583E493FC740193FD129ECFBD
:1073FD007F017B027A0179C87564EF120691EF2443
:10740D00F6FF7D3B7B027A0179C81205A80278A0B0
:10741D007F017B057AA979EE129AF87F027B057AB6
:10742D00A979FD129AF80278A0E4900117F0900165
:10743D0017E0FFC394065065EF25E02457F582E46D
:10744D00347CF583E0FEA3E0FF4E60517566057553
:10745D0067AA756803900117E08E698F6A248BF512
:10746D0082E4347CF583E070087B057AAA790C8080
:10747D00067B057AAA79168B6B8A6C896D7B027AED
:10748D0001790312EE05900117E004FF7B027A01EA
:10749D007903129AF8900117E004F080919001178A
:1074AD00E0902F30F00278A07B057AAA791D9065C7
:1074BD00FFE0FCA3E0FD129ECF7F0C7D1912059E0F
:1074CD000278A07B057AAA792D7F407E137D337CCF
:0F74DD0033129EB17F0C7D141204BB7B057AAA7B
:1074EC0079479013AF12EC66129EE97F0C7D1F1248
:1074FC0004BB901A44E0D3940040117B057AAA791E
:10750C005990669512EC66129EE9800C7B057AAA5E
:10751C00796BE4FDFC129ECF7F0C7D2A1204BB120A
:10752C009B3F8B698A6A896B7566057567AA756856
:10753C00877B027A0179C812EE057F0C7D35120427
:10754C00BB7F0C7D407BE612000C7B057AAA7996FA
:10755C009003A1E0FD7C00129ECF7F0C7D451204B0
:10756C00BB129BE2AC06AD077B057AAA79A8129EEA
:10757C00CF7F0C7D501204BB7B057AAA79BE906537
:10758C00FFE0FCA3E0FD129ECF7F0C7D5B1204BBE1
:10759C000278A07B057AAA79D090660B12EC661261
:1075AC009EB17F0C7D141204BB7B057AAA79E59001
:1075BC00660712EC66129EB190CA10E493FF7D1F11
:1075CC001204BB7B057AAA79F290660312EC661260
:1075DC009EB190CA10E493FF7D2A1204BB7B057AFE
:1075EC00AA79FF9002D1E0FD7C00129ECF7F0C7D2A
:1075FC00351204BB7F0C7D407BE612000C9065F4C9
:10760C0012EC6612ECCF7F107E0E7D007C0012F522
:10761C001C12ECEE7B057AAB7916129EE97F0C7D81
:10762C00451204BB0278A0E54D6428706B7F027B89
:10763C00057AAB7924129AF8E4901DF7F0906C451A
:10764C00E07009FFFEFDFC12ECCF8031906C7AE00B
:10765C002400FD906C79E034C0FCE412E4E912ECF7
:10766C00CF7F477E407D007C0012E3E512ECCF7F9C
:10767C00427EC87D007C0012E36D12ECCF7F427E0F
:10768C00C87D007C0012E25E7B057AAB7931129EDC
:10769C00B17F117D661204BB7F017B057AAB7952F9
:1076AC00129AF8E4901DF7F0906999E07003027853
:1076BC00A07F077D437BE775667712092B7F117DD1
:1076CC004A7B057AAB795C1204C57F117D547BDD56
:1076DC0012000C7566057567AB7568647569027583
:1076EC006A69756B997B027A0179C812EE057F1174
:1076FC007D591204BB0278A07F017B057AAB795CC3
:10770C00129AF87F027B057AA77991129AF87F0377
:10771C007B057AAB7975129AF80278A075660575B7
:05772C0067AB75687FEA
:10773100756902756A69756B997B027A0179C8125C
:10774100EE057F0C7D221204BB906C45E07009FFB1
:10775100FEFDFC12ECCF8031906C7AE02400FD90AC
:107761006C79E034C0FCE412E4E912ECCF7F477E8F
:10777100407D007C0012E3E512ECCF7F427EC87DA4
:10778100007C0012E36D12ECCF7F427EC87D007C4D
:107791000012E25E7B057AAB7991129EB17F0C7D7E
:1077A1002F1204BB7480FF7E017B027A6C794575D0
:1077B1006000756101120A677B057AAB79B3906C41
:1077C10045E0FD7C00129ECF7F0C7D3C1204BB0284
:1077D10078A07F017B057AAB79CE129AF87F027B84
:1077E100057AAB79DD129AF87F037B057AAB79F3E1
:1077F100129AF80278A07F0C7D197B057AAB79FE8D
:107801001205A8901A69E0C3940A5071E490011717
:10781100F0900117E02499F582E43469F583E0FFE3
:1078210060047E0180027E00EE6038756605756732
:10783100AC75680A8F697B027A0179C812EE057FFF
:10784100027B027A0179C8900117E075F00CA4243B
:1078510070F5641206917D1912059E900117E004DE
:10786100F080AE901A69E075F00CA4FE2468FF7DEB
:1078710014EE2477FB75662812092B8022756605A4
:107881007567AC75680D756902756A69756B997B69
:10789100027A0179C812EE057F6C7D1912059EE40A
:0578A100901DF7F0222C
:1078A6008B4D8A4E894F8D507B057AAC7910129D8F
:1078B6005E7F02AB4DAA4EA94F7564771206917D85
:1078C6002DAB4DAA4EA94F1205A87F187D557B6397
:1078D60075666E12092B7F237D5D7B057AAC791761
:1078E6001205A8E55060197F8B7D557BD675666EAF
:1078F60012092B7F9C7D5D7B057AAC791E1205A84B
:0479060012033F2207
:10790A00906CE2E060727480FF7E017B027A6C798F
:10791A0045756000756101120A67902F2FE075F0B6
:10792A0040A42400FFE5F03414FE7B027A6C7977D8
:10793A00756000756140120A67906C77E0FAA3E0FF
:10794A00FB2428FFE43AFEC3906C7AE09FFF906C18
:10795A0079E09EFE7C007D0A12E9F39066AEEEF0B5
:10796A00A3EFF0AF03AE027B027A1D798E75600039
:10797A00756128120A678057902F2FE0FF7E007CDE
:10798A00007D6312E9DF74022FF9741E3EFA7B024E
:10799A00C00378777C6CAD03D0037E007F6312E965
:1079AA004F906C94E0FEA3E0FFC3906C9BE09F9025
:1079BA0066AFF0906C9AE09E9066AEF0788E7C1D71
:1079CA007D027B027A6C79B27E007F2812E94F90A1
:1079DA006C7C12EC6612ECCF7F407E7E7D057C00CB
:1079EA0012EB3512ECEE906C46EFF0906C7C12ECD8
:1079FA006612ECCF7F407E7E7D057C0012EB35124D
:107A0A00ECF612ECCF7F707E177D007C0012EB350E
:107A1A0012ECEE906C44EFF0906C7C12EC6612EC77
:107A2A00CF7F707E177D007C0012EB3512ECF612C8
:107A3A00ECCF7F647E007D007C0012EB3512ECEE09
:107A4A00906C48EFF0906C7C12EC6612ECCF7F647D
:107A5A007E007D007C0012EB3512ECF6906C6AEF2A
:107A6A00F09065FFE0FEA3E08E58F5599065FF742B
:107A7A000BF0A374B8F0E4FFFE7DFF12199A90652B
:097A8A00FFE558F0A3E559F022D4
:107A93008F57E55720E10620E203027BC1E557300B
:107AA300E1087B057AAC792480067B057AAC793CC6
:107AB300129D5EC2AF12790A7566057567AC75686B
:107AC30054902F2FE004756900F56A906CE2E06032
:107AD30009906C45E0FF7E0080079003A1E0FF7EE4
:107AE300008E6B8F6C7B027A0179C812EE057F0CD6
:107AF3007D1912059E7566057567AC756867906C90
:107B030083E0756900F56AA3E0756B00F56CA3E08B
:107B1300756D00F56E7B027A0179C812EE057F0C54
:107B23007D3712059E7566057567AC756880906C28
:107B330082E0756900F56A906C81E0756B00F56C05
:107B4300906C80E0756D00F56E7B027A0179C81246
:107B5300EE057F0C7D4612059E7566057567AC754F
:107B63006897906C46E0756900F56A906C44E0751F
:107B73006B00F56C906C48E0756D00F56E906C6A67
:107B8300E0756F00F5707B027A0179C812EE057F0C
:107B93000C7D5512059E906C9CE07006906C7BE00A
:107BA300601A7F0C7D677B057AAC79B51204C57FBB
:107BB3000C7D717B057AAC79D51204C5D2AFE5573C
:107BC30030E5237B057AA57950129D5E7F357D2DA7
:107BD3007B057AAC79FB1205A87F177D3C7B057A80
:107BE300AD790F1205A8E55720E303027E4990689B
:107BF30020E060087B057AA5795080067B057AA38F
:107C03007904129D5E906820E07019906C9CE0707E
:107C130006906C7BE0600D7F327D027B057AAD7947
:107C23002B1204C5C2AF906CDDE0FCA3E0FDE412AF
:107C3300E4E912ECCF7F427E707D007C0012E36D9D
:107C430012ECCF90668812EC6612E26212ECCF7FE0
:107C5300427EC87D007C0012E36D12ECCF7F3F7E35
:107C6300007D007C0012E26212E52190012212ECF9
:107C73008290012212EC6612ECCF7F407E7E7D055E
:107C83007C0012EB3512ECEE90011CEFF090012218
:107C930012EC6612ECCF7F407E7E7D057C0012EBFA
:107CA3003512ECF612ECCF7F707E177D007C00124C
:057CB300EB3512ECEEC0
:107CB80090011DEFF090012212EC6612ECCF7F705C
:107CC8007E177D007C0012EB3512ECF612ECCF7FAC
:107CD800647E007D007C0012EB3512ECEE90011EF4
:107CE800EFF090012212EC6612ECCF7F647E007DEB
:107CF800007C0012EB3512ECF690011FEFF0756670
:107D0800057567AD756840906CDDE0FAA3E0FB7C13
:107D1800007D3CFFAE0212E9F38E698F6A7C007D1C
:107D28003CAF03AE0212E9F38C6B8D6C90011CE042
:107D3800756D00F56EA3E0756F00F570A3E07571C1
:107D480000F572A3E0757300F5747B027A0179C8B7
:107D580012EE057F0C7D157B027A0179C81204C5E5
:107D68007F0C7D1E7B8012000C7B057AA6796890BB
:107D780065FFE0FCA3E0FD129ECF7F017B027A0144
:107D880079C87567821205507D201204BB7B057A7D
:107D9800AD79669069D412EC66129F077F0C7D2F2F
:107DA8001204BB9069D812EC6612ECCF7F447E7A3D
:107DB8007D007C0012E3E57B057AAD7978129EB1EF
:107DC8007F0C7D3C1204BB7B057AAD798A9069DC17
:107DD80012EC66129EB17F0C7D491204BB7F007EB7
:107DE800007D007C0012ECCF9069E012EC6612E492
:107DF80094500A9069E012EC8E000000007B057A2E
:107E0800AD79A19069E012EC66129EB17F0C7D56A7
:107E18001204BB7B057AAD79B49069E412EC661262
:107E28009F077F0C7D631204BB7B057AAD79C690F2
:107E380069E812EC66129F077F0C7D701204BBD2B2
:107E4800AFE55720E403028011C2AF12790A7B051F
:107E58007AAD79D7902F2FE02401FDE433FC129EF0
:107E6800CF7F8A7D151204BB7F8A7D1E7BE51200B9
:107E78000C7F857D0F7BEA75667A12092B7566057E
:107E88007567AD7568EA906C46E0756900F56A90AB
:107E98006C44E0756B00F56C906C48E0756D00F50E
:107EA8006E906C6AE0756F00F5707B027A0179C894
:107EB80012EE057F8A7D221204BB906CDBE0600322
:107EC800027FBF7B057AAE790C9069D412EC6612FA
:107ED8009F077F8A7D2F1204BB7B057AAE7922909B
:0F7EE8001DA612EC66129F077F8A7D3C1204BB19
:107EF7007F427EC87D007C0012ECCF901DAE12EC55
:107F07006612E36D12ECCF901DB212EC66E412E438
:107F1700E512E3E512ECCF7F3F7E007D007C001287
:107F2700E26212E521900120EEF0A3EFF0756605FD
:107F37007567AE7568388E69F56AC374649FF56CAA
:107F4700E49EF56B7B027A0179C812EE057F8A7D84
:107F5700491204BB7B057AAE79519069E412EC664D
:107F6700129F077F8A7D561204BB7B057AAE79671D
:107F7700901DAA12EC66129F077F8A7D631204BBCD
:107F87007F007E007D007C0012ECCF9069E012EC50
:107F97006612E494500A9069E012EC8E000000002B
:107FA7007B057AAE797E9069E012EC66129EB17F0E
:107FB7008A7D701204BB80509069D812EC6612EC6F
:107FC700CF7F447E7A7D007C0012E3E57B057AAEA5
:107FD7007995129EB17F8A7D2F1204BB7B057AAEFD
:107FE70079AB9069DC12EC66129EB17F8A7D3C12F8
:107FF70004BB7B057AAE79C69069E812EC66129FDE
:0B800700077F8A7D491204BBD2AF2224
:108012008F538D54906C4BE064087058E554D394A0
:10802200064051E55424F9FD75F0068475F080A4EC
:108032002400FBE5F03404FAED75F00684E5F075F2
:10804200F010A4AEF02BF556EE3AF555E553701349
:10805200AF56AE557B027A2F7921F56075610C120D
:108062000A6722AF56AE557B027A2F7921755C0CD6
:10807200120B8922E5537025AF54FEFC7D0C12E9E8
:10808200DF74D82FF974153EFA7B02C00378217C85
:108092002FAD03D0037E007F0C12E94F22AF547E36
:1080A200007C007D0C12E9DF74D82FF974153EA80C
:1080B20001FC7D027B027A2F79217E007F0C12E97E
:0280C2004F224B
:1080C400ED70030281A8902F21EFF0906C55E0FF32
:1080D400E4FCFDFE12ECCF7F107E277D007C0012B5
:1080E400EAD312ECCF906C54E0FFE4FCFDFE12ECFA
:1080F400CF7FA07E867D017C0012EAD312EAAC1207
:10810400ECCF906C56E0FFE4FCFDFE12ECCF7FE870
:108114007E037D007C0012EAD312EAAC12ECCF900D
:108124006C57E0FFE4FCFDFE12ECCF7F647E007D23
:10813400007C0012EAD312EAAC12ECCF906C58E047
:10814400FFE4FCFDFE12ECCF7F0A7E007D007C0084
:1081540012EAD312EAAC12ECCF906C59E0FFE4FCC3
:10816400FDFE12EAACEC12E4E5902F2212EC8278C8
:10817400267C2F7D027B027A6C795A7E007F07125F
:10818400E94F7F01901A6AE0FD128012901A6AE0AA
:1081940024F975F00684E5F0B405037F0B22901AE8
:1081A4006AE004F0E4FF901A6AE0FD128012902F56
:1081B4002212EC6612ECCF7F477EC37D507C001206
:1081C400E3E512E521906C54EFF0902F2212EC6657
:1081D40012E52112ECCF7FA07E867D017C0012EB9C
:1081E4003512ECF68F4D8E4C8D4B8C4A12ECCF7FB2
:1081F400107E277D007C0012EB3512ECEE906C555E
:10820400EFF0AF4DAE4CAD4BAC4A12ECCF7F107ECD
:10821400277D007C0012EB3512ECF68F4D8E4C8DD1
:108224004B8C4A12ECCF7FE87E037D007C0012EB7E
:108234003512ECEE906C56EFF0AF4DAE4CAD4BAC4E
:108244004A12ECCF7FE87E037D007C0012EB3512EE
:10825400ECF68F4D8E4C8D4B8C4A12ECCF7F647EA6
:10826400007D007C0012EB3512ECEE906C57EFF0C1
:10827400AF4DAE4CAD4BAC4A12ECCF7F647E007D6B
:10828400007C0012EB3512ECF68F4D8E4C8D4B8C2E
:108294004A12ECCF7F0A7E007D007C0012EB35127F
:1082A400ECEE906C58EFF0AF4DAE4CAD4BAC4A12C7
:1082B400ECCF7F0A7E007D007C0012EB3512ECF6D9
:1082C4008F4D8E4C8D4B8C4A906C59EFF0785A7CC4
:1082D4006C7D027B027A2F79267E007F0712E94F9C
:0D82E400902F21E0B401037F20227F1F2294
:1082F1008F527E007F407D007B027A01792712ED4B
:1083010047E4900126F0900126E0FEC39406400365
:108311000283C1E4FFE5522EFD128012902F21E06D
:1083210070030283C17B027A01792712F57EC3EFC4
:108331009420EE6480948040030283B878677C01C6
:108341007D027B027A0179277E007F2012E94F901E
:108351002F21E0640270347566057567AE7568DBC0
:10836100756902756A01756B67902F26E0756C005F
:10837100F56DA3E0756E00F56FA3E0757000F57102
:108381007B027A01792712EE05802C7566057567E7
:10839100AE7568EF756902756A01756B67902F227A
:1083A10012EC6612E5218F6F8E6E8D6D8C6C7B02E7
:1083B1007A01792712EE05900126E004F002830785
:1083C100900126E070147566057567AE7568F97BD6
:1083D100027A01796712EE0580247566057567AF2B
:1083E100756800900126E0756900F56A756B027584
:1083F1006C01756D277B027A01796712EE057B02AC
:108401007A01796712F57ED3EF941EEE6480948031
:10841100401378857C017D027B057AAF79077E0068
:0C8421007F0412E94F7B027A0179672288
:10842D008F4AE4901DFBF09066ACF0906C47F09095
:10843D00039EF0ED24FE6010047028901DFB740166
:10844D00F0E4906C71F0801B906C477401F0E49037
:10845D006C71F09069C3F0A3F09017DC12EC8E00F4
:10846D00000000E54A6406602CAF4A9065F3EFF01A
:10847D009013A3EFF0906C4BE0B408137430FF7EB3
:10848D00017B047A00794A755C01120B8980069094
:0D849D006C69E54AF0AF4AE4FD1284AA22A2
:1084AA008F4B8D4C906C6112EC8E00000000E54BF6
:1084BA00F4704A123A8C7E007F047D007B027A694E
:1084CA00799512ED477E007F047D007B027A6679FA
:1084DA009C12ED47902D807401F09065ECF0E490C9
:1084EA006820F0906C71E06008E064016003028A21
:1084FA00FD906C717402F0E49069AEF022E4FFAD75
:10850A004B12801290039EE0703C906C47E060032F
:10851A0002859D901DFBE0600302859D9065F3E056
:10852A00600AE0FFC3E54B9F6406601A9065F3E0BA
:10853A00C39406500BE0FFE54BB5070AE54C7006FD
:10854A00902F21E0704D123A8CE4906820F0907BD5
:10855A00E8F090667CF09003A004F07F0C9065F33D
:10856A00E0C3940650047D01800B9065F3E0FEC3DE
:10857A00E54B9EFEFDE4FB1296CBE4906C47F0902F
:10858A00039EF09002D2E07006901A437402F01231
:10859A00350522E54BC394065011906C71E0C394E3
:1085AA000250087402F0E49069AEF0906821E0701D
:1085BA0009901A44E07003028AF0E54C70030286BF
:1085CA00A1E490667CF09065F1F0A3F0906995F0D3
:1085DA0090669CF0902F29E0FF906996F090669D36
:1085EA00F0902F2AE0FE906997F090669EF0E4A33F
:1085FA00F0902D80F090682004F0E490681DF090CF
:10860A007BE804F0EF7007EE70047F0180027F00C0
:10861A009001A9EFF0E4FFE54B04FD12801290658A
:10862A00F3E0600DE54B04FFE0FEC3EF9E640660D5
:10863A0006902F21E070257E007F047D007B027A60
:10864A0066799C12ED4790667C7401F09002D2E044
:10865A006003028AFD901A437402F0229001A9E095
:10866A00600790667C7401F0227F08E4FDFB129695
:10867A00CB9002D2E0700B901A437483F07F2012E1
:10868A007A9390667C7401F01235057F04E4FD7BD1
:10869A0001128EEA028AF8902F21E0FF6402600834
:1086AA00EF64016003028AF8E4906C71F09069AE9D
:1086BA0004F06F60030289BB901DFBE0600F9069B4
:1086CA00B312EC66906C4C12EC82028970906C4783
:1086DA00E070030288F8906C4BE0B4082C906C7838
:1086EA00E02428FF906C77E03400FEC3906C7AE0B7
:1086FA009FFF906C79E09EFE7C007D0A12E9F39060
:10870A006C49EEF0A3EFF0801B906C94E0FEA3E0BE
:10871A00FFC3906C9BE09F906C4AF0906C9AE09E2D
:10872A00906C49F07E027F587D007B027A1779E5CA
:10873A0012ED477E027F587D007B027A6979EC123E
:10874A00ED47E49001A7F0A3F0906C49E0FCA3E0A8
:10875A00FD9001A7E0FEA3E0FFC39DEE9C4003024B
:10876A0088E0906C4BE0B4082B7C007D0A12E9DFAC
:10877A00906C78E02428FD906C77E03400CD2FFFD0
:10878A00ED3EFE7B027A66797E75600075610A129B
:10879A000A6780369001A7E0FEA3E0FF906C95E09F
:1087AA002FFF906C94E03EFE7C007D0A12E9DF7494
:0F87BA00332FF9742F3EFA7B02C003787E7C6662
:1087C900AD03D0037E007F0A12E94F906C4AE02482
:1087D900FFFF906C49E034FFFE9001A7E0FCA3E0A5
:1087E900FD6F7002EE6C70507F457EBB7D80FC1280
:1087F900ECCF90667EE0FCA3E0FDE412E4E912E32D
:10880900E512ECCF906682E0FCA3E0FDE412E4E916
:1088190012E36D12E521AC06AD079001A8E025E051
:10882900FF9001A7E033FE74E52FF582EE3417F5CA
:1088390083ECF0A3EDF0803D906682E0FCA3E0FDBF
:10884900E412E4E912ECCF7F417E207D007C001226
:10885900E3E512E521AC06AD079001A8E025E0FFAC
:108869009001A7E033FE74E52FF582EE3417F58306
:10887900ECF0A3EDF07F477E6A7D607C0012ECCFBF
:108889009001A8E025E0FF9001A7E033FE74E52FF1
:10889900F582EE3417F583E0FCA3E0FDE412E4E988
:1088A90012E3E512E521AC06AD079001A8E025E049
:1088B900FF9001A7E033FE74EC2FF582EE3469F5E1
:1088C90083ECF0A3EDF09001A8E004F070069001AC
:1088D900A7E004F00287539069E012EC66906C4CB3
:1088E90012EC82E4906C71F09069AE04F08078909B
:1088F9002F2212EC66906C4C12EC82902F2BE0FF29
:108909007E007C007D3C12E9DFA3E02FFDEC3EFCFC
:10891900E412E4E912ECCF906C4C12EC6612ECCF45
:108929007F447E7A7D007C0012E3E512E36D12E557
:1089390021906C52EEF0A3EFF0FDAC06E412E4E9ED
:1089490012ECCF7F007E007D007C0012E494700D54
:10895900906C717402F0E49069AEF0800AE4906C56
:1089690071F09069AE04F0906C4C12EC6612E5213E
:10897900906C6112EC82E49065F1F0A3F0FE7F0443
:10898900FD7B027A69799512ED477E007F047D00AF
:108999007B027A66799C12ED47902D807401F090E4
:1089A90065ECF09066AB7403F0901A43747CF002A6
:1089B9008AA2902F27E0FF7E007C007D3C12E9DF30
:1089C900AA06AB07902F26E0FF7E007C0E7D1012D1
:1089D900E9DFEF2BFFEE3AFE902F28E07C002FFF16
:1089E900EC3EFE906C50F0A3EFF0FDAC06E412E40F
:1089F900E912ECCF902F2BE0FF7E007C007D3C122A
:108A0900E9DFA3E02FFDEC3EFCE412E4E912E3E523
:108A190012ECCF7F447E7A7D007C0012E36D906C6E
:108A29004C12EC82906C50E0FCA3E0FDE412E4E906
:108A390012E521906C52EEF0A3EFF0E49065F1F0AD
:108A4900A3F0902F26E0906995F090669CF0902F06
:108A590027E0906996F090669DF0902F28E0906944
:108A690097F090669EF0E4A3F0902D80F09065EC6D
:108A790004F0901A43747AF0902F2BE07011A3E060
:108A8900700D906C717402F0E49069AEF0800AE4A4
:108A9900906C71F09069AE04F0123A8C901DFBE075
:108AA90070257F099065F3E0FEC3E54B9EFDE54B1C
:108AB900C3940650047B00800B9065F3E0FEC3E588
:108AC9004B9EFEFB1296CBE4906820F07F01124585
:108AD90068907BE87401F0E490681DF07F057D01E2
:108AE9007B01128EEA80087F04E4FDFB1296CBE439
:058AF9009066ACF022C4
:108AFE008F528D5378167C667D027B027A1D798E9D
:108B0E007E007F6612E94F901A43E0647D6005E0B7
:108B1E00647C704B90662212EC6612ECCF906C4C1B
:108B2E0012EC6612E494500C906C6112EC8E000004
:108B3E000000804890662212EC6612ECCF906C4CCE
:108B4E0012EC6612E25E12ECCF7F3F7E007D007C5F
:108B5E000012E26212E521906C6112EC82801D7FA0
:108B6E003F7E007D007C0012ECCF90662212EC66F8
:108B7E0012E26212E521906C6112EC82902D84E07B
:108B8E006004E4F080817B057AA5793E90664212FE
:108B9E00EC66129F077FA1E4FD1206EB9066ABE038
:108BAE0090CA349324FE6049147003028C521470E0
:108BBE0003028C5224FC4003028D3F240860030202
:108BCE008D4F7B057AA5793A90664A12EC66129F14
:108BDE00077F337D201207687B057AA5793A906668
:108BEE001612EC66129F077F1E7D4B1206EB028D4E
:108BFE004F7B057AA5793A90664612EC66129F076E
:108C0E007F337D2012076890661A12EC6612ECCF45
:108C1E007F447E7A7D007C0012E3E59001AC12EC7D
:108C2E0082902D84E06004E4F080DC7B057AAF79DD
:108C3E000B9001AC12EC66129F077F0D7D4B120656
:108C4E00EB028D4F9066ABE090CA34936403704D87
:108C5E0090664E12EC6612E521AC06AD077B057AE6
:108C6E00A57947129ECF7F447D201207687F417EF3
:108C7E00207D007C0012ECCF90664E12EC6612E363
:108C8E006D12E5217C007D0A12E9F37B057AA57948
:108C9E0042129ECF7F797D20120768800CE4FF126E
:108CAE009F4F7F397D201207687FA07E867D017CD5
:108CBE000012ECCF906C6112EC6612EBDC404D9022
:108CCE006C6112EC6612ECCF7FA07E867D017C007B
:108CDE0012EB3512ECEEAD07AC067B057AAF790FD1
:108CEE00129ECF7F057D4B12059E906C6112EC6635
:108CFE0012ECCF7FA07E867D017C0012EB3512EC4C
:108D0E00F67B057AAF7912129EE9801C7F057D4BAA
:108D1E007B057AA579361205A87B057AAF7918906E
:108D2E006C6112EC66129EE97F0D7D4B1206EB8094
:108D3E00109066ABE090CA3493FFAD52AB53125B0A
:108D4E00899066ABE090CA3493D394044003028EAC
:108D5E00E9906C71E0D3940040097F7F7D657B7F45
:0A8D6E0012002E906C71E090CA3DD7
:108D78009324FE6023147003028E1F147003028E66
:108D88004C147003028E4C24046003028EE97F09A0
:108D9800E4FD7B01125B89227B057AA5793A90660E
:108DA8002E12EC66129F077F1E7D691206EB906CEF
:108DB80047E060399069C4E025E0FF9069C3E0337B
:108DC800FE74EC2FF582EE3469F583E0FAA3E0FB3C
:108DD8007C007D3CFFAE0212E9F3902F2BEFF07C74
:108DE800007D3CAF03AE0212E9F3A3EDF075660512
:108DF8007567A7756875902F2BE0756900F56AA3EC
:108E0800E0756B00F56C7B027A0179C812EE057F7C
:108E1800887D691206EB227B057AA5793A90662E41
:108E280012EC66129F077F1E7D691206EB7B057A9E
:108E3800A5793E90663212EC66129F077FA17D6984
:108E48001206EB227F417E207D007C0012ECCF9041
:108E5800661E12EC6612E36D12E5217C007D0A1293
:108E6800E9F37B057AA57942129ECF7F467D691288
:108E780006EB90661E12EC6612E521AC06AD077B88
:108E8800057AA57947129ECF7F257D691206EB905A
:108E98006C71E090CA3D93B404117B057AA5793EC4
:108EA80090662612EC66129F07802F7F007E007D59
:108EB800007C0012ECCF90662A12EC6612E49460F3
:108EC8000A40087B057AA5793E80067B057AA57954
:108ED8003690662A12EC66129F077FA17D691206FA
:028EE800EB227B
:108EEA008F4F8D508B51E49001B0F0901A43E0649B
:108EFA00796018E064786013E0647B600EE0647D5A
:108F0A006009E0647C6004E0B47A03D38001C39210
:108F1A0009901A43E064816009E064826004E0B465
:108F2A008303D38001C3920A200906200A03029010
:108F3A006EE54F30E25A7566057567AF75681D9024
:108F4A006995E0756900F56AA3E0756B00F56CA395
:108F5A00E0756D00F56E7B027A0179C812EE059014
:108F6A006820E060187F28E4FD7B027A0179C81244
:108F7A0005A87F017D0C7B6412000C800D7F0DE437
:108F8A00FD7B027A0179C81206F59001B07401F0EE
:108F9A00300948E54F30E143906820E0703D901D6C
:108FAA00FAE0FFD3940040087B057AA5793E800653
:108FBA007B057AA57936EFFD7C00129ECF7FA190C2
:108FCA0066ABE090CA3493D3940450047D4B80027C
:108FDA007D691206EB9001B07401F0300912E54F79
:108FEA0030E00DE4FFAD50128AFE9001B07401F03A
:108FFA009001B0E06007E551600312033F30096455
:10900A00E54F6404705E906820E0705890681DE037
:10901A006052E4FFAD50128AFE901DFAE0FFD3942D
:10902A000040087B057AA5793E80067B057AA579FA
:10903A0036EFFD7C00129ECF7FA19066ABE090CA0E
:10904A003493D3940450047D4B80027D691206EB5D
:10905A00D3906CE0E09402906CDFE094004005E469
:05906A0090681DF022DA
:10906F008F4A8D4BE4FF12CDD3EF7002FF227F01A9
:10907F007D0512D0DE9013A7EFF0640C60037F0024
:10908F0022129366E54A1470030291EF0460030203
:10909F00931C7F017D2312D0DEEF7F00FEC006C040
:1090AF00070F7D2412D0DEEFFDD0E02D9013AEF030
:1090BF00D0E034009013ADF0E49001B1F09001B125
:1090CF00E0C39404400302919C1293669001B1E0B7
:1090DF00FBC374039B75F008A4A3F090669512EC84
:1090EF006612ECCF7F01EB240AFD12D0DEE4FCFD0B
:1090FF00FE9001B2E0FBF812EC1512EAAC90669507
:10910F0012EC8290660312EC6612ECCF7F01900195
:10911F00B1E02414FD12D0DEE4FCFDFE9001B2E0BC
:10912F00FBF812EC1512EAAC90660312EC82906613
:10913F000712EC6612ECCF7F019001B1E02418FD0D
:10914F0012D0DEE4FCFDFE9001B2E0FBF812EC154C
:10915F0012EAAC90660712EC8290660B12EC661264
:10916F00ECCF7F019001B1E0241CFD12D0DEE4FCB6
:10917F00FDFE9001B2E0FBF812EC1512EAAC90661E
:10918F000B12EC829001B1E004F00290CC7F017DD4
:10919F002D12D0DE9002D1EFF0E0FCE412E4ED12DC
:1091AF00ECCF7F407EC97D0F7CDB12E36D12ECCFDD
:1091BF007F447E7A7D007C0012E3E5906C6D12ECAB
:1091CF0082906C6D12EC6612ECCF90CA2F12EC727B
:1091DF00EC12E4E512E3E59069A412EC8202931C11
:1091EF00E54B640270309013ADE0FEA3E0FF7C010D
:1091FF007D0012EA48AB077D237F0112D0499013FF
:10920F00ADE0FEA3E0FF7C017D0012EA48AB057DD7
:10921F00247F0112D049E54B6401600302931C9037
:10922F0001B1F09001B1E0C39404400302931C120A
:10923F0093669001B1E0FEC374039E75F008A4FF1E
:10924F00A3F0FBEE240AFDC00590669512EC66A80C
:10925F000312EC0112ECCF7FFF7E007D007C001229
:10926F00EB7FAB077F01D00512D0499001B1E0240D
:10927F0014FDC00590660312EC669001B2E0FBF896
:10928F0012EC0112ECCF7FFF7E007D007C0012EB11
:10929F007FAB077F01D00512D0499001B1E02418B0
:1092AF00FDC00590660712EC669001B2E0FBF81264
:1092BF00EC0112ECCF7FFF7E007D007C0012EB7F74
:1092CF00AB077F01D00512D0499001B1E0241CFDFE
:1092DF00C00590660B12EC669001B2E0FBF812EC41
:1092EF000112ECCF7FFF7E007D007C0012EB7FAB85
:1092FF00077F01D00512D0497F017D2D9002D1E06B
:10930F00FB12D0499001B1E004F00292327F0122AA
:10931F00E49001B4F0FF12CDD39001B3EFF0C2AFE0
:10932F007F017D0512D0DE9001B4EFF012936690AD
:10933F0001B4E0FF901A44E06F6014E4FFFD129057
:10934F006FE4FFFD12549F9001B4E0901A44F0D2E5
:07935F00AF9001B3E0FF2213
:0793660075A61E75A6E122A9
:10936D00E49001B5F0A3F0C39001B6E09F9001B574
:10937D00E09E5026E49001B7F09001B7E0C3941938
:10938D005008129366E004F080EF9001B6E004F00F
:0B939D0070069001B5E004F080CD22C6
:1093A80053F3F8EF42F343F348E5F330E4FB53F3A8
:1093B800EFAFF5EF75F004A4FFE5F454037C002F3C
:0D93C800FFEC35F0FE9069ACF0A3EFF02251
:1093D500901A43E0647B6006906820E06018906610
:1093E5009CE07012A3E0700EA3E0700A90667CF01A
:1093F5009066AC04F02290669FE004F0C39464503C
:1094050003029479E4F09065EC04F09065F2E004D1
:10941500F070069065F1E004F0902D80E064017035
:109425002990669EE004F0C3943C4048E4F09066C1
:109435009DE004F0C3943C403BE4F090669CE0045E
:10944500F0C3940A402EE4F0802A90669EE014F062
:10945500F47021743BF090669DE014F0F47015747F
:109465003BF090669CE014F0F47009F0A3F0A3F0D3
:1094750090667CF0C3901DE8E09470901DE7E09441
:1094850017406D902D8BE06067E4901DE7F0A3F029
:109495009065EB04F0906C47E06055906C4AE024D1
:1094A500FFFF906C49E034FFFE9069C3E0FAA3E04A
:1094B500FBD39FEA9E50399017DC12EC6612ECCF75
:1094C500EB25E0FFEA33FE74E52FF582EE3417F560
:1094D50083E0FEA3E0FFE4FCFD12EAAC9017DC128A
:1094E500EC829069C4E004F070069069C3E004F072
:0194F5002254
:1094F6009069C6E0FED3940340079066157401F0A8
:1095060022EE1392C3EED394014003D38001C3929B
:10951600C45329E09069C7E04229908001E529F00B
:109526009069C8E044C0FCA3E0F5828C83EFF0901C
:1095360069C9E004F070069069C8E004F0D3906948
:10954600C9E094FF9069C8E0943F4018E4F0A3F0A6
:109556009069C7E004F0E0D3941F4008E4F09069F6
:05956600C6E004F02244
:10956B00EF24E5603F047078120006E4FF12E08CF4
:10957B007F1E7E0012936DE4FF12E08C7F1E7E0037
:10958B0012936D9002D47489F09002D6741AF0780D
:10959B00D77C027D027B027A6679A17F0612E94FA6
:1095AB0012006F2290020DE09066A4F090020EE084
:1095BB009066A5F090020FE09066A6F0900210E086
:1095CB009066A3F0900211E09066A2F0900212E078
:1095DB009066A1F07F0112E08C7F1E7E0012936DCE
:0195EB00225D
:1095EC007F1C7D17E4FB1296157FC87E0012936DCD
:1095FC007F1A12956B7FC87E0012936D7F01129CAF
:09960C00B07FC87E0012936D22AC
:109615001200069002D47485F09002D6EFF0A3ED07
:08962500F0A3EBF012006F222C
:10962D00908002E09001B8F020E20E906C72E06044
:10963D000E9066B07401F08006906C727401F0901B
:10964D008002E0440FF454F0907BEBF07009901A17
:10965D0042E070030296CA907BEBE0F9B4F01490EF
:10966D0066A9E0700E901A6B74F0F09066A9740103
:10967D00F0803A9066A9E07034901A42E0FF69706C
:10968D0024E954F060179069B2E0FE9065E5E0D3EF
:10969D009E400A901A6BE9F0E49065E5F09065E55F
:1096AD00E004F08008E97005901A6BEFF0E970089E
:0E96BD009066A9F09065E5F0901A42E9F0225F
:1096CB008F528D538B5475552775561075570575DD
:1096DB0058A2755905755A05755BA2755C05755DC4
:1096EB0005755EA2755F057B057AAC7910129D5EE0
:1096FB00E55214B41C004003029AA290970DF8286F
:10970B00287302976102976D0297820297970297CF
:10971B00AC0297B80297C40297D00297E502989DC6
:10972B0002989D0298D002990E02992902994A0239
:10973B00995F029AA20299740299970299BF0299B2
:10974B00CB0299DD02993E029A01029A4D029A755B
:10975B00029A80029A997557057558AF75592C0264
:10976B009AA27557057558AF755945755D05755EA8
:10977B00AF755F4D029AA27557057558AF75594570
:10978B00755D05755EAF755F62029AA275570575BB
:10979B0058AF755945755D05755EAF755F79029A62
:1097AB00A27557057558AF75598E029AA275570554
:1097BB007558AF75599C029AA27557057558AF75B8
:1097CB0059AB029AA27557057558AF7559C2755D9D
:1097DB0005755EAF755FCA029AA2906C47E0FF6099
:1097EB00087B057AAF79D780067B057AAF79E98B51
:1097FB00578A5889597B057AAF79FAEF60067C0056
:10980B007D018009E55404FF7E00AC06FD129ECF5E
:10981B007F0F7D537B027A0179C81205A87F077DE4
:10982B004B7BE775667812092B902F21E064027051
:07983B002B7566057567B08F
:1098420075680890669CE0756900F56AA3E0756B1F
:1098520000F56CA3E0756D00F56E7B027A0179C8A4
:1098620012EE0580207F3F7E007D007C0012ECCF4F
:10987200906C4C12EC6612E26212E5217B057AB022
:10988200791F129EE97F0F7D667B027A0179C812E9
:1098920005A875554E755620029AA275570575583A
:1098A200AF7559E97566057567B0756831756900F8
:1098B20085536A756B0085546C7B027A0179C812F4
:1098C200EE05755D02755E01755FC8029AA2906C25
:1098D20047E0600C755A05755BB0755C47029AA249
:1098E2007557057558B07559577B057AB07968E593
:1098F20053FD7C00129ECF755A02755B01755CC8E0
:10990200755D05755EB0755F76029AA2755705752D
:1099120058B0755980755A05755BB0755C90755570
:109922004E755620029AA27557057558B075599C06
:10993200755A05755BB0755C90029AA275570575EC
:1099420058B07559AA029AA27557057558B075593B
:10995200B2755A05755BB0755CC2029AA27557055D
:109962007558B07559D8755A05755BB0755CED02BE
:109972009AA27557057558B07559FF7B057AB1796A
:109982001AE553FD7C00129ECF755A02755B017574
:019992005C78
:10999300C8029AA27557057558B175592D7B057A7A
:1099A300B17941E553FD7C00129ECF755A02755B78
:1099B30001755CC8E4F555F556029AA2755705750D
:1099C30058B1755951029AA27557057558B1755911
:1099D3006A75551F755640029AA27557057558B199
:1099E300755982755A05755BB1755C99755D057519
:1099F3005EB1755FAE7555037556E8029AA2E553DD
:109A0300B4FF0B7557057558B17559C18035E553CA
:109A1300601E7557057558B17559D77B057AAF79AF
:109A23000FFD7C00129ECF7F6B7D4612076880136B
:109A33007B057AB179EAE4FDFC129ECF7F517D323A
:109A4300120768E4F555F55680557557057558B1F5
:109A53007559ED7B057AB179FDE553FD7C00129EC6
:109A6300CF755D02755E01755FC875553A75569879
:109A7300802D7557057558B275590C802275570599
:109A83007558B275591B755A05755BB2755C3EE422
:109A9300F555F55680097557057558B275594D7FBB
:109AA30002AB57AA58A9597564771206917D2DAB5D
:109AB30057AA58A9591205A87F02AB5AAA5BA95CF9
:109AC3007564771206917D3CAB5AAA5BA95C1205BB
:109AD300A87F02AB5DAA5EA95F7564771206917DCC
:109AE3004BAB5DAA5EA95F1205A812033FAF56AE4A
:059AF3005512936D22E5
:109AF8008F528B538A54895590681FE0B552047F62
:109B08000180027F00901DF7EFF07566057567B25A
:109B180075685D85536985546A85556B7B027A0142
:109B280079C812EE057F0CE55275F011A42408FDE2
:079B380012059E1293662244
:109B3F00E49001B9F0A3F0A3F09001BBE0C3943C13
:109B4F005019E4FF1293A89001BAE02FF09001B9D9
:109B5F00E03EF09001BBE004F080DE9001B9E0FE42
:109B6F00A3E0FF7C007D3C12E9F39001B9EEF0A376
:109B7F00EFF0E4A3F09001BBE0FFC3940B502FEF85
:109B8F0025E02419F582E434CAF583E493FC7401CB
:109B9F0093FDD39001BAE09D9001B9E09C500790DE
:109BAF0001BCEFF080089001BBE004F080C790018A
:109BBF00BCE0FFD3940250077B057AB2796422EFA1
:109BCF00C3940840077B057AB27968227B057AB285
:039BDF00796D227B
:109BE2009003A1E0D394005003029CA2906615E07A
:109BF20060057E007F00229003A1E075F063A4243B
:109C0200BFF582E5F0341DF583E0FFE4FCFDFE12B2
:109C1200ECCF7F007E407D007C0012EAD312ECCFB5
:109C22009003A1E075F063A424BEF582E5F0341D33
:109C3200F583E0FFE4FCFDFE12ECCF7F007E007DA9
:109C4200087C0012EAD312EAAC12ECCF9003A1E036
:109C520075F063A424C0F582E5F0341DF583E0FEBF
:109C6200A3E0FFE4FCFD12EAAC9001BF12EC82908B
:109C720001BF12EC6612ECCF7FEB7E517D007C00BF
:109C820012EB3512ECEEC374649FFF7E009001BDAF
:109C9200EEF0A3EFF0D39464EE940040087F6422C8
:0E9CA2007E007F64229001BDE0FEA3E0FF2261
:109CB000EF602C146003029D5D1200069002D474C4
:109CC00088F09002D67420F09013AF12EC668F4F9C
:109CD0008E4E8D4D8C4C7F0412A00D12006F227F92
:109CE000057B027A66791112A0CE7F817EB17D4F0D
:109CF0007C0112ECCF90661112EC6612EBB1405A67
:109D00007FC07EF37D5E7C0112ECCF90661112EC79
:109D10006612EBB16002504290661112EC6690132D
:109D2000AF12EC82E4FFFE906611E0FD12DF5A7F75
:109D3000017E00906612E0FD12DF5A7F027E0090E5
:109D40006613E0FD12DF5A7F037E00906614E0FD8B
:0E9D500012DF5AC2AF12DF6CD2AF12350522FD
:109D5E008B608A6189629069C5E07059FF12023F7B
:109D6E00E4901DF7F0FFFDAB60AA61A9621205A891
:109D7E00906991E064017031906C4BE06408702939
:109D8E00906999E0647B6021901A43E064616019E8
:109D9E007F017B027A6979997567EF1205507D0311
:109DAE007B027A6979991204C5E4FF7D0C7BEE750E
:0B9DBE00667E12092BE49069C5F022BC
:109DC900300C2290020BE075F00AA4FE90020AE022
:109DD90075F064A42EFE90020CE02E9001C3F0B53C
:089DE90007037F01227F002225
:109DF100E4FFFE12DF48906611EFF07F017E001252
:109E0100DF48906612EFF07F027E0012DF48906615
:109E110013EFF07F037E0012DF48906614EFF0909D
:109E2100661112EC669013AF12EC827F047E001271
:109E3100DF48906611EFF07F057E0012DF489066E3
:109E410012EFF0906611E0FFA3E09065FFCFF0A361
:109E5100EFF09065FFE07002A3E0600FD390660021
:109E6100E0943C9065FFE0940040089065FFE4F0C9
:109E7100A304F07F087E0012DF48906611EFF07FA7
:109E8100097E0012DF48906612EFF07F0A7E001211
:109E9100DF48906613EFF07F0B7E0012DF4890667B
:109EA10014EFF090661112EC669065F412EC8222C8
:109EB1008B588A59895A8B668A6789688F6C8E6B31
:0E9EC1008D6A8C697B027A0179C812EE052247
:109ECF008B608A6189628B668A6789688C698D6A03
:0A9EDF007B027A0179C812EE052219
:109EE9008B608A6189628B668A6789688F6C8E6BE1
:0E9EF9008D6A8C697B027A0179C812EE05220F
:109F07008B588A59895A8F5E8E5D8D5C8C5B85581C
:109F170066855967855A687F3F7E007D007C001201
:109F2700ECCFAF5EAE5DAD5CAC5B12E26212E521D9
:109F37008E698F6A7B027A0179C812EE05902D84AB
:089F4700E06004E4F080C72291
:109F4F008F577F007E007D007C0012ECCF90664E15
:109F5F0012EC6612E49470089001C4F0A3F0801F15
:109F6F007F457E617D007C0012ECCF90664E12EC37
:109F7F006612E3E512E5219001C4EEF0A3EFF09035
:109F8F002D84E06004E4F080B9E55760087B057A22
:109F9F00B2797480067B057AA779758B668A678993
:109FAF00689001C4E0FAA3E0FB7C007D3CFFAE02A9
:109FBF0012E9F38E698F6A7C007D3CAF03AE02120B
:109FCF00E9F38C6B8D6C7B027A0179C812EE052256
:109FDF00AB07EDAE047807CEC313CE13D8F9547F79
:109FEF00FF74D32BF582E43402F583EFF0ED547F49
:0E9FFF00FF74D42BF582E43402F583EFF022D8
:10A00D00AB07AF4FAE4EAD4DAC4C781C12EC011200
:10A01D00ECCF7F0F7E007D007C0012EB7F74D32B85
:10A02D00F582E43402F583EFF0AF4FAE4EAD4DAC9B
:10A03D004C781512EC0112ECCF7F7F7E007D007CF9
:10A04D000012EB7F74D42BF582E43402F583EFF02C
:10A05D00AF4FAE4EAD4DAC4C780E12EC0112ECCFB5
:10A06D007F7F7E007D007C0012EB7F74D52BF58207
:10A07D00E43402F583EFF0AF4FAE4EAD4DAC4C78FE
:10A08D000712EC0112ECCF7F7F7E007D007C001269
:10A09D00EB7F74D62BF582E43402F583EFF07F7FEE
:10A0AD007E007D007C0012ECCFAF4FAE4EAD4DACBF
:10A0BD004C12EB7F74D72BF582E43402F583EFF06D
:01A0CD002270
:10A0CE008F4A74092FF582E43402F583E0FFE4FC35
:10A0DE00FDFE781512EC1512ECCF7408254AF582A8
:10A0EE00E43402F583E0FFE4FCFDFE781C12EC156F
:10A0FE0012EAAC12ECCF740A254AF582E43402F56A
:10A10E0083E0FFE4FCFDFE780E12EC1512EAAC12B1
:10A11E00ECCF740B254AF582E43402F583E0FFE4BC
:10A12E00FCFDFE780712EC1512EAAC12ECCF740CA3
:10A13E00254AF582E43402F583E0FFE4FCFDFE12CD
:06A14E00EAAC12EC4A220B
:10A154007F1BE4FDFB1296CBC2AF7E007F287D00FF
:10A164007B027A7C795712ED47907CB37478F09037
:10A174007CB27401F0907CB47439F0907C7F741FCD
:10A18400F0A37486F0E4FFFD12D2D79001C6EFF07D
:10A19400FD907CB37404F0907CB27402F0907CB4B3
:10A1A4007441F0907C7F7419F0A3749AF07F0112CB
:10A1B400D2D7D2AF907C57E07002A3E0700A7F1C24
:0BA1C400FDFB1296CB7F00227F0122E2
:10D11C00005EBCE2613FDD83C29C7E20A3FD1F410B
:10D12C009DC3217FFCA2401E5F01E3BD3E6082DCFB
:10D13C00237D9FC1421CFEA0E1BF5D0380DE3C62EB
:10D14C00BEE0025CDF81633D7C22C09E1D43A1FFDB
:10D15C004618FAA427799BC584DA3866E5BB5907CB
:10D16C00DB856739BAE406581947A5FB7826C49ABB
:10D17C00653BD987045AB8E6A7F91B45C6987A24AB
:10D18C00F8A6441A99C7257B3A6486D85B05E7B99B
:10D19C008CD2306EEDB3510F4E10F2AC2F7193CD8B
:10D1AC00114FADF3702ECC92D38D6F31B2EC0E507B
:10D1BC00AFF1134DCE90722C6D33D18F0C52B0EE6B
:10D1CC00326C8ED0530DEFB1F0AE4C1291CF2D735B
:10D1DC00CA947628ABF517490856B4EA6937D58B4B
:10D1EC005709EBB536688AD495CB2977F4AA48163B
:10D1FC00E9B7550B88D6346A2B7597C94A14F6A82B
:10D20C00742AC896154BA9F7B6E80A54D7896B351A
:0ACCD000E4907C09F0907C32F02221
:10CCDA00E4907BEDF0A3F0C3907BEEE09FEE6480DE
:10CCEA00F8907BEDE0648098500EA3E004F07006A3
:09CCFA00907BEDE004F080DF22E4
:10CD0300C2B57F507E0012CCDAD2B57F0612CCDAE0
:10CD1300A2B5E433907BEFF07F4612CCDA907BEF41
:03CD2300E0FF220C
:10CD2600C2B5D2B5E4907BF0F0907BF0E0C39403FB
:0DCD36005005E004F080F2A2B5E433FF22C6
:10CD4300C2B5EFB40102D2B57F0D7E0012CCDAD2A8
:02CD5300B52207
:10CD5500E4907BF2F0907BF1F0907BF1E0C39408D6
:10CD6500502F12CD26EF601A907BF2E0FF907BF1F9
:10CD7500E0FE7401A806088002C333D8FC4F907BFF
:10CD8500F2F07F107E0012CCDA907BF1E004F080A7
:07CD9500C8907BF2E0FF22D1
:10CD9C00AD07E4907BF3F0907BF3E0FFC394085075
:10CDAC001EEDA807088003A2E713D8FB907BF4F0D4
:10CDBC005401FFF012CD43907BF3E004F080D87F58
:07CDCC000D7E0012CCDA22FB
:10CDD3008F4C907BF67404F0E4907C33F0FE7F2854
:10CDE300FD7B027A7C790A12ED47C2AF12CD03EFC5
:10CDF3007068907C09F0907C32F012CE62EF60553F
:10CE0300907C33E004F0E4907BF5F0907BF5E0C395
:10CE130094085032E0FF2434F582E4347CF583E057
:10CE2300FE907C33E075F008A4240AF582E4347C98
:10CE3300F583E5822FF582E43583F583EEF0907B6D
:10CE4300F5E004F080C512CE62EF6009907C33E018
:0FCE5300C3940A40ABD2AF7F0122D2AF7F00223F
:10CE6200907BF77401F0E4A3F0A304F0E4A3F0A331
:10CE7200F0129366E4907BFDF0907C08F012CD03F3
:10CE82007E00907BFEEEF0A3EFF07006907C32E025
:10CE92006007E4907C09F0FF227FF012CD9C129390
:10CEA20066E4907BFAF012CD26EFB40106907BFA8D
:10CEB2007402F07F107E0012CCDA12CD26EFB4019C
:10CEC20007907BFAE04401F0907BFAE0FF64037084
:10CED2000302CFBAEFD394004009EFC313907BFC57
:10CEE200F0804E907C09E0FF907BF7E0FEC39F50FC
:10CEF20026A3E02434F582E4347CF583E0FD907BC4
:10CF0200F9E0FCED5CD3940040047D0180027D00D9
:10CF1200907BFCEDF0800FEEB507047F0180027F6D
:10CF220000907BFCEFF0907BFCE07005907BFBEEC9
:10CF3200F0907BFCE0FFB40121907BF8E02434F513
:10CF420082E4347CF583C083C082E0FE907BF9E00A
:10CF5200FDEE4DD082D083F08020907BF8E0243427
:10CF6200F582E4347CF583C083C082E0FE907BF9D5
:10CF7200E0F4FDEE5DD082D083F012CD43907BF7DA
:10CF8200E004F0907BF9E0FF25E0F0701C907BF864
:10CF9200E02434F582E4347CF583E0FF12CFF19093
:10CFA2007BF8E004F0A3E004F0129366907BF8E0D3
:10CFB200C39408500302CEA3907BF7E0C394414090
:10CFC20006907C08E06007E4907C09F0801B907B6F
:10CFD200FBE0907C09F070047F0180027F00907C6E
:0FCFE20032EFF0907BFD7401F0907BFDE0FF22B9
:0FCFF100907C08E06F90D11C93FF907C08F02299
:10D00000AC0712CD03EF6005D2AF7F00227F55122F
:10D01000CD9CE4907C00F0907C00E0FFC39408502D
:10D0200025EC75F008A4240AF582E4347CF583E548
:10D03000822FF582E43583F583E0FF12CD9C907C4E
:09D0400000E004F080D17F012220
:10D04900AA07A905C2AF12D000EF7002FF227F0F15
:10D0590012CD9CAF0112CD9CE4FF12CD9CAF0312FF
:10D06900CD9CAF0212D000EF7002FF227FAA12CD31
:10D079009C12CD55907C01EFF012CD55907C02EFBA
:10D08900F012CD55907C03EFF012CD55907C04EF52
:10D09900F0AF0212D000EF7002FF227F5512CD9C33
:10D0A900907C01E0FF12CD9C907C02E0FF12CD9CA8
:10D0B900907C03E0FF12CD9C1293667FBC7E021226
:10D0C900CCDA12936612CD03EF6005D2AF7F00224E
:05D0D900D2AF7F01222F
:10D0DE00AC07AB0512CD03EF60037F0022C2AFAFEA
:10D0EE000412D0007FF012CD9CAF0312CD9CE4FF52
:10D0FE0012CD9C12CD55907C07EFF012CD03EF6050
:0ED10E0005D2AF7F0022D2AF907C07E0FF2257
:10DF2A0025642E20253575202825732900414E5455
:0EDF3A002B53706F7274005375756E746F0008
:10CCAD00417C8901417C8A07417CB607487CAAB941
:10CCBD00A521FBBD72C345487C81B9AD3228757E77
:02CCCD00C74D51
:10D21C0012D2C47F647E0012DEE6E4907C3CF09077
:10D22C007C3CE004F012DE09EF64016009907C3C68
:10D23C00E0C3940A40E91293667F647E0012DEE636
:10D24C0012D2C47F647E0012DEE6129366E4907CF8
:10D25C003CF0907C3CE004F012D8CAEF6401600909
:10D26C00907C3CE0C3940A40E97FD07E0712DEE656
:10D27C00E4907C3CF0907CB3E0B4780DE4FF7B024E
:10D28C007A7C79AA12D7FD8012907CB3E0B4040B9F
:10D29C00E4FF7B027A7C798112D7FD907C3CE00420
:10D2AC00F012DC20EF6009907C3CE0C3940A40C58E
:08D2BC007F647E0012DEE62211
:10D2C4005328BF908000E528F0000000432840E583
:03D2D40028F0221D
:10D2D7008F4A907C40EDF012D21CE4907C3DF09098
:10D2E7007C3DE0FFC39408400302D417E4FDFC1221
:10D2F700DD12E4907C3EF0907C3EE004F0E4A3F085
:10D30700907C3FE004F0907C3DE0FF7D5112D79583
:10D31700EF64016009907C3FE0C3940A40E2E49027
:10D327007C3FF0907C3FE004F012DC95EF640160F5
:10D3370009907C3FE0C3940A40E9907C3DE0FF12EE
:10D34700DA96907C9FEEF0A3EFF0129366907C9FA5
:10D35700E07002A3E07009907C3EE0C394324097EE
:10D36700907C3EE0C39432400302D4171293667F49
:10D37700057D4B7BE975667912092B907C9FE0FE52
:10D38700A3E0FF907C40E0FD25E02457F582E434DC
:10D397007CF583EEF0A3EFF0748B2DF582E4347CFB
:10D3A700F583E54AF07566057567DF75682AED044C
:10D3B700756900F56A907C9FE0FEA3E08E6BF56CC3
:10D3C700E54A70087B057ADF793780067B057ADFC7
:10D3D70079418B6D8A6E896F7B027A0179C812EE6B
:10D3E70005907C40E0FE1313543F75F064A42414A9
:10D3F700FFEE540375F00AA42450FD1204BB120378
:10D407003F907C40E004F0907C3DE004F002D2E6DF
:09D4170012D21C907C40E0FF22BF
:10D420008F4F8D5012DC33EF7002FF22E55024FE47
:10D43000605A14700302D4D92402600302D5251265
:10D44000DABBEF64A5703F907C89E0640170377FA0
:10D450000112DB6FEF640160037F00227F4112DB6A
:10D460006FEF640160037F0022AF4F12DB6FEF6448
:10D470000160037F0022E54F64E5FF12DB6FEF647C
:10D480000160067F00227F00227F012212DABBEFBB
:10D4900064A5703F907C89E0640170377F0112DBE6
:10D4A0006FEF640160037F00227F4B12DB6FEF643C
:10D4B0000160037F0022AF4F12DB6FEF6401600356
:10D4C0007F0022E54F64EFFF12DB6FEF640160061F
:10D4D0007F00227F00227F012212DABBEF64A57059
:10D4E0003F907C89E0640170377F0112DB6FEF644D
:10D4F0000160037F00227F4C12DB6FEF6401600349
:10D500007F0022AF4F12DB6FEF640160037F0022C8
:10D51000E54F64E8FF12DB6FEF640160067F0022D5
:06D520007F00227F0122C2
:10D526008F4F8D508B5112DC33EF7002FF2212DACF
:10D53600BBEF64A5705D907C89E0640170557F0344
:10D5460012DB6FEF640160037F00227F4212DB6F04
:10D55600EF640160037F0022AF4F12DB6FEF6401BF
:10D5660060037F0022AF5012DB6FEF640160037F20
:10D576000022AF5112DB6FEF640160037F0022E5EA
:10D586004F64E465506551FF12DB6FEF640160067E
:09D596007F00227F00227F0122A8
:10D59F008F4F8C508D518B5212DC33EF7002FF2264
:10D5AF0012DABBEF64A5600302D63F907C89E0647A
:10D5BF0001600302D63F7F0512DB6FEF640160034A
:10D5CF007F00227F5112DB6FEF640160037F002227
:10D5DF00AF4F12DB6FEF640160037F0022AF51E5A5
:10D5EF005112DB6FEF640160037F0022E550FF12E1
:10D5FF00DB6FEF640160037F0022AF5212DB6FEF2E
:10D60F00640160037F0022AF5312DB6FEF64016090
:10D61F00037F0022E551E54F64F16551FDE5506D43
:10D62F0065526553FF12DB6FEF640160067F0022C6
:06D63F007F00227F0122A2
:10D645008F4F8C508D5112DC33EF7002FF2212DAAE
:10D65500BBEF64A57064907C89E06401705C7F0316
:10D6650012DB6FEF640160037F00227F4312DB6FE3
:10D67500EF640160037F0022AF4F12DB6FEF64019F
:10D6850060037F0022AF51E55112DB6FEF6401604B
:10D69500037F0022E550FF12DB6FEF640160037F1B
:10D6A5000022E551E54F64E56551FDE5506DFF123A
:10D6B500DB6FEF640160067F00227F00227F01227D
:10D6C5008F4F8D5012DC33EF7002FF2212DABBEF61
:10D6D50064A5704E907C89E0640170467F0212DB80
:10D6E5006FEF640160037F00227F4412DB6FEF64FC
:10D6F5000160037F0022AF4F12DB6FEF640160030F
:10D705007F0022AF5012DB6FEF640160037F0022C0
:10D71500E54F64E36550FF12DB6FEF640160067F40
:08D7250000227F00227F012297
:10D72D008F4F8D5012DC33EF7002FF2212DABBEFF8
:10D73D0064A5704E907C89E0640170467F0212DB17
:10D74D006FEF640160037F00227F4512DB6FEF6492
:10D75D000160037F0022AF4F12DB6FEF64016003A6
:10D76D007F0022AF5012DB6FEF640160037F002258
:10D77D00E54F64E26550FF12DB6FEF640160067FD9
:08D78D0000227F00227F01222F
:10D795008F4B8D4C12DC33EF7002FF2212DABBEF98
:10D7A50064A5704E907C89E0640170467F0212DBAF
:10D7B5006FEF640160037F00227F4D12DB6FEF6422
:10D7C5000160037F0022AF4B12DB6FEF6401600342
:10D7D5007F0022AF4C12DB6FEF640160037F0022F4
:10D7E500E54B64EA654CFF12DB6FEF640160067F71
:08D7F50000227F00227F0122C7
:10D7FD008F4B8B4C8A4D894E12DC33EF7002FF221A
:10D80D0012DABBEF64A5600302D8C4907C89E06492
:10D81D0001600302D8C4907C4274A5F07F0912DB2D
:10D82D006FEF640160037F0022907C42E06409F099
:10D83D007F4612DB6FEF640160037F0022907C4214
:10D84D00E06446F0AF4B12DB6FEF640160037F00C5
:10D85D0022907C42E0654BF0E4907C41F0907C415D
:10D86D00E0FFC394085040AB4CAA4DA94E8F827572
:10D87D00830012E99CFF12DB6FEF640160037F00F0
:10D88D0022907C42E0FFAB4CAA4DA94E907C41E02A
:10D89D00F58275830012E99CFEEF6E907C42F0904C
:10D8AD007C41E004F080B6907C42E0FF12DB6FEF2C
:0DD8BD00640160067F00227F00227F0122AF
:10D8CA0012DABBEF64A5703C907C89E06401703485
:10D8DA007F0112DB6FEF640160037F00227F4A122F
:10D8EA00DB6FEF640160037F0022E4FF12DB6FEF5E
:10D8FA00640160037F00227FEE12DB6FEF64016038
:0AD90A00067F00227F00227F012229
:10D914008F548B558A56895712DABB907C43EFF0AB
:10D92400907C89E06401600302DA93907C43E0FF19
:10D93400245C600302DA93907C45EFF012DABB902A
:10D944007CA9EFF0907C89E0B40112907C45E0FF63
:10D95400907CA9E0FEEF6E907C45F080037FFF226F
:10D9640012DABB907CB6EFF0907C89E0B40112909F
:10D974007C45E0FF907CB6E0FEEF6E907C45F08045
:10D98400037FFF2212DABB907C8AEFF0907C89E05F
:10D99400B40112907C45E0FF907C8AE0FEEF6E902B
:10D9A4007C45F080037FFF22E4907C44F0907C442B
:10D9B400E0FFC39408501474A12FF582E4347CF57D
:10D9C40083E4F0907C44E004F080E2E4907C44F052
:10D9D400907CA9E014FF907C44E0C39F503E12DA8F
:10D9E400BB907C44E0FE24A1F582E4347CF583EF13
:10D9F400F0907C89E0B40119907C45E0FF74A12E7D
:10DA0400F582E4347CF583E0FEEF6E907C45F08093
:10DA1400037FFF22907C44E004F080B4907C45E0D6
:10DA2400FEC00612DABBD0E06F907C45F0706090C7
:10DA34007CA9E064037010907CB6E0B44006907C4E
:10DA4400A2E0FF227FFF2274F4FF7E0112DEE69043
:10DA54007CA7E0FF907CB5E06F6031EFF0AB55AA96
:10DA640056A957AE02AF01EF4E601E907CB3E0B4EE
:10DA74007809907CA8E012E9CB800E907CB3E0B4E6
:10DA84000407907CA1E012E9CB7F42227F40227FF1
:02DA940041222D
:10DA9600907CB6E0B45107907C8AE06F60057E000A
:10DAA6007F0022907CA2E0FE907CA1E07C00240016
:05DAB600FFEC3EFE2222
:10DABB00907C467401F0E4A3F0907C8904F012D2C0
:10DACB00C4E4907C48F0907C48E0C3940840030287
:10DADB00DB601293665328FB908000E528F0000072
:10DAEB000000000000000000432804E528F0E4904B
:10DAFB007C49F0A3F0907C4AE004F07006907C49DE
:10DB0B00E004F012936620950FC3907C4AE09410CA
:10DB1B00907C49E0942740DDC3907C4AE0941090C0
:10DB2B007C49E094274009907C897402F07F0022A5
:10DB3B00908002E0F52A30E109907C46E0FFA3E0FB
:10DB4B002FF012D2C4907C46E025E0F0907C48E0A8
:10DB5B0004F002DAD1432801908000E528F0907C94
:04DB6B0047E0FF226E
:10DB6F008F54907C4B7401F0907C89F012D2C4E4F6
:10DB7F00907C4CF0907C4CE0C39408400302DC1A7C
:10DB8F00129366907C4BE05554600B4328029080B3
:10DB9F0000E528F080095328FD908000E528F05318
:10DBAF0028FB908000E528F0000000000000000036
:10DBBF000000432804E528F0E4907C4DF0A3F0909A
:10DBCF007C4EE004F07006907C4DE004F0129366FA
:10DBDF0020950FC3907C4EE09410907C4DE09427DD
:10DBEF0040DDC3907C4EE09410907C4DE094274034
:10DBFF0009907C897403F07F002212D2C4907C4B71
:10DC0F00E025E0F0A3E004F002DB83907C89E0FFE5
:01DC1F0022E2
:10DC200012DC95EFB40109E4FFFBFAF912D91422D2
:03DC30007F02224E
:10DC3300908002E0F52A20E008E4FFFBFAF912D90C
:10DC4300145328FE908000E528F0129366E4907C3C
:10DC53004FF0907C4FE0D394C85018908002E0F5C9
:10DC63002A30E00F00000000129366907C4FE0041E
:10DC7300F080DF907C4FE0C394C8401343280190A9
:10DC83008000E528F07F027E0012DEE67F00227F1F
:02DC930001226C
:10DC9500129366432801908000E528F0E4907C50BB
:10DCA500F0A3F0C3907C51E094E8907C50E094039D
:10DCB500501C908002E0F52A30E013129366907CA8
:10DCC50051E004F07006907C50E004F080D5C390DC
:10DCD5007C51E094E8907C50E0940340037F00225F
:03DCE5007F01229A
:10DCE8008B458A468947129366432801908000E550
:10DCF80028F0908002E0F52A20E00C7F01AB45AACD
:0ADD080046A94712D914227F4122D8
:10DD12008F4B8C4C8D4DE4F54EAF4BE4FDFB12D591
:10DD220026054E12DC20EF6007E54EC3941440E94D
:10DD3200E54EC3941440037F0022E4F54EAF4BAD91
:10DD42004DAC4C907CB3E0FB907CB2E0F55312D525
:10DD52009F054E12DC20EF6007E54EC3941440DDB0
:10DD6200E54EC3941440037F0022E4F54EAF4B907E
:10DD72007CB4E0FD12D72D054E12DC20EF6007E5E2
:10DD82004EC3941440E7E54EC3941440037F00222F
:10DD9200E4F54E907C80E025E0FD907C7FE033FC52
:10DDA200AF4B12D645054E12DC20EF6007E54EC39D
:10DDB200941440DFE54EC3941440037F0022E4F53F
:10DDC2004EAF4B7DF012D6C5054E12DC20EF600738
:10DDD200E54EC3941440EAE54EC3941440037F0019
:10DDE20022E4F54EAF4B7D0212D420054E12DC2008
:10DDF200EF6007E54EC3941440EAE54EC394144025
:07DE0200037F00227F0122D3
:10DE0900129366432804908000E528F0432801E531
:10DE190028F05328FDE528F0D2955328FBE528F092
:10DE2900E4907C52F0A3F0C3907C53E094FA907C88
:10DE390052E09400500EA3E004F07006907C52E08A
:10DE490004F080E35328FE908000E528F0E4907CFC
:10DE590052F0A3F0907C53E004F07006907C52E0FD
:10DE690004F0129366908002E0F52A20E00FC39037
:10DE79007C53E09430907C52E0947540D7C3907CF9
:10DE890053E09430907C52E0947540037F0022E483
:10DE9900907C52F0A3F0907C53E004F07006907CE3
:10DEA90052E004F0129366908002E0F52A30E00F08
:10DEB900C3907C53E09430907C52E0947540D7C372
:10DEC900907C53E09430907C52E0947540037F003D
:0DDED90022432804908000E528F07F0122FC
:10DEE6008E588F59E4907C55F0A3F0C3907C56E091
:10DEF6009559907C55E095585029E4907C54F090C3
:10DF06007C54E0C39419500B129366907C54E00441
:10DF1600F080EC907C56E004F07006907C55E004AE
:04DF2600F080C8229D
:10DF4800E5D220E0FB75D2028F828E83E0FFE4F5F4
:02DF5800D222D3
:10DF5A00E5D220E0FB75D2028F828E83EDF0E4F5E4
:02DF6A00D222C1
:10DF6C00C2AFE5D220E0FB75D25075D2A0D2AF2261
:10DF7C00E4907CB7F0907CB7E0C39F500600E004BF
:04DF8C00F080F2220D
:10DF9000AE07EE7003430501C2C27F0C12DF7CD2D4
:10DFA000B312DF7C907CB87401F0907CB8E0D3941D
:10DFB00008501FED1392B47F0C12DF7CD2C212DF27
:10DFC0007CC2C212DF7CEDC313FD907CB8E004F08C
:10DFD00080D8EE64017039907CB804F0907CB8E091
:10DFE000D39408501FEB1392B47F0C12DF7CD2C283
:10DFF00012DF7CC2C212DF7CEBC313FB907CB8E063
:10E0000004F080D87F0C12DF7CC2B312DF7C805515
:10E01000EE7052907CB904F0E4FB907CB804F09070
:10E020007CB8E0D39408502E7F0C12DF7CD2C21251
:10E03000DF7CD2B430B406907CB9E02BFB907CB985
:10E04000E025E0F07F0C12DF7CC2C212DF7C907C06
:10E05000B8E004F080C97F0C12DF7CC2B312DF7C11
:08E06000C2B4AF03227F0022CD
:10E06800EF75F00A84C454F0FEEF75F00A84EE25CB
:03E07800F0FF2294
:10E07B00EF5DFEC4540F75F00AA4FEEF540F2EFF94
:01E08B002272
:10E08C00C2AFEF700302E11514600302E1B57F012A
:10E09C007D8EE4FB12DF909066A3E0FF12E068AB8C
:10E0AC00077F017D8412DF909066A2E0FF12E0688A
:10E0BC00AB077F017D8212DF909066A1E0FF12E03A
:10E0CC0068AB077F017D8012DF909066A4E0FF12A1
:10E0DC00E068AB077F017D8612DF909066A5E0FFBC
:10E0EC0012E068AB077F017D8812DF909066A6E096
:10E0FC00FF12E068AB077F017D8C12DF907F017D02
:10E10C008E7B8012DF9002E1B5E4FF7D84FB12DF91
:10E11C0090907CBAEFF030E70EE0FF7D1012E07BC0
:10E12C009066A3EFF0800F907CBAE0FF7D3012E098
:10E13C007B9066A3EFF0E4FF7D82FB12DF90907C76
:10E14C00BAEFF07D7012E07B9066A2EFF0E4FF7DF9
:10E15C0080FB12DF90907CBAEFF07D7012E07B9028
:10E16C0066A1EFF0E4FF7D86FB12DF90907CBAEFA6
:10E17C00F07D3012E07B9066A4EFF0E4FF7D88FB2D
:10E18C0012DF90907CBAEFF07D1012E07B9066A5C8
:10E19C00EFF0E4FF7D8CFB12DF90907CBAEFF07D0A
:0CE1AC00FF12E07B9066A6EFF0D2AF22DD
:10E1B800020C37E493A3F8E493A34003F68001F23A
:10E1C80008DFF48029E493A3F85407240CC8C33368
:10E1D800C4540F4420C8834004F456800146F6DF37
:10E1E800E4800B010204081020408090CA58E47EA5
:10E1F800019360BCA3FF543F30E509541FFEE4932C
:10E20800A360010ECF54C025E060A840B8E493A3F2
:10E21800FAE493A3F8E493A3C8C582C8CAC583CA1D
:10E22800F0A3C8C582C8CAC583CADFE9DEE780BED5
:01CCCF000064
:0300000002E238E1
:0CE23800787FE4F6D8FD75817E02E1F3EA
:10E24400DA0CD902800BD906300701B3500502E578
:10E25400D6920702E5C2D9F680F9D2068002C20638
:10E2640012E607300606C86002B207C89206DAD082
:10E27400D9E4B8000A12E64EA206920702E5AB60A2
:10E28400FBB53100400F12E64EA20692F7A20792A8
:10E2940006A2F79207C398F40424E740DF2419ADDB
:10E2A4002DAC2CAB2B7A00C394084008CDCCCBFA10
:10E2B400E4CD80F424086010F9C3ED13FDEC13FCE5
:10E2C400EB13FBEA13FAD9F1A206300701B340308D
:10E2D4008A35E52E2BF536E52F3CF537E5303DF54F
:10E2E40038501A13F538E53713F537E53613F53694
:10E2F400E53513F5350531E5317002053202E56186
:10E30400E4C39AF535E52E9BF536E52F9CF537E504
:10E31400309DF538500DB207C378357F04E496F686
:10E3240008DFFA7A047019E531C39408F531500214
:10E334001532E4C535C536C537F538DAE802E602E4
:10E3440020E7BAE5317002153215317835C37F0400
:08E35400E633F608DFFA80E869
:10E35C00DA03B8000302E5D6D9028002D9F702E548
:10E36C00C212E607300701B392077004D9E78005A3
:10E37C00DADEB8000302E602D9E2C3947E5002153D
:10E38C00322531F531500205327833760008B83930
:10E39C00FA782B7933E608FAE8FC782E8AF0E6084E
:10E3AC00A427F709E5F037F7500989F00907E7606A
:10E3BC00FBA9F0B831E61919ECF8B82ED802E561D2
:10E3CC0002E5EDB8FFFA02E5D6D9FB02E5C2DAF6B2
:10E3DC00B800F002E60212EB9212E607300701B326
:10E3EC0092077007D9E3B800E280DBDAE1B80002EB
:10E3FC0080E1D9D5C8C39850021532247F5002054C
:10E40C0032F531783876007A1A7B80C3E52E952B5D
:10E41C00E52F952CE530952D4016C3E52E952BF563
:10E42C002EE52F952CF52FE530952DF530E64BF696
:10E43C00DA0302E561EB03FB30E703187600C3E572
:10E44C002E33F52EE52F33F52FE53033F53040CA5A
:05E45C0030E7DD80B691
:10E46100D908A207300601B3400A12E5D67480220A
:10E47100DAF8D9ECA2069206D082D08312ECF6C06B
:10E4810083C082A206E492E1B2E11422D9DCA207A0
:10E49100B380E312E6079206DAD6D9F0A207300676
:10E4A10001B35005A207B380CDFEFFC3985004AF5E
:10E4B10031F404C3136009C3EE983007B9B380B6D1
:10E4C100EFF539B206EED083D08212E276C082C077
:10E4D10083E8600EC539C3953994145005A207B37A
:04E4E10080A3E4220E
:10E4E5007920800C7910800479087D007E007F00FA
:10E4F5003392D530D50312EBA3EC33400FEF33FF46
:10E50500EE33FEED33FDEC33FCD9EE22EECCF5F027
:0CE51500747E29A2D513FF92F7AEF0220D
:10E52100EF8EF0A2F7D2F73392D5C3947F5006E471
:10E53100FFFEFDFC229420400474FF80F304CCFE16
:10E54100E4FFFAE5F0CC6012C3CC13CCCD13CDCEF1
:10E5510013CECF13CF0450EEDAEC30D5D702EBA3B4
:10EDA600E57A2466F8E6057A2278633018027866F2
:10EDB600E475F00112ECBF02E9812011EB7F2ED23F
:10EDC600118018EF540F2490D43440D4FF30150B23
:10EDD600EF24BFB41A0050032461FFE57B600215DF
:10EDE6007B057EE57E7002057D20195830180D786A
:10EDF60063E475F00112ECBFEF02E9CB02F557743C
:10EE060003D2188003E4C218F57A8B638A64896595
:10EE1600E4F57BF57DF57EE57B60077F2012EDE16D
:10EE260080F5F57CC212C211C213C214C216C217F3
:10EE3600C21912EDAFFF700D3018057F0012EDF507
:10EE4600AF7EAE7D22B42550C2D5C21512EDAFFFFE
:10EE560024D0B40A00501E75F00A20D50DC57BA437
:10EE6600257BF57B7002D21480E0D211C57CA425E7
:10EE76007CF57C80D524CFB41A00EF5004C2E5D2CD
:10EE86001502F0C6D21280C0D21180BCD21380B84F
:10EE9600D2D580B612EDA6FF12EDE102EE1DD21715
:10EEA60080A6D21680A212EDA6FB12EDA6FA12EDEE
:10EEB600A6F94A4B700679B17AF17B05201333E542
:10EEC6007B602FAF7CBF00011F7E008E82758300A2
:10EED60012E99C60050EEE6F70F1C2D5EBC0E0EA58
:10EEE600C0E0E9C0E0EE12F121D0E0F9D0E0FAD0BE
:10EEF600E0FB12E981FF60A3EBC0E0EAC0E0E9C0F5
:10EF0600E012EDE1D0E02401F9D0E03400FAD0E0DF
:10EF1600FBE57C60DDD57CDA8081D213809E12F120
:10EF26000660F7E57C12E664A97C600BE57C12F1CD
:10EF3600A4EF7003D57CF5EA30E702F404C39950D8
:10EF460077EAF4257C0430E701E404F57C800D12B1
:10EF5600F10660C6EA057C257C12E664EA7879F655
:10EF660030E701E4257C04D57C042016011412F157
:10EF760021E4C0E012F1A47879E6601320E70714D3
:10EF8600F612EDC9802204F6D0E014C0E07F00122C
:10EF9600EDC9E57C600712EDC0157C800B301603C9
:10EFA60012EDC0D0E002EE1DD0E00480C512F106DD
:10EFB60060A0E57C0412E6647879EAF6E57C042034
:10EFC6001602600104240412F12174FF04C0E01249
:10EFD600F1A412EDC9E57C201602600312EDC0D043
:10EFE600E0B57CE87F4512EDD37879E67F2B30E7F4
:10EFF600047F2DF404C0E012EDE1D0E075F00A8440
:10F00600C0F012EDCAD0E012EDCA02EE1D791080F2
:10F016000C79088008D2D5790A8006790AC2D5C249
:01F0260017D2
:10F02700E4FAFDFEFF12EDA6FC7B0820121312ED99
:10F03700A6FD7B1030110A12EDA6FE12EDA6FF7B8E
:10F0470020EC3382D592D55013C3E43011069FFFCD
:10F05700E49EFEE42012039DFDE49CFCE4CBF8C291
:10F0670012EC700CCFCECDCCE824F8F870F38017F3
:10F07700C3EF33FFEE33FEED33FDEC33FCEB33FB35
:10F08700994002FB0FD8E9EB301205F8D0E0C448ED
:10F09700B212C0E00AEC4D4E4F78207B0070C2EAF6
:10F0A700C0E012F123D0F0D0E0201204C4C0E0C4C5
:10F0B700B212C0F012EDCAD0F0D5F0EB02EE1D127D
:10F0C700ED21EEAC53F01358EE8E4CEE8A42F0175A
:10F0D7004FF01B44F01B49EE9A43F02155EF55467C
:10F0E700EFB345EF2447F1C350EE922DEE962EEE87
:10F0F700A42BEEA823EE9420F1BE2A0000EE9E106A
:10F107001103757C0612EDA6FC12EDA6FD12EDA605
:10F11700FE12EDA6FF787202E691790AA2D52014B5
:10F1270014301609B910020404B9080104A2D52045
:10F1370017025001042013619213B57B005032C0AF
:10F14700E07F203014177F30A21372177216500D0C
:10F1570012F178C213C217C2167F30800F30160320
:10F16700E9C0E012EDE1301603D0E0F9D0E0B57B5D
:10F17700CE3016177F30B9100C12EDE17F583015DD
:10F18700077F788003B9080312EDE13013057F2D5F
:10F1970002EDE17F2B2017F822921380D47F00B471
:10F1A700070050052472F8E6FF22286E756C6C295B
:10F1B700002D4958504443D21902EE4E12EDA6B421
:10F1C70006004001E490F1B89312EDD2743A12EDC3
:09F1D700D2D214757B0402F0137E
:10F1E0009E92DA331160B135FEE57F37898421398B
:10F1F000FFC3AE3A5B951D3C4758633DF0FD753E3D
:10F200001872313F0000803F02E7FD02E80DD9FB94
:10F2100050F602E80812E7E2D9F412ECCF7C3B7D0D
:10F22000AA7EB87F3F12E36D12E7E292D5247B50AD
:10F2300010A2D570DB500AE5F024045004A2D5805A
:10F24000CF12E7D912ECCF12E521EFF582F404FCDE
:10F2500012E4ED12E262C08290F1E0740912E7AAB2
:10F2600012E7E2D0F092D525F0A2D57001C313FFCA
:05F27000EE92E7FE2212
:10F27500DA48923ECDCCCC3EABAA2A3F00000040F6
:10F285000000803FF037983FF304B53FFC44D73F7B
:10F295001772313E1772B13E9115053FD95BDE3EBF
:10F2A50002E80DD9FB02E7FDD2108002C21012E779
:10F2B500E2D9F040EBD360EDC5F07F3FFEF8ED7A83
:10F2C50000C39496C8948B40230AC89469C8941ABD
:10F2D500401A0AC89468C8941F40110AC8945AC8AD
:10F2E5009425400805F07A00CEC2E7CEC0F08C41E7
:10F2F5008D428E438F44EA2323C0E02485F5827531
:10F3050083F25002058312ECCFC083C08212EC72E7
:10F31500D082D08312E25EEFB2E7FF12E7D912EC9A
:10F325007212ECCFAC41AD42AE43AF4412E2621271
:10F33500ECCF12E7D012E3E28C418D428E438F442D
:10F3450090F275740312E7A012ECCFAC41AD42AE5A
:10F3550043AF4412E36DD0E060142491F5827583C8
:10F36500F25002058312ECCF12EC7212E26212E740
:10F37500D9D0E0C3947FFDE49400FC12E4E912ECDB
:10F38500CF7C187D727E317F3F12E36D12ECCF1278
:10F39500E7D012E26230100E12ECCF7CD97D5B7E95
:07F3A500DE7F3E12E36D2242
:10F3AC0083FA703AE4E9AABCF8E0813EE6E99DBF35
:10F3BC000000803F1A3C2839666999BBE335A33DB0
:10F3CC00E75D25BFDB0FC93FCCDB8D41EE3649C471
:10F3DC003F91C9453DF8B0C50000803F34F517C3D7
:10F3EC0073FA2F45DDFD0AC612F49B04A2E19211BB
:10F3FC001420E01590F3AC740412E7A0802912F4E9
:10F40C009B30E102B21120E0EB8C4C8D4D8E4E8F77
:10F41C004F90F3C0740412E7A012ECCFAC4CAD4D7E
:10F42C00AE4EAF4F12E36D301104EF6480FFEE333C
:10F43C00EF337001FF2212F49BC0E08C4C8D4D8E8B
:10F44C004E8F4F90F3E4740312E7A012ECCFAC4C48
:10F45C00AD4DAE4EAF4F12E36DECC54CFCEDC54D52
:10F46C00FDEEC54EFEEFC54FFF90F3D4740312E7CB
:10F47C00A0D08212ECCFAC4CAD4DAE4EAF4FE5826E
:10F48C0030E00712E3E5B211809D12E3E28098EEC2
:10F49C0033EF3324605007D0E0D0E002E80DEFA248
:10F4AC00E7547F9211FF12ECCF7C837DF97E227F93
:10F4BC003E12E36DEE33EF332481501012ECCF1279
:10F4CC00E52112E4E5EFB2E7FF12E262EE33EF332F
:10F4DC00602A2403F8C313FFEE92E7FEE82481E4CC
:10F4EC00501A12ECCF12E521EF04C2E0FCC0E0127E
:10F4FC00E4EDEFB2E7FF12E262D0E003FAEE33EF95
:10F50C0033600B148FF0A2F713FFEE92E7FEEA22A2
:10E56100E53820E7137835C37F04E633F608DFFA90
:10E57100E531700215321531E5353378367F03E622
:10E581003400F6500E08DFF77538800531E531703B
:10E59100020532E53220E7547027E531604E046010
:10E5A1002085383085372F85362E5320F0AC2EAD9F
:10E5B1002FA207E53113FFE53092E7FEA83102EC07
:10E5C100F6E4F530F52FF52EF5327531FF5320F0D5
:10E5D10043200580D874FFF530F52FF52E753200F4
:10E5E100F531D2075320F043200980C15320F04375
:10E5F1002003E4F530F52FF52EF532F531C2078011
:06E60100AC5320F080EC98
:10E6070079017A018530F0E531A2F7339207753247
:10E6170000F5316002D2F785F030A831B8FF08095C
:10E62700E530C2E76001098C2B8D2C8EF0A2F7EF45
:10E637003304700A0AC2F705F00AD5F0011A14600C
:07E6470002D2F785F02D223D
:10E64E00C88831C530C52DC530C52FC52CC52FC5C1
:06E65E002EC52BC52E2283
:10E66400F91420E72524FA50037907E4F42402FB83
:10E6740018DBFDE624FB5011E4F618E604F6B40AB0
:0DE6840008E4F6D9F57401F60A22C2D52289
:10E69100EE33EF3392D5FB602AB4FF33EEC2E77B52
:10E6A1000560067AE679B6E4227AE679BF20D504D8
:10E6B1007AE679BA224E614E002B494E46002D4929
:10E6C1004E4600E47A08F608DAFC7B007407221251
:10E6D100ECCF8882EBFF75F010A4FAABF08FF074E9
:10E6E1004DA42BFBACF050010CC3EA94F0FAEB946F
:10E6F1003AFBEC9426FCE530C2E7FF75F056A4F432
:10E701002414C5F0F434C58FF0A42AE5F03BE43CB1
:10E71100F620E70B12E84D12ED0E12E3E5800BF443
:10E721000412E84D12ED0E12E36DEE33EF33C39494
:10E731008240097050EED2E794A0504912ECF6A83D
:10E7410082E6FAEEA2E7D2E7FEEF332482FBE4C3CE
:10E75100CC33CCCD33CDCE33CE33DBF3F6087B07D0
:10E761008CF0740AA4FCAFF08DF0740AA42FFDAFF5
:10E77100F050010F8EF0740AA42FFEE435F0F60874
:10E78100DBDE740722A882E604F620E70812E84DD2
:0FE7910012E3E580AAF40412E84D12E36D80A0B4
:10E7A000C0E012ECCF12E36D8002C0E012E7D91294
:10E7B000EC72A3D0E0C0E012ECCF12E7D012E36D10
:10E7C00012ECCF12EC72A312E262D0E0D5E0E622A6
:10E7D000AC3BAD3CAE3DAF3E228C3B8D3C8E3D8F85
:10E7E0003E2279018EF0A2F7EF3304700A09C2F7D6
:10E7F00005F009D5F0011A146002D2F72274FF1354
:10E80000FF7E80E47805800BE47803800474FF7851
:0DE8100009FFFEFDFCE52054F048F5202234
:10E81D000000803F000020410000C84200007A4403
:10E82D0000401C460050C347002474498096184B85
:10E83D0020BCBE4CCA1B0E5A1CC25367AEC59D747C
:10E84D00FB600654076014232312E86EEB54386006
:10E85D002A12ECCF12E86812E36D22EB5438032430
:10E86D001CAA83A98290E81DFF93FCEFA393FDEFF3
:0CE87D00A393FEEFA393FF8A83898222FD
:10E88900E709F608DFFA8046E709F208DFFA803E71
:10E8990088828C83E709F0A3DFFA8076E309F6081A
:10E8A900DFFA806EE309F208DFFA806688828C83DA
:10E8B900E309F0A3DFFA805A89828A83E0A3F60884
:10E8C900DFFA804E89828A83E0A3F208DFFA804268
:10E8D90080AE80B480BA80C480CA80D080DA80E4F7
:10E8E90080378023805389828A83ECFAE493A3C812
:10E8F900C582C8CCC583CCF0A3C8C582C8CCC583A2
:10E90900CCDFE9DEE7800D89828A83E493A3F608E8
:10E91900DFF9ECFAA9F0EDFB2289828A83ECFAE0AF
:10E92900A3C8C582C8CCC583CCF0A3C8C582C8CC4E
:10E93900C583CCDFEADEE880DB89828A83E493A39E
:10E94900F208DFF980CC88F0ED14B4040050C32438
:10E959001E83F582EB14B4050050B7241583258274
:10E96900F582EF4E60ACEF60010EE58290E8D97355
:08E97900000402000C0600126C
:10E98100BB020689828A83E0224003BB0402E7229C
:0BE99100400789828A83E49322E3227E
:10E99C00BB020CE58229F582E5833AF583E022403F
:10E9AC0003BB0406E92582F8E622400DE58229F531
:0FE9BC0082E5833AF583E49322E92582F8E2228B
:10E9CB00BB020689828A83F0224003BB0402F72232
:04E9DB005001F322D2
:10E9DF00EFF88DF0A4FFEDC5F0CEA42EFEEC88F07D
:04E9EF00A42EFE2232
:10E9F300BC000BBE0029EF8DF084FFADF022E4CC08
:10EA0300F875F008EF2FFFEE33FEEC33FCEE9DECD0
:10EA1300984005FCEE9DFE0FD5F0E9E4CEFD22ED16
:10EA2300F8F5F0EE8420D21CFEADF075F008EF2F60
:10EA3300FFED33FD4007985006D5F0F222C398FD51
:05EA43000FD5F0EA22EE
:10EA4800C2D5EC30E709B2D5E4C39DFDE49CFCEEE9
:10EA580030E709B2D5E4C39FFFE49EFE12E9F33024
:0AEA6800D507C3E49FFFE49EFE22E1
:10EA7200BB0210E58229F582E5833AF583E0F5F0E1
:10EA8200A3E0224003BB0409E92582F886F008E6E8
:10EA920022400DE5832AF583E993F5F0A3E9932259
:0AEAA200E92582F8E2F5F008E2220F
:10EAAC00EF2531FFEE3530FEED352FFDEC352EFC2C
:03EABC0002ECF673
:10EABF00C3EF9531FFEE9530FEED952FFDEC952EC2
:04EACF00FC02ECF663
:10EAD300EFF88531F0A4FFE531C5F0CEF9A42EFEA1
:10EAE300E435F0CDFA88F0E530A42EFEED35F0FDE7
:10EAF300E433CC8531F0A42CFCE5308AF0A42CFC63
:10EB0300E52F89F0A42CFCE52E88F0A42CFC89F0D9
:10EB1300E530A42DFDEC35F0FCE52F88F0A42DFDA8
:10EB2300EC35F0FC8AF0E531A42DFDEC35F0FC0268
:02EB3300ECF6FE
:10EB3500E4CCF8E4CDF9E4CEFAE4CFFB75F020C3DC
:10EB4500E53133F531E53033F530E52F33F52FE594
:10EB55002E33F52EEF33FFEE33FEED33FDEC33FCB4
:10EB6500EF9BEE9AED99EC98400CFCEF9BFFEE9A2B
:0AEB7500FEED99FD0531D5F0C62232
:10F51C00C2D5EC30E70FB2D5E4C39FFFE49EFEE406
:10F52C009DFDE49CFCE52E30E705B2D512F54112A9
:10F53C00EB3530D515E4C39531F531E49530F53024
:0BF54C00E4952FF52FE4952EF52E22FC
:10EB7F00EF5531FFEE5530FEED552FFDEC552EFCC8
:03EB8F0002ECF69F
:10EB9200CFC531CFCEC530CECDC52FCDCCC52ECC35
:01EBA2002250
:0EEBA300C3E49FFFE49EFEE49DFDE49CFC2283
:10EBB100C3EF9531F8EE953048F8ED952F48F8EC14
:10EBC100952EA2E748F830D201B392D5D082D083F6
:0BEBD10012ECEEE8A2D5C083C0822247
:10EBDC00C3EF9531F8EE953048F8ED952F48F8ECE9
:10EBEC00952E48F892D5D082D08312ECEEE8A2D5BF
:05EBFC00C083C082226D
:10EC0100E86010ECA2E713FCED13FDEE13FEEF1329
:04EC1100FFD8F02216
:10EC1500E8600FEFC333FFEE33FEED33FDEC33FC5D
:03EC2500D8F12201
:10EC2800BB020789828A8302EC664003BB0405E9BC
:10EC3800F802ED76400789828A8302EC72E9F802CD
:02EC4800ED825B
:10EC4A00BB020789828A8302EC824003BB0405E97E
:0CEC5A00F802ED8E400122E9F802ED9A6C
:0CEC6600E0FCA3E0FDA3E0FEA3E0FF2221
:10EC7200E493FCA3E493FDA3E493FEA3E493FF22B5
:0CEC8200ECF0A3EDF0A3EEF0A3EFF02205
:10EC8E00A8828583F0D083D08212ECA512ECA51257
:10EC9E00ECA512ECA5E473E493A3C583C5F0C5837C
:10ECAE00C8C582C8F0A3C583C5F0C583C8C582C8D0
:01ECBE002233
:10ECBF00FAE6FB0808E6F925F0F618E6CA3AF62256
:10ECCF00E53A053A6010D0F0D0E0C02EC02FC0302A
:10ECDF00C031C0E0C0F08F318E308D2F8C2E22AF1F
:10ECEF0031AE30AD2FAC2EE53A146010D0F0D0E03D
:0FECFF00D031D030D02FD02EC0E0C0F0153A2247
:10ED0E00D0F0D0E0C02EC02FC030C031053AC0E0E8
:03ED1E00C0F02220
:10ED2100D083D082F8E4937012740193700DA3A381
:10ED310093F8740193F5828883E473740293686095
:06ED4100EFA3A3A380DF95
:10F55700EFB40A07740D12F562740A309811A8996E
:10F56700B8130CC2983098FDA899C298B811F63014
:07F5770099FDC299F59922EC
:10F57E008B538A548955E4FFFEAB530555E555AAC6
:10F58E00547002055414F912E98160070FEF7001EF
:04F59E000E80E622D3
:10ED4700EF4E6013EDBB021089828A83EF60010EDC
:10ED5700EDF0A3DFFCDEFA2289F04003BB0407F7DE
:0FED670009DFFCA9F02250EFF309DFFCA9F0222D
:0CED7600E6FC08E6FD08E6FE08E6FF22C9
:0CED8200E2FC08E2FD08E2FE08E2FF22CD
:0CED8E00ECF608EDF608EEF608EFF622B1
:0CED9A00ECF208EDF208EEF208EFF222B5
:00000001FF
